
hello_world.elf:     file format elf32-littlearm

Sections:
Idx Name          Size      VMA       LMA       File off  Algn
  0 .isr_vector   000000c0  08000000  08000000  00010000  2**0
                  CONTENTS, ALLOC, LOAD, READONLY, DATA
  1 .text         00002708  080000c0  080000c0  000100c0  2**2
                  CONTENTS, ALLOC, LOAD, READONLY, CODE
  2 .rodata       00000080  080027c8  080027c8  000127c8  2**2
                  CONTENTS, ALLOC, LOAD, READONLY, DATA
  3 .ARM.extab    00000000  08002848  08002848  0002000c  2**0
                  CONTENTS
  4 .ARM          00000008  08002848  08002848  00012848  2**2
                  CONTENTS, ALLOC, LOAD, READONLY, DATA
  5 .preinit_array 00000000  08002850  08002850  0002000c  2**0
                  CONTENTS, ALLOC, LOAD, DATA
  6 .init_array   00000004  08002850  08002850  00012850  2**2
                  CONTENTS, ALLOC, LOAD, DATA
  7 .fini_array   00000004  08002854  08002854  00012854  2**2
                  CONTENTS, ALLOC, LOAD, DATA
  8 .data         0000000c  20000000  08002858  00020000  2**2
                  CONTENTS, ALLOC, LOAD, DATA
  9 .bss          000000a8  2000000c  08002864  0002000c  2**2
                  ALLOC
 10 ._user_heap_stack 00000604  200000b4  08002864  000200b4  2**0
                  ALLOC
 11 .ARM.attributes 00000028  00000000  00000000  0002000c  2**0
                  CONTENTS, READONLY
 12 .debug_info   00008219  00000000  00000000  00020034  2**0
                  CONTENTS, READONLY, DEBUGGING, OCTETS
 13 .debug_abbrev 000013a7  00000000  00000000  0002824d  2**0
                  CONTENTS, READONLY, DEBUGGING, OCTETS
 14 .debug_aranges 00000698  00000000  00000000  000295f8  2**3
                  CONTENTS, READONLY, DEBUGGING, OCTETS
 15 .debug_ranges 00000620  00000000  00000000  00029c90  2**3
                  CONTENTS, READONLY, DEBUGGING, OCTETS
 16 .debug_macro  000131c8  00000000  00000000  0002a2b0  2**0
                  CONTENTS, READONLY, DEBUGGING, OCTETS
 17 .debug_line   0000858d  00000000  00000000  0003d478  2**0
                  CONTENTS, READONLY, DEBUGGING, OCTETS
 18 .debug_str    00077bb9  00000000  00000000  00045a05  2**0
                  CONTENTS, READONLY, DEBUGGING, OCTETS
 19 .comment      00000050  00000000  00000000  000bd5be  2**0
                  CONTENTS, READONLY
 20 .debug_frame  000016b8  00000000  00000000  000bd610  2**2
                  CONTENTS, READONLY, DEBUGGING, OCTETS

Disassembly of section .text:

080000c0 <__do_global_dtors_aux>:
 80000c0:	b510      	push	{r4, lr}
 80000c2:	4c06      	ldr	r4, [pc, #24]	; (80000dc <__do_global_dtors_aux+0x1c>)
 80000c4:	7823      	ldrb	r3, [r4, #0]
 80000c6:	2b00      	cmp	r3, #0
 80000c8:	d107      	bne.n	80000da <__do_global_dtors_aux+0x1a>
 80000ca:	4b05      	ldr	r3, [pc, #20]	; (80000e0 <__do_global_dtors_aux+0x20>)
 80000cc:	2b00      	cmp	r3, #0
 80000ce:	d002      	beq.n	80000d6 <__do_global_dtors_aux+0x16>
 80000d0:	4804      	ldr	r0, [pc, #16]	; (80000e4 <__do_global_dtors_aux+0x24>)
 80000d2:	e000      	b.n	80000d6 <__do_global_dtors_aux+0x16>
 80000d4:	bf00      	nop
 80000d6:	2301      	movs	r3, #1
 80000d8:	7023      	strb	r3, [r4, #0]
 80000da:	bd10      	pop	{r4, pc}
 80000dc:	2000000c 	.word	0x2000000c
 80000e0:	00000000 	.word	0x00000000
 80000e4:	080027b0 	.word	0x080027b0

080000e8 <frame_dummy>:
 80000e8:	4b04      	ldr	r3, [pc, #16]	; (80000fc <frame_dummy+0x14>)
 80000ea:	b510      	push	{r4, lr}
 80000ec:	2b00      	cmp	r3, #0
 80000ee:	d003      	beq.n	80000f8 <frame_dummy+0x10>
 80000f0:	4903      	ldr	r1, [pc, #12]	; (8000100 <frame_dummy+0x18>)
 80000f2:	4804      	ldr	r0, [pc, #16]	; (8000104 <frame_dummy+0x1c>)
 80000f4:	e000      	b.n	80000f8 <frame_dummy+0x10>
 80000f6:	bf00      	nop
 80000f8:	bd10      	pop	{r4, pc}
 80000fa:	46c0      	nop			; (mov r8, r8)
 80000fc:	00000000 	.word	0x00000000
 8000100:	20000010 	.word	0x20000010
 8000104:	080027b0 	.word	0x080027b0

08000108 <__udivsi3>:
 8000108:	2200      	movs	r2, #0
 800010a:	0843      	lsrs	r3, r0, #1
 800010c:	428b      	cmp	r3, r1
 800010e:	d374      	bcc.n	80001fa <__udivsi3+0xf2>
 8000110:	0903      	lsrs	r3, r0, #4
 8000112:	428b      	cmp	r3, r1
 8000114:	d35f      	bcc.n	80001d6 <__udivsi3+0xce>
 8000116:	0a03      	lsrs	r3, r0, #8
 8000118:	428b      	cmp	r3, r1
 800011a:	d344      	bcc.n	80001a6 <__udivsi3+0x9e>
 800011c:	0b03      	lsrs	r3, r0, #12
 800011e:	428b      	cmp	r3, r1
 8000120:	d328      	bcc.n	8000174 <__udivsi3+0x6c>
 8000122:	0c03      	lsrs	r3, r0, #16
 8000124:	428b      	cmp	r3, r1
 8000126:	d30d      	bcc.n	8000144 <__udivsi3+0x3c>
 8000128:	22ff      	movs	r2, #255	; 0xff
 800012a:	0209      	lsls	r1, r1, #8
 800012c:	ba12      	rev	r2, r2
 800012e:	0c03      	lsrs	r3, r0, #16
 8000130:	428b      	cmp	r3, r1
 8000132:	d302      	bcc.n	800013a <__udivsi3+0x32>
 8000134:	1212      	asrs	r2, r2, #8
 8000136:	0209      	lsls	r1, r1, #8
 8000138:	d065      	beq.n	8000206 <__udivsi3+0xfe>
 800013a:	0b03      	lsrs	r3, r0, #12
 800013c:	428b      	cmp	r3, r1
 800013e:	d319      	bcc.n	8000174 <__udivsi3+0x6c>
 8000140:	e000      	b.n	8000144 <__udivsi3+0x3c>
 8000142:	0a09      	lsrs	r1, r1, #8
 8000144:	0bc3      	lsrs	r3, r0, #15
 8000146:	428b      	cmp	r3, r1
 8000148:	d301      	bcc.n	800014e <__udivsi3+0x46>
 800014a:	03cb      	lsls	r3, r1, #15
 800014c:	1ac0      	subs	r0, r0, r3
 800014e:	4152      	adcs	r2, r2
 8000150:	0b83      	lsrs	r3, r0, #14
 8000152:	428b      	cmp	r3, r1
 8000154:	d301      	bcc.n	800015a <__udivsi3+0x52>
 8000156:	038b      	lsls	r3, r1, #14
 8000158:	1ac0      	subs	r0, r0, r3
 800015a:	4152      	adcs	r2, r2
 800015c:	0b43      	lsrs	r3, r0, #13
 800015e:	428b      	cmp	r3, r1
 8000160:	d301      	bcc.n	8000166 <__udivsi3+0x5e>
 8000162:	034b      	lsls	r3, r1, #13
 8000164:	1ac0      	subs	r0, r0, r3
 8000166:	4152      	adcs	r2, r2
 8000168:	0b03      	lsrs	r3, r0, #12
 800016a:	428b      	cmp	r3, r1
 800016c:	d301      	bcc.n	8000172 <__udivsi3+0x6a>
 800016e:	030b      	lsls	r3, r1, #12
 8000170:	1ac0      	subs	r0, r0, r3
 8000172:	4152      	adcs	r2, r2
 8000174:	0ac3      	lsrs	r3, r0, #11
 8000176:	428b      	cmp	r3, r1
 8000178:	d301      	bcc.n	800017e <__udivsi3+0x76>
 800017a:	02cb      	lsls	r3, r1, #11
 800017c:	1ac0      	subs	r0, r0, r3
 800017e:	4152      	adcs	r2, r2
 8000180:	0a83      	lsrs	r3, r0, #10
 8000182:	428b      	cmp	r3, r1
 8000184:	d301      	bcc.n	800018a <__udivsi3+0x82>
 8000186:	028b      	lsls	r3, r1, #10
 8000188:	1ac0      	subs	r0, r0, r3
 800018a:	4152      	adcs	r2, r2
 800018c:	0a43      	lsrs	r3, r0, #9
 800018e:	428b      	cmp	r3, r1
 8000190:	d301      	bcc.n	8000196 <__udivsi3+0x8e>
 8000192:	024b      	lsls	r3, r1, #9
 8000194:	1ac0      	subs	r0, r0, r3
 8000196:	4152      	adcs	r2, r2
 8000198:	0a03      	lsrs	r3, r0, #8
 800019a:	428b      	cmp	r3, r1
 800019c:	d301      	bcc.n	80001a2 <__udivsi3+0x9a>
 800019e:	020b      	lsls	r3, r1, #8
 80001a0:	1ac0      	subs	r0, r0, r3
 80001a2:	4152      	adcs	r2, r2
 80001a4:	d2cd      	bcs.n	8000142 <__udivsi3+0x3a>
 80001a6:	09c3      	lsrs	r3, r0, #7
 80001a8:	428b      	cmp	r3, r1
 80001aa:	d301      	bcc.n	80001b0 <__udivsi3+0xa8>
 80001ac:	01cb      	lsls	r3, r1, #7
 80001ae:	1ac0      	subs	r0, r0, r3
 80001b0:	4152      	adcs	r2, r2
 80001b2:	0983      	lsrs	r3, r0, #6
 80001b4:	428b      	cmp	r3, r1
 80001b6:	d301      	bcc.n	80001bc <__udivsi3+0xb4>
 80001b8:	018b      	lsls	r3, r1, #6
 80001ba:	1ac0      	subs	r0, r0, r3
 80001bc:	4152      	adcs	r2, r2
 80001be:	0943      	lsrs	r3, r0, #5
 80001c0:	428b      	cmp	r3, r1
 80001c2:	d301      	bcc.n	80001c8 <__udivsi3+0xc0>
 80001c4:	014b      	lsls	r3, r1, #5
 80001c6:	1ac0      	subs	r0, r0, r3
 80001c8:	4152      	adcs	r2, r2
 80001ca:	0903      	lsrs	r3, r0, #4
 80001cc:	428b      	cmp	r3, r1
 80001ce:	d301      	bcc.n	80001d4 <__udivsi3+0xcc>
 80001d0:	010b      	lsls	r3, r1, #4
 80001d2:	1ac0      	subs	r0, r0, r3
 80001d4:	4152      	adcs	r2, r2
 80001d6:	08c3      	lsrs	r3, r0, #3
 80001d8:	428b      	cmp	r3, r1
 80001da:	d301      	bcc.n	80001e0 <__udivsi3+0xd8>
 80001dc:	00cb      	lsls	r3, r1, #3
 80001de:	1ac0      	subs	r0, r0, r3
 80001e0:	4152      	adcs	r2, r2
 80001e2:	0883      	lsrs	r3, r0, #2
 80001e4:	428b      	cmp	r3, r1
 80001e6:	d301      	bcc.n	80001ec <__udivsi3+0xe4>
 80001e8:	008b      	lsls	r3, r1, #2
 80001ea:	1ac0      	subs	r0, r0, r3
 80001ec:	4152      	adcs	r2, r2
 80001ee:	0843      	lsrs	r3, r0, #1
 80001f0:	428b      	cmp	r3, r1
 80001f2:	d301      	bcc.n	80001f8 <__udivsi3+0xf0>
 80001f4:	004b      	lsls	r3, r1, #1
 80001f6:	1ac0      	subs	r0, r0, r3
 80001f8:	4152      	adcs	r2, r2
 80001fa:	1a41      	subs	r1, r0, r1
 80001fc:	d200      	bcs.n	8000200 <__udivsi3+0xf8>
 80001fe:	4601      	mov	r1, r0
 8000200:	4152      	adcs	r2, r2
 8000202:	4610      	mov	r0, r2
 8000204:	4770      	bx	lr
 8000206:	e7ff      	b.n	8000208 <__udivsi3+0x100>
 8000208:	b501      	push	{r0, lr}
 800020a:	2000      	movs	r0, #0
 800020c:	f000 f806 	bl	800021c <__aeabi_idiv0>
 8000210:	bd02      	pop	{r1, pc}
 8000212:	46c0      	nop			; (mov r8, r8)

08000214 <__aeabi_uidivmod>:
 8000214:	2900      	cmp	r1, #0
 8000216:	d0f7      	beq.n	8000208 <__udivsi3+0x100>
 8000218:	e776      	b.n	8000108 <__udivsi3>
 800021a:	4770      	bx	lr

0800021c <__aeabi_idiv0>:
 800021c:	4770      	bx	lr
 800021e:	46c0      	nop			; (mov r8, r8)

08000220 <__aeabi_uldivmod>:
 8000220:	2b00      	cmp	r3, #0
 8000222:	d111      	bne.n	8000248 <__aeabi_uldivmod+0x28>
 8000224:	2a00      	cmp	r2, #0
 8000226:	d10f      	bne.n	8000248 <__aeabi_uldivmod+0x28>
 8000228:	2900      	cmp	r1, #0
 800022a:	d100      	bne.n	800022e <__aeabi_uldivmod+0xe>
 800022c:	2800      	cmp	r0, #0
 800022e:	d002      	beq.n	8000236 <__aeabi_uldivmod+0x16>
 8000230:	2100      	movs	r1, #0
 8000232:	43c9      	mvns	r1, r1
 8000234:	0008      	movs	r0, r1
 8000236:	b407      	push	{r0, r1, r2}
 8000238:	4802      	ldr	r0, [pc, #8]	; (8000244 <__aeabi_uldivmod+0x24>)
 800023a:	a102      	add	r1, pc, #8	; (adr r1, 8000244 <__aeabi_uldivmod+0x24>)
 800023c:	1840      	adds	r0, r0, r1
 800023e:	9002      	str	r0, [sp, #8]
 8000240:	bd03      	pop	{r0, r1, pc}
 8000242:	46c0      	nop			; (mov r8, r8)
 8000244:	ffffffd9 	.word	0xffffffd9
 8000248:	b403      	push	{r0, r1}
 800024a:	4668      	mov	r0, sp
 800024c:	b501      	push	{r0, lr}
 800024e:	9802      	ldr	r0, [sp, #8]
 8000250:	f000 f834 	bl	80002bc <__udivmoddi4>
 8000254:	9b01      	ldr	r3, [sp, #4]
 8000256:	469e      	mov	lr, r3
 8000258:	b002      	add	sp, #8
 800025a:	bc0c      	pop	{r2, r3}
 800025c:	4770      	bx	lr
 800025e:	46c0      	nop			; (mov r8, r8)

08000260 <__aeabi_lmul>:
 8000260:	b5f0      	push	{r4, r5, r6, r7, lr}
 8000262:	46ce      	mov	lr, r9
 8000264:	4647      	mov	r7, r8
 8000266:	b580      	push	{r7, lr}
 8000268:	0007      	movs	r7, r0
 800026a:	4699      	mov	r9, r3
 800026c:	0c3b      	lsrs	r3, r7, #16
 800026e:	469c      	mov	ip, r3
 8000270:	0413      	lsls	r3, r2, #16
 8000272:	0c1b      	lsrs	r3, r3, #16
 8000274:	001d      	movs	r5, r3
 8000276:	000e      	movs	r6, r1
 8000278:	4661      	mov	r1, ip
 800027a:	0400      	lsls	r0, r0, #16
 800027c:	0c14      	lsrs	r4, r2, #16
 800027e:	0c00      	lsrs	r0, r0, #16
 8000280:	4345      	muls	r5, r0
 8000282:	434b      	muls	r3, r1
 8000284:	4360      	muls	r0, r4
 8000286:	4361      	muls	r1, r4
 8000288:	18c0      	adds	r0, r0, r3
 800028a:	0c2c      	lsrs	r4, r5, #16
 800028c:	1820      	adds	r0, r4, r0
 800028e:	468c      	mov	ip, r1
 8000290:	4283      	cmp	r3, r0
 8000292:	d903      	bls.n	800029c <__aeabi_lmul+0x3c>
 8000294:	2380      	movs	r3, #128	; 0x80
 8000296:	025b      	lsls	r3, r3, #9
 8000298:	4698      	mov	r8, r3
 800029a:	44c4      	add	ip, r8
 800029c:	4649      	mov	r1, r9
 800029e:	4379      	muls	r1, r7
 80002a0:	4372      	muls	r2, r6
 80002a2:	0c03      	lsrs	r3, r0, #16
 80002a4:	4463      	add	r3, ip
 80002a6:	042d      	lsls	r5, r5, #16
 80002a8:	0c2d      	lsrs	r5, r5, #16
 80002aa:	18c9      	adds	r1, r1, r3
 80002ac:	0400      	lsls	r0, r0, #16
 80002ae:	1940      	adds	r0, r0, r5
 80002b0:	1889      	adds	r1, r1, r2
 80002b2:	bcc0      	pop	{r6, r7}
 80002b4:	46b9      	mov	r9, r7
 80002b6:	46b0      	mov	r8, r6
 80002b8:	bdf0      	pop	{r4, r5, r6, r7, pc}
 80002ba:	46c0      	nop			; (mov r8, r8)

080002bc <__udivmoddi4>:
 80002bc:	b5f0      	push	{r4, r5, r6, r7, lr}
 80002be:	4657      	mov	r7, sl
 80002c0:	464e      	mov	r6, r9
 80002c2:	4645      	mov	r5, r8
 80002c4:	46de      	mov	lr, fp
 80002c6:	b5e0      	push	{r5, r6, r7, lr}
 80002c8:	0004      	movs	r4, r0
 80002ca:	000d      	movs	r5, r1
 80002cc:	4692      	mov	sl, r2
 80002ce:	4699      	mov	r9, r3
 80002d0:	b083      	sub	sp, #12
 80002d2:	428b      	cmp	r3, r1
 80002d4:	d830      	bhi.n	8000338 <__udivmoddi4+0x7c>
 80002d6:	d02d      	beq.n	8000334 <__udivmoddi4+0x78>
 80002d8:	4649      	mov	r1, r9
 80002da:	4650      	mov	r0, sl
 80002dc:	f000 f8ba 	bl	8000454 <__clzdi2>
 80002e0:	0029      	movs	r1, r5
 80002e2:	0006      	movs	r6, r0
 80002e4:	0020      	movs	r0, r4
 80002e6:	f000 f8b5 	bl	8000454 <__clzdi2>
 80002ea:	1a33      	subs	r3, r6, r0
 80002ec:	4698      	mov	r8, r3
 80002ee:	3b20      	subs	r3, #32
 80002f0:	469b      	mov	fp, r3
 80002f2:	d433      	bmi.n	800035c <__udivmoddi4+0xa0>
 80002f4:	465a      	mov	r2, fp
 80002f6:	4653      	mov	r3, sl
 80002f8:	4093      	lsls	r3, r2
 80002fa:	4642      	mov	r2, r8
 80002fc:	001f      	movs	r7, r3
 80002fe:	4653      	mov	r3, sl
 8000300:	4093      	lsls	r3, r2
 8000302:	001e      	movs	r6, r3
 8000304:	42af      	cmp	r7, r5
 8000306:	d83a      	bhi.n	800037e <__udivmoddi4+0xc2>
 8000308:	42af      	cmp	r7, r5
 800030a:	d100      	bne.n	800030e <__udivmoddi4+0x52>
 800030c:	e078      	b.n	8000400 <__udivmoddi4+0x144>
 800030e:	465b      	mov	r3, fp
 8000310:	1ba4      	subs	r4, r4, r6
 8000312:	41bd      	sbcs	r5, r7
 8000314:	2b00      	cmp	r3, #0
 8000316:	da00      	bge.n	800031a <__udivmoddi4+0x5e>
 8000318:	e075      	b.n	8000406 <__udivmoddi4+0x14a>
 800031a:	2200      	movs	r2, #0
 800031c:	2300      	movs	r3, #0
 800031e:	9200      	str	r2, [sp, #0]
 8000320:	9301      	str	r3, [sp, #4]
 8000322:	2301      	movs	r3, #1
 8000324:	465a      	mov	r2, fp
 8000326:	4093      	lsls	r3, r2
 8000328:	9301      	str	r3, [sp, #4]
 800032a:	2301      	movs	r3, #1
 800032c:	4642      	mov	r2, r8
 800032e:	4093      	lsls	r3, r2
 8000330:	9300      	str	r3, [sp, #0]
 8000332:	e028      	b.n	8000386 <__udivmoddi4+0xca>
 8000334:	4282      	cmp	r2, r0
 8000336:	d9cf      	bls.n	80002d8 <__udivmoddi4+0x1c>
 8000338:	2200      	movs	r2, #0
 800033a:	2300      	movs	r3, #0
 800033c:	9200      	str	r2, [sp, #0]
 800033e:	9301      	str	r3, [sp, #4]
 8000340:	9b0c      	ldr	r3, [sp, #48]	; 0x30
 8000342:	2b00      	cmp	r3, #0
 8000344:	d001      	beq.n	800034a <__udivmoddi4+0x8e>
 8000346:	601c      	str	r4, [r3, #0]
 8000348:	605d      	str	r5, [r3, #4]
 800034a:	9800      	ldr	r0, [sp, #0]
 800034c:	9901      	ldr	r1, [sp, #4]
 800034e:	b003      	add	sp, #12
 8000350:	bcf0      	pop	{r4, r5, r6, r7}
 8000352:	46bb      	mov	fp, r7
 8000354:	46b2      	mov	sl, r6
 8000356:	46a9      	mov	r9, r5
 8000358:	46a0      	mov	r8, r4
 800035a:	bdf0      	pop	{r4, r5, r6, r7, pc}
 800035c:	4642      	mov	r2, r8
 800035e:	2320      	movs	r3, #32
 8000360:	1a9b      	subs	r3, r3, r2
 8000362:	4652      	mov	r2, sl
 8000364:	40da      	lsrs	r2, r3
 8000366:	4641      	mov	r1, r8
 8000368:	0013      	movs	r3, r2
 800036a:	464a      	mov	r2, r9
 800036c:	408a      	lsls	r2, r1
 800036e:	0017      	movs	r7, r2
 8000370:	4642      	mov	r2, r8
 8000372:	431f      	orrs	r7, r3
 8000374:	4653      	mov	r3, sl
 8000376:	4093      	lsls	r3, r2
 8000378:	001e      	movs	r6, r3
 800037a:	42af      	cmp	r7, r5
 800037c:	d9c4      	bls.n	8000308 <__udivmoddi4+0x4c>
 800037e:	2200      	movs	r2, #0
 8000380:	2300      	movs	r3, #0
 8000382:	9200      	str	r2, [sp, #0]
 8000384:	9301      	str	r3, [sp, #4]
 8000386:	4643      	mov	r3, r8
 8000388:	2b00      	cmp	r3, #0
 800038a:	d0d9      	beq.n	8000340 <__udivmoddi4+0x84>
 800038c:	07fb      	lsls	r3, r7, #31
 800038e:	0872      	lsrs	r2, r6, #1
 8000390:	431a      	orrs	r2, r3
 8000392:	4646      	mov	r6, r8
 8000394:	087b      	lsrs	r3, r7, #1
 8000396:	e00e      	b.n	80003b6 <__udivmoddi4+0xfa>
 8000398:	42ab      	cmp	r3, r5
 800039a:	d101      	bne.n	80003a0 <__udivmoddi4+0xe4>
 800039c:	42a2      	cmp	r2, r4
 800039e:	d80c      	bhi.n	80003ba <__udivmoddi4+0xfe>
 80003a0:	1aa4      	subs	r4, r4, r2
 80003a2:	419d      	sbcs	r5, r3
 80003a4:	2001      	movs	r0, #1
 80003a6:	1924      	adds	r4, r4, r4
 80003a8:	416d      	adcs	r5, r5
 80003aa:	2100      	movs	r1, #0
 80003ac:	3e01      	subs	r6, #1
 80003ae:	1824      	adds	r4, r4, r0
 80003b0:	414d      	adcs	r5, r1
 80003b2:	2e00      	cmp	r6, #0
 80003b4:	d006      	beq.n	80003c4 <__udivmoddi4+0x108>
 80003b6:	42ab      	cmp	r3, r5
 80003b8:	d9ee      	bls.n	8000398 <__udivmoddi4+0xdc>
 80003ba:	3e01      	subs	r6, #1
 80003bc:	1924      	adds	r4, r4, r4
 80003be:	416d      	adcs	r5, r5
 80003c0:	2e00      	cmp	r6, #0
 80003c2:	d1f8      	bne.n	80003b6 <__udivmoddi4+0xfa>
 80003c4:	9800      	ldr	r0, [sp, #0]
 80003c6:	9901      	ldr	r1, [sp, #4]
 80003c8:	465b      	mov	r3, fp
 80003ca:	1900      	adds	r0, r0, r4
 80003cc:	4169      	adcs	r1, r5
 80003ce:	2b00      	cmp	r3, #0
 80003d0:	db24      	blt.n	800041c <__udivmoddi4+0x160>
 80003d2:	002b      	movs	r3, r5
 80003d4:	465a      	mov	r2, fp
 80003d6:	4644      	mov	r4, r8
 80003d8:	40d3      	lsrs	r3, r2
 80003da:	002a      	movs	r2, r5
 80003dc:	40e2      	lsrs	r2, r4
 80003de:	001c      	movs	r4, r3
 80003e0:	465b      	mov	r3, fp
 80003e2:	0015      	movs	r5, r2
 80003e4:	2b00      	cmp	r3, #0
 80003e6:	db2a      	blt.n	800043e <__udivmoddi4+0x182>
 80003e8:	0026      	movs	r6, r4
 80003ea:	409e      	lsls	r6, r3
 80003ec:	0033      	movs	r3, r6
 80003ee:	0026      	movs	r6, r4
 80003f0:	4647      	mov	r7, r8
 80003f2:	40be      	lsls	r6, r7
 80003f4:	0032      	movs	r2, r6
 80003f6:	1a80      	subs	r0, r0, r2
 80003f8:	4199      	sbcs	r1, r3
 80003fa:	9000      	str	r0, [sp, #0]
 80003fc:	9101      	str	r1, [sp, #4]
 80003fe:	e79f      	b.n	8000340 <__udivmoddi4+0x84>
 8000400:	42a3      	cmp	r3, r4
 8000402:	d8bc      	bhi.n	800037e <__udivmoddi4+0xc2>
 8000404:	e783      	b.n	800030e <__udivmoddi4+0x52>
 8000406:	4642      	mov	r2, r8
 8000408:	2320      	movs	r3, #32
 800040a:	2100      	movs	r1, #0
 800040c:	1a9b      	subs	r3, r3, r2
 800040e:	2200      	movs	r2, #0
 8000410:	9100      	str	r1, [sp, #0]
 8000412:	9201      	str	r2, [sp, #4]
 8000414:	2201      	movs	r2, #1
 8000416:	40da      	lsrs	r2, r3
 8000418:	9201      	str	r2, [sp, #4]
 800041a:	e786      	b.n	800032a <__udivmoddi4+0x6e>
 800041c:	4642      	mov	r2, r8
 800041e:	2320      	movs	r3, #32
 8000420:	1a9b      	subs	r3, r3, r2
 8000422:	002a      	movs	r2, r5
 8000424:	4646      	mov	r6, r8
 8000426:	409a      	lsls	r2, r3
 8000428:	0023      	movs	r3, r4
 800042a:	40f3      	lsrs	r3, r6
 800042c:	4644      	mov	r4, r8
 800042e:	4313      	orrs	r3, r2
 8000430:	002a      	movs	r2, r5
 8000432:	40e2      	lsrs	r2, r4
 8000434:	001c      	movs	r4, r3
 8000436:	465b      	mov	r3, fp
 8000438:	0015      	movs	r5, r2
 800043a:	2b00      	cmp	r3, #0
 800043c:	dad4      	bge.n	80003e8 <__udivmoddi4+0x12c>
 800043e:	4642      	mov	r2, r8
 8000440:	002f      	movs	r7, r5
 8000442:	2320      	movs	r3, #32
 8000444:	0026      	movs	r6, r4
 8000446:	4097      	lsls	r7, r2
 8000448:	1a9b      	subs	r3, r3, r2
 800044a:	40de      	lsrs	r6, r3
 800044c:	003b      	movs	r3, r7
 800044e:	4333      	orrs	r3, r6
 8000450:	e7cd      	b.n	80003ee <__udivmoddi4+0x132>
 8000452:	46c0      	nop			; (mov r8, r8)

08000454 <__clzdi2>:
 8000454:	b510      	push	{r4, lr}
 8000456:	2900      	cmp	r1, #0
 8000458:	d103      	bne.n	8000462 <__clzdi2+0xe>
 800045a:	f000 f807 	bl	800046c <__clzsi2>
 800045e:	3020      	adds	r0, #32
 8000460:	e002      	b.n	8000468 <__clzdi2+0x14>
 8000462:	0008      	movs	r0, r1
 8000464:	f000 f802 	bl	800046c <__clzsi2>
 8000468:	bd10      	pop	{r4, pc}
 800046a:	46c0      	nop			; (mov r8, r8)

0800046c <__clzsi2>:
 800046c:	211c      	movs	r1, #28
 800046e:	2301      	movs	r3, #1
 8000470:	041b      	lsls	r3, r3, #16
 8000472:	4298      	cmp	r0, r3
 8000474:	d301      	bcc.n	800047a <__clzsi2+0xe>
 8000476:	0c00      	lsrs	r0, r0, #16
 8000478:	3910      	subs	r1, #16
 800047a:	0a1b      	lsrs	r3, r3, #8
 800047c:	4298      	cmp	r0, r3
 800047e:	d301      	bcc.n	8000484 <__clzsi2+0x18>
 8000480:	0a00      	lsrs	r0, r0, #8
 8000482:	3908      	subs	r1, #8
 8000484:	091b      	lsrs	r3, r3, #4
 8000486:	4298      	cmp	r0, r3
 8000488:	d301      	bcc.n	800048e <__clzsi2+0x22>
 800048a:	0900      	lsrs	r0, r0, #4
 800048c:	3904      	subs	r1, #4
 800048e:	a202      	add	r2, pc, #8	; (adr r2, 8000498 <__clzsi2+0x2c>)
 8000490:	5c10      	ldrb	r0, [r2, r0]
 8000492:	1840      	adds	r0, r0, r1
 8000494:	4770      	bx	lr
 8000496:	46c0      	nop			; (mov r8, r8)
 8000498:	02020304 	.word	0x02020304
 800049c:	01010101 	.word	0x01010101
	...

080004a8 <main>:
/**
  * @brief  The application entry point.
  * @retval int
  */
int main(void)
{
 80004a8:	b590      	push	{r4, r7, lr}
 80004aa:	b087      	sub	sp, #28
 80004ac:	af00      	add	r7, sp, #0
  /* USER CODE END 1 */

  /* MCU Configuration--------------------------------------------------------*/

  /* Reset of all peripherals, Initializes the Flash interface and the Systick. */
  HAL_Init();
 80004ae:	f000 f97d 	bl	80007ac <HAL_Init>
  /* USER CODE BEGIN Init */

  /* USER CODE END Init */

  /* Configure the system clock */
  SystemClock_Config();
 80004b2:	f000 f81d 	bl	80004f0 <SystemClock_Config>
  /* USER CODE BEGIN SysInit */

  /* USER CODE END SysInit */

  /* Initialize all configured peripherals */
  MX_GPIO_Init();
 80004b6:	f000 f8bd 	bl	8000634 <MX_GPIO_Init>
  MX_USART2_UART_Init();
 80004ba:	f000 f88b 	bl	80005d4 <MX_USART2_UART_Init>
  /* Infinite loop */
  /* USER CODE BEGIN WHILE */
  while (1)
  {
    /* USER CODE END WHILE */
	  uint8_t Data[]= "have a great day\n";
 80004be:	1d3b      	adds	r3, r7, #4
 80004c0:	4a09      	ldr	r2, [pc, #36]	; (80004e8 <main+0x40>)
 80004c2:	ca13      	ldmia	r2!, {r0, r1, r4}
 80004c4:	c313      	stmia	r3!, {r0, r1, r4}
 80004c6:	6811      	ldr	r1, [r2, #0]
 80004c8:	6019      	str	r1, [r3, #0]
 80004ca:	8892      	ldrh	r2, [r2, #4]
 80004cc:	809a      	strh	r2, [r3, #4]
	  HAL_UART_Transmit(&huart2,Data,sizeof(Data),10);
 80004ce:	1d39      	adds	r1, r7, #4
 80004d0:	4806      	ldr	r0, [pc, #24]	; (80004ec <main+0x44>)
 80004d2:	230a      	movs	r3, #10
 80004d4:	2212      	movs	r2, #18
 80004d6:	f001 fbd7 	bl	8001c88 <HAL_UART_Transmit>
	  HAL_Delay(1000);
 80004da:	23fa      	movs	r3, #250	; 0xfa
 80004dc:	009b      	lsls	r3, r3, #2
 80004de:	0018      	movs	r0, r3
 80004e0:	f000 f9d4 	bl	800088c <HAL_Delay>
  {
 80004e4:	e7eb      	b.n	80004be <main+0x16>
 80004e6:	46c0      	nop			; (mov r8, r8)
 80004e8:	080027c8 	.word	0x080027c8
 80004ec:	20000028 	.word	0x20000028

080004f0 <SystemClock_Config>:
/**
  * @brief System Clock Configuration
  * @retval None
  */
void SystemClock_Config(void)
{
 80004f0:	b590      	push	{r4, r7, lr}
 80004f2:	b09d      	sub	sp, #116	; 0x74
 80004f4:	af00      	add	r7, sp, #0
  RCC_OscInitTypeDef RCC_OscInitStruct = {0};
 80004f6:	2438      	movs	r4, #56	; 0x38
 80004f8:	193b      	adds	r3, r7, r4
 80004fa:	0018      	movs	r0, r3
 80004fc:	2338      	movs	r3, #56	; 0x38
 80004fe:	001a      	movs	r2, r3
 8000500:	2100      	movs	r1, #0
 8000502:	f002 f94d 	bl	80027a0 <memset>
  RCC_ClkInitTypeDef RCC_ClkInitStruct = {0};
 8000506:	2324      	movs	r3, #36	; 0x24
 8000508:	18fb      	adds	r3, r7, r3
 800050a:	0018      	movs	r0, r3
 800050c:	2314      	movs	r3, #20
 800050e:	001a      	movs	r2, r3
 8000510:	2100      	movs	r1, #0
 8000512:	f002 f945 	bl	80027a0 <memset>
  RCC_PeriphCLKInitTypeDef PeriphClkInit = {0};
 8000516:	003b      	movs	r3, r7
 8000518:	0018      	movs	r0, r3
 800051a:	2324      	movs	r3, #36	; 0x24
 800051c:	001a      	movs	r2, r3
 800051e:	2100      	movs	r1, #0
 8000520:	f002 f93e 	bl	80027a0 <memset>

  /** Configure the main internal regulator output voltage
  */
  __HAL_PWR_VOLTAGESCALING_CONFIG(PWR_REGULATOR_VOLTAGE_SCALE1);
 8000524:	4b29      	ldr	r3, [pc, #164]	; (80005cc <SystemClock_Config+0xdc>)
 8000526:	681b      	ldr	r3, [r3, #0]
 8000528:	4a29      	ldr	r2, [pc, #164]	; (80005d0 <SystemClock_Config+0xe0>)
 800052a:	401a      	ands	r2, r3
 800052c:	4b27      	ldr	r3, [pc, #156]	; (80005cc <SystemClock_Config+0xdc>)
 800052e:	2180      	movs	r1, #128	; 0x80
 8000530:	0109      	lsls	r1, r1, #4
 8000532:	430a      	orrs	r2, r1
 8000534:	601a      	str	r2, [r3, #0]

  /** Initializes the RCC Oscillators according to the specified parameters
  * in the RCC_OscInitTypeDef structure.
  */
  RCC_OscInitStruct.OscillatorType = RCC_OSCILLATORTYPE_HSI;
 8000536:	0021      	movs	r1, r4
 8000538:	187b      	adds	r3, r7, r1
 800053a:	2202      	movs	r2, #2
 800053c:	601a      	str	r2, [r3, #0]
  RCC_OscInitStruct.HSIState = RCC_HSI_ON;
 800053e:	187b      	adds	r3, r7, r1
 8000540:	2201      	movs	r2, #1
 8000542:	60da      	str	r2, [r3, #12]
  RCC_OscInitStruct.HSICalibrationValue = RCC_HSICALIBRATION_DEFAULT;
 8000544:	187b      	adds	r3, r7, r1
 8000546:	2210      	movs	r2, #16
 8000548:	611a      	str	r2, [r3, #16]
  RCC_OscInitStruct.PLL.PLLState = RCC_PLL_ON;
 800054a:	187b      	adds	r3, r7, r1
 800054c:	2202      	movs	r2, #2
 800054e:	629a      	str	r2, [r3, #40]	; 0x28
  RCC_OscInitStruct.PLL.PLLSource = RCC_PLLSOURCE_HSI;
 8000550:	187b      	adds	r3, r7, r1
 8000552:	2200      	movs	r2, #0
 8000554:	62da      	str	r2, [r3, #44]	; 0x2c
  RCC_OscInitStruct.PLL.PLLMUL = RCC_PLLMUL_6;
 8000556:	187b      	adds	r3, r7, r1
 8000558:	2280      	movs	r2, #128	; 0x80
 800055a:	0312      	lsls	r2, r2, #12
 800055c:	631a      	str	r2, [r3, #48]	; 0x30
  RCC_OscInitStruct.PLL.PLLDIV = RCC_PLLDIV_3;
 800055e:	187b      	adds	r3, r7, r1
 8000560:	2280      	movs	r2, #128	; 0x80
 8000562:	0412      	lsls	r2, r2, #16
 8000564:	635a      	str	r2, [r3, #52]	; 0x34
  if (HAL_RCC_OscConfig(&RCC_OscInitStruct) != HAL_OK)
 8000566:	187b      	adds	r3, r7, r1
 8000568:	0018      	movs	r0, r3
 800056a:	f000 fbe5 	bl	8000d38 <HAL_RCC_OscConfig>
 800056e:	1e03      	subs	r3, r0, #0
 8000570:	d001      	beq.n	8000576 <SystemClock_Config+0x86>
  {
    Error_Handler();
 8000572:	f000 f875 	bl	8000660 <Error_Handler>
  }

  /** Initializes the CPU, AHB and APB buses clocks
  */
  RCC_ClkInitStruct.ClockType = RCC_CLOCKTYPE_HCLK|RCC_CLOCKTYPE_SYSCLK
 8000576:	2124      	movs	r1, #36	; 0x24
 8000578:	187b      	adds	r3, r7, r1
 800057a:	220f      	movs	r2, #15
 800057c:	601a      	str	r2, [r3, #0]
                              |RCC_CLOCKTYPE_PCLK1|RCC_CLOCKTYPE_PCLK2;
  RCC_ClkInitStruct.SYSCLKSource = RCC_SYSCLKSOURCE_PLLCLK;
 800057e:	187b      	adds	r3, r7, r1
 8000580:	2203      	movs	r2, #3
 8000582:	605a      	str	r2, [r3, #4]
  RCC_ClkInitStruct.AHBCLKDivider = RCC_SYSCLK_DIV1;
 8000584:	187b      	adds	r3, r7, r1
 8000586:	2200      	movs	r2, #0
 8000588:	609a      	str	r2, [r3, #8]
  RCC_ClkInitStruct.APB1CLKDivider = RCC_HCLK_DIV1;
 800058a:	187b      	adds	r3, r7, r1
 800058c:	2200      	movs	r2, #0
 800058e:	60da      	str	r2, [r3, #12]
  RCC_ClkInitStruct.APB2CLKDivider = RCC_HCLK_DIV1;
 8000590:	187b      	adds	r3, r7, r1
 8000592:	2200      	movs	r2, #0
 8000594:	611a      	str	r2, [r3, #16]

  if (HAL_RCC_ClockConfig(&RCC_ClkInitStruct, FLASH_LATENCY_1) != HAL_OK)
 8000596:	187b      	adds	r3, r7, r1
 8000598:	2101      	movs	r1, #1
 800059a:	0018      	movs	r0, r3
 800059c:	f000 ffa0 	bl	80014e0 <HAL_RCC_ClockConfig>
 80005a0:	1e03      	subs	r3, r0, #0
 80005a2:	d001      	beq.n	80005a8 <SystemClock_Config+0xb8>
  {
    Error_Handler();
 80005a4:	f000 f85c 	bl	8000660 <Error_Handler>
  }
  PeriphClkInit.PeriphClockSelection = RCC_PERIPHCLK_USART2;
 80005a8:	003b      	movs	r3, r7
 80005aa:	2202      	movs	r2, #2
 80005ac:	601a      	str	r2, [r3, #0]
  PeriphClkInit.Usart2ClockSelection = RCC_USART2CLKSOURCE_PCLK1;
 80005ae:	003b      	movs	r3, r7
 80005b0:	2200      	movs	r2, #0
 80005b2:	60da      	str	r2, [r3, #12]
  if (HAL_RCCEx_PeriphCLKConfig(&PeriphClkInit) != HAL_OK)
 80005b4:	003b      	movs	r3, r7
 80005b6:	0018      	movs	r0, r3
 80005b8:	f001 f9b6 	bl	8001928 <HAL_RCCEx_PeriphCLKConfig>
 80005bc:	1e03      	subs	r3, r0, #0
 80005be:	d001      	beq.n	80005c4 <SystemClock_Config+0xd4>
  {
    Error_Handler();
 80005c0:	f000 f84e 	bl	8000660 <Error_Handler>
  }
}
 80005c4:	46c0      	nop			; (mov r8, r8)
 80005c6:	46bd      	mov	sp, r7
 80005c8:	b01d      	add	sp, #116	; 0x74
 80005ca:	bd90      	pop	{r4, r7, pc}
 80005cc:	40007000 	.word	0x40007000
 80005d0:	ffffe7ff 	.word	0xffffe7ff

080005d4 <MX_USART2_UART_Init>:
  * @brief USART2 Initialization Function
  * @param None
  * @retval None
  */
static void MX_USART2_UART_Init(void)
{
 80005d4:	b580      	push	{r7, lr}
 80005d6:	af00      	add	r7, sp, #0
  /* USER CODE END USART2_Init 0 */

  /* USER CODE BEGIN USART2_Init 1 */

  /* USER CODE END USART2_Init 1 */
  huart2.Instance = USART2;
 80005d8:	4b14      	ldr	r3, [pc, #80]	; (800062c <MX_USART2_UART_Init+0x58>)
 80005da:	4a15      	ldr	r2, [pc, #84]	; (8000630 <MX_USART2_UART_Init+0x5c>)
 80005dc:	601a      	str	r2, [r3, #0]
  huart2.Init.BaudRate = 115200;
 80005de:	4b13      	ldr	r3, [pc, #76]	; (800062c <MX_USART2_UART_Init+0x58>)
 80005e0:	22e1      	movs	r2, #225	; 0xe1
 80005e2:	0252      	lsls	r2, r2, #9
 80005e4:	605a      	str	r2, [r3, #4]
  huart2.Init.WordLength = UART_WORDLENGTH_8B;
 80005e6:	4b11      	ldr	r3, [pc, #68]	; (800062c <MX_USART2_UART_Init+0x58>)
 80005e8:	2200      	movs	r2, #0
 80005ea:	609a      	str	r2, [r3, #8]
  huart2.Init.StopBits = UART_STOPBITS_1;
 80005ec:	4b0f      	ldr	r3, [pc, #60]	; (800062c <MX_USART2_UART_Init+0x58>)
 80005ee:	2200      	movs	r2, #0
 80005f0:	60da      	str	r2, [r3, #12]
  huart2.Init.Parity = UART_PARITY_NONE;
 80005f2:	4b0e      	ldr	r3, [pc, #56]	; (800062c <MX_USART2_UART_Init+0x58>)
 80005f4:	2200      	movs	r2, #0
 80005f6:	611a      	str	r2, [r3, #16]
  huart2.Init.Mode = UART_MODE_TX_RX;
 80005f8:	4b0c      	ldr	r3, [pc, #48]	; (800062c <MX_USART2_UART_Init+0x58>)
 80005fa:	220c      	movs	r2, #12
 80005fc:	615a      	str	r2, [r3, #20]
  huart2.Init.HwFlowCtl = UART_HWCONTROL_NONE;
 80005fe:	4b0b      	ldr	r3, [pc, #44]	; (800062c <MX_USART2_UART_Init+0x58>)
 8000600:	2200      	movs	r2, #0
 8000602:	619a      	str	r2, [r3, #24]
  huart2.Init.OverSampling = UART_OVERSAMPLING_16;
 8000604:	4b09      	ldr	r3, [pc, #36]	; (800062c <MX_USART2_UART_Init+0x58>)
 8000606:	2200      	movs	r2, #0
 8000608:	61da      	str	r2, [r3, #28]
  huart2.Init.OneBitSampling = UART_ONE_BIT_SAMPLE_DISABLE;
 800060a:	4b08      	ldr	r3, [pc, #32]	; (800062c <MX_USART2_UART_Init+0x58>)
 800060c:	2200      	movs	r2, #0
 800060e:	621a      	str	r2, [r3, #32]
  huart2.AdvancedInit.AdvFeatureInit = UART_ADVFEATURE_NO_INIT;
 8000610:	4b06      	ldr	r3, [pc, #24]	; (800062c <MX_USART2_UART_Init+0x58>)
 8000612:	2200      	movs	r2, #0
 8000614:	625a      	str	r2, [r3, #36]	; 0x24
  if (HAL_UART_Init(&huart2) != HAL_OK)
 8000616:	4b05      	ldr	r3, [pc, #20]	; (800062c <MX_USART2_UART_Init+0x58>)
 8000618:	0018      	movs	r0, r3
 800061a:	f001 fae1 	bl	8001be0 <HAL_UART_Init>
 800061e:	1e03      	subs	r3, r0, #0
 8000620:	d001      	beq.n	8000626 <MX_USART2_UART_Init+0x52>
  {
    Error_Handler();
 8000622:	f000 f81d 	bl	8000660 <Error_Handler>
  }
  /* USER CODE BEGIN USART2_Init 2 */

  /* USER CODE END USART2_Init 2 */

}
 8000626:	46c0      	nop			; (mov r8, r8)
 8000628:	46bd      	mov	sp, r7
 800062a:	bd80      	pop	{r7, pc}
 800062c:	20000028 	.word	0x20000028
 8000630:	40004400 	.word	0x40004400

08000634 <MX_GPIO_Init>:
  * @brief GPIO Initialization Function
  * @param None
  * @retval None
  */
static void MX_GPIO_Init(void)
{
 8000634:	b580      	push	{r7, lr}
 8000636:	b082      	sub	sp, #8
 8000638:	af00      	add	r7, sp, #0
/* USER CODE BEGIN MX_GPIO_Init_1 */
/* USER CODE END MX_GPIO_Init_1 */

  /* GPIO Ports Clock Enable */
  __HAL_RCC_GPIOA_CLK_ENABLE();
 800063a:	4b08      	ldr	r3, [pc, #32]	; (800065c <MX_GPIO_Init+0x28>)
 800063c:	6ada      	ldr	r2, [r3, #44]	; 0x2c
 800063e:	4b07      	ldr	r3, [pc, #28]	; (800065c <MX_GPIO_Init+0x28>)
 8000640:	2101      	movs	r1, #1
 8000642:	430a      	orrs	r2, r1
 8000644:	62da      	str	r2, [r3, #44]	; 0x2c
 8000646:	4b05      	ldr	r3, [pc, #20]	; (800065c <MX_GPIO_Init+0x28>)
 8000648:	6adb      	ldr	r3, [r3, #44]	; 0x2c
 800064a:	2201      	movs	r2, #1
 800064c:	4013      	ands	r3, r2
 800064e:	607b      	str	r3, [r7, #4]
 8000650:	687b      	ldr	r3, [r7, #4]

/* USER CODE BEGIN MX_GPIO_Init_2 */
/* USER CODE END MX_GPIO_Init_2 */
}
 8000652:	46c0      	nop			; (mov r8, r8)
 8000654:	46bd      	mov	sp, r7
 8000656:	b002      	add	sp, #8
 8000658:	bd80      	pop	{r7, pc}
 800065a:	46c0      	nop			; (mov r8, r8)
 800065c:	40021000 	.word	0x40021000

08000660 <Error_Handler>:
/**
  * @brief  This function is executed in case of error occurrence.
  * @retval None
  */
void Error_Handler(void)
{
 8000660:	b580      	push	{r7, lr}
 8000662:	af00      	add	r7, sp, #0
  \details Disables IRQ interrupts by setting the I-bit in the CPSR.
           Can only be executed in Privileged modes.
 */
__STATIC_FORCEINLINE void __disable_irq(void)
{
  __ASM volatile ("cpsid i" : : : "memory");
 8000664:	b672      	cpsid	i
}
 8000666:	46c0      	nop			; (mov r8, r8)
  /* USER CODE BEGIN Error_Handler_Debug */
  /* User can add his own implementation to report the HAL error return state */
  __disable_irq();
  while (1)
 8000668:	e7fe      	b.n	8000668 <Error_Handler+0x8>
	...

0800066c <HAL_MspInit>:
/* USER CODE END 0 */
/**
  * Initializes the Global MSP.
  */
void HAL_MspInit(void)
{
 800066c:	b580      	push	{r7, lr}
 800066e:	af00      	add	r7, sp, #0
  /* USER CODE BEGIN MspInit 0 */

  /* USER CODE END MspInit 0 */

  __HAL_RCC_SYSCFG_CLK_ENABLE();
 8000670:	4b07      	ldr	r3, [pc, #28]	; (8000690 <HAL_MspInit+0x24>)
 8000672:	6b5a      	ldr	r2, [r3, #52]	; 0x34
 8000674:	4b06      	ldr	r3, [pc, #24]	; (8000690 <HAL_MspInit+0x24>)
 8000676:	2101      	movs	r1, #1
 8000678:	430a      	orrs	r2, r1
 800067a:	635a      	str	r2, [r3, #52]	; 0x34
  __HAL_RCC_PWR_CLK_ENABLE();
 800067c:	4b04      	ldr	r3, [pc, #16]	; (8000690 <HAL_MspInit+0x24>)
 800067e:	6b9a      	ldr	r2, [r3, #56]	; 0x38
 8000680:	4b03      	ldr	r3, [pc, #12]	; (8000690 <HAL_MspInit+0x24>)
 8000682:	2180      	movs	r1, #128	; 0x80
 8000684:	0549      	lsls	r1, r1, #21
 8000686:	430a      	orrs	r2, r1
 8000688:	639a      	str	r2, [r3, #56]	; 0x38
  /* System interrupt init*/

  /* USER CODE BEGIN MspInit 1 */

  /* USER CODE END MspInit 1 */
}
 800068a:	46c0      	nop			; (mov r8, r8)
 800068c:	46bd      	mov	sp, r7
 800068e:	bd80      	pop	{r7, pc}
 8000690:	40021000 	.word	0x40021000

08000694 <HAL_UART_MspInit>:
* This function configures the hardware resources used in this example
* @param huart: UART handle pointer
* @retval None
*/
void HAL_UART_MspInit(UART_HandleTypeDef* huart)
{
 8000694:	b590      	push	{r4, r7, lr}
 8000696:	b089      	sub	sp, #36	; 0x24
 8000698:	af00      	add	r7, sp, #0
 800069a:	6078      	str	r0, [r7, #4]
  GPIO_InitTypeDef GPIO_InitStruct = {0};
 800069c:	240c      	movs	r4, #12
 800069e:	193b      	adds	r3, r7, r4
 80006a0:	0018      	movs	r0, r3
 80006a2:	2314      	movs	r3, #20
 80006a4:	001a      	movs	r2, r3
 80006a6:	2100      	movs	r1, #0
 80006a8:	f002 f87a 	bl	80027a0 <memset>
  if(huart->Instance==USART2)
 80006ac:	687b      	ldr	r3, [r7, #4]
 80006ae:	681b      	ldr	r3, [r3, #0]
 80006b0:	4a18      	ldr	r2, [pc, #96]	; (8000714 <HAL_UART_MspInit+0x80>)
 80006b2:	4293      	cmp	r3, r2
 80006b4:	d129      	bne.n	800070a <HAL_UART_MspInit+0x76>
  {
  /* USER CODE BEGIN USART2_MspInit 0 */

  /* USER CODE END USART2_MspInit 0 */
    /* Peripheral clock enable */
    __HAL_RCC_USART2_CLK_ENABLE();
 80006b6:	4b18      	ldr	r3, [pc, #96]	; (8000718 <HAL_UART_MspInit+0x84>)
 80006b8:	6b9a      	ldr	r2, [r3, #56]	; 0x38
 80006ba:	4b17      	ldr	r3, [pc, #92]	; (8000718 <HAL_UART_MspInit+0x84>)
 80006bc:	2180      	movs	r1, #128	; 0x80
 80006be:	0289      	lsls	r1, r1, #10
 80006c0:	430a      	orrs	r2, r1
 80006c2:	639a      	str	r2, [r3, #56]	; 0x38

    __HAL_RCC_GPIOA_CLK_ENABLE();
 80006c4:	4b14      	ldr	r3, [pc, #80]	; (8000718 <HAL_UART_MspInit+0x84>)
 80006c6:	6ada      	ldr	r2, [r3, #44]	; 0x2c
 80006c8:	4b13      	ldr	r3, [pc, #76]	; (8000718 <HAL_UART_MspInit+0x84>)
 80006ca:	2101      	movs	r1, #1
 80006cc:	430a      	orrs	r2, r1
 80006ce:	62da      	str	r2, [r3, #44]	; 0x2c
 80006d0:	4b11      	ldr	r3, [pc, #68]	; (8000718 <HAL_UART_MspInit+0x84>)
 80006d2:	6adb      	ldr	r3, [r3, #44]	; 0x2c
 80006d4:	2201      	movs	r2, #1
 80006d6:	4013      	ands	r3, r2
 80006d8:	60bb      	str	r3, [r7, #8]
 80006da:	68bb      	ldr	r3, [r7, #8]
    /**USART2 GPIO Configuration
    PA15     ------> USART2_RX
    PA2     ------> USART2_TX
    */
    GPIO_InitStruct.Pin = GPIO_PIN_15|GPIO_PIN_2;
 80006dc:	0021      	movs	r1, r4
 80006de:	187b      	adds	r3, r7, r1
 80006e0:	4a0e      	ldr	r2, [pc, #56]	; (800071c <HAL_UART_MspInit+0x88>)
 80006e2:	601a      	str	r2, [r3, #0]
    GPIO_InitStruct.Mode = GPIO_MODE_AF_PP;
 80006e4:	187b      	adds	r3, r7, r1
 80006e6:	2202      	movs	r2, #2
 80006e8:	605a      	str	r2, [r3, #4]
    GPIO_InitStruct.Pull = GPIO_NOPULL;
 80006ea:	187b      	adds	r3, r7, r1
 80006ec:	2200      	movs	r2, #0
 80006ee:	609a      	str	r2, [r3, #8]
    GPIO_InitStruct.Speed = GPIO_SPEED_FREQ_VERY_HIGH;
 80006f0:	187b      	adds	r3, r7, r1
 80006f2:	2203      	movs	r2, #3
 80006f4:	60da      	str	r2, [r3, #12]
    GPIO_InitStruct.Alternate = GPIO_AF4_USART2;
 80006f6:	187b      	adds	r3, r7, r1
 80006f8:	2204      	movs	r2, #4
 80006fa:	611a      	str	r2, [r3, #16]
    HAL_GPIO_Init(GPIOA, &GPIO_InitStruct);
 80006fc:	187a      	adds	r2, r7, r1
 80006fe:	23a0      	movs	r3, #160	; 0xa0
 8000700:	05db      	lsls	r3, r3, #23
 8000702:	0011      	movs	r1, r2
 8000704:	0018      	movs	r0, r3
 8000706:	f000 f999 	bl	8000a3c <HAL_GPIO_Init>
  /* USER CODE BEGIN USART2_MspInit 1 */

  /* USER CODE END USART2_MspInit 1 */
  }

}
 800070a:	46c0      	nop			; (mov r8, r8)
 800070c:	46bd      	mov	sp, r7
 800070e:	b009      	add	sp, #36	; 0x24
 8000710:	bd90      	pop	{r4, r7, pc}
 8000712:	46c0      	nop			; (mov r8, r8)
 8000714:	40004400 	.word	0x40004400
 8000718:	40021000 	.word	0x40021000
 800071c:	00008004 	.word	0x00008004

08000720 <NMI_Handler>:
/******************************************************************************/
/**
  * @brief This function handles Non maskable Interrupt.
  */
void NMI_Handler(void)
{
 8000720:	b580      	push	{r7, lr}
 8000722:	af00      	add	r7, sp, #0
  /* USER CODE BEGIN NonMaskableInt_IRQn 0 */

  /* USER CODE END NonMaskableInt_IRQn 0 */
  /* USER CODE BEGIN NonMaskableInt_IRQn 1 */
  while (1)
 8000724:	e7fe      	b.n	8000724 <NMI_Handler+0x4>

08000726 <HardFault_Handler>:

/**
  * @brief This function handles Hard fault interrupt.
  */
void HardFault_Handler(void)
{
 8000726:	b580      	push	{r7, lr}
 8000728:	af00      	add	r7, sp, #0
  /* USER CODE BEGIN HardFault_IRQn 0 */

  /* USER CODE END HardFault_IRQn 0 */
  while (1)
 800072a:	e7fe      	b.n	800072a <HardFault_Handler+0x4>

0800072c <SVC_Handler>:

/**
  * @brief This function handles System service call via SWI instruction.
  */
void SVC_Handler(void)
{
 800072c:	b580      	push	{r7, lr}
 800072e:	af00      	add	r7, sp, #0

  /* USER CODE END SVC_IRQn 0 */
  /* USER CODE BEGIN SVC_IRQn 1 */

  /* USER CODE END SVC_IRQn 1 */
}
 8000730:	46c0      	nop			; (mov r8, r8)
 8000732:	46bd      	mov	sp, r7
 8000734:	bd80      	pop	{r7, pc}

08000736 <PendSV_Handler>:

/**
  * @brief This function handles Pendable request for system service.
  */
void PendSV_Handler(void)
{
 8000736:	b580      	push	{r7, lr}
 8000738:	af00      	add	r7, sp, #0

  /* USER CODE END PendSV_IRQn 0 */
  /* USER CODE BEGIN PendSV_IRQn 1 */

  /* USER CODE END PendSV_IRQn 1 */
}
 800073a:	46c0      	nop			; (mov r8, r8)
 800073c:	46bd      	mov	sp, r7
 800073e:	bd80      	pop	{r7, pc}

08000740 <SysTick_Handler>:

/**
  * @brief This function handles System tick timer.
  */
void SysTick_Handler(void)
{
 8000740:	b580      	push	{r7, lr}
 8000742:	af00      	add	r7, sp, #0
  /* USER CODE BEGIN SysTick_IRQn 0 */

  /* USER CODE END SysTick_IRQn 0 */
  HAL_IncTick();
 8000744:	f000 f886 	bl	8000854 <HAL_IncTick>
  /* USER CODE BEGIN SysTick_IRQn 1 */

  /* USER CODE END SysTick_IRQn 1 */
}
 8000748:	46c0      	nop			; (mov r8, r8)
 800074a:	46bd      	mov	sp, r7
 800074c:	bd80      	pop	{r7, pc}

0800074e <SystemInit>:
  * @brief  Setup the microcontroller system.
  * @param  None
  * @retval None
  */
void SystemInit (void)
{
 800074e:	b580      	push	{r7, lr}
 8000750:	af00      	add	r7, sp, #0
  /* Configure the Vector Table location add offset address ------------------*/
#if defined (USER_VECT_TAB_ADDRESS)
  SCB->VTOR = VECT_TAB_BASE_ADDRESS | VECT_TAB_OFFSET; /* Vector Table Relocation in Internal SRAM */
#endif /* USER_VECT_TAB_ADDRESS */
}
 8000752:	46c0      	nop			; (mov r8, r8)
 8000754:	46bd      	mov	sp, r7
 8000756:	bd80      	pop	{r7, pc}

08000758 <Reset_Handler>:

    .section  .text.Reset_Handler
  .weak  Reset_Handler
  .type  Reset_Handler, %function
Reset_Handler:  
   ldr   r0, =_estack
 8000758:	480d      	ldr	r0, [pc, #52]	; (8000790 <LoopForever+0x2>)
   mov   sp, r0          /* set stack pointer */
 800075a:	4685      	mov	sp, r0
   
/* Call the clock system initialization function.*/
  bl  SystemInit
 800075c:	f7ff fff7 	bl	800074e <SystemInit>

/* Copy the data segment initializers from flash to SRAM */
  ldr r0, =_sdata
 8000760:	480c      	ldr	r0, [pc, #48]	; (8000794 <LoopForever+0x6>)
  ldr r1, =_edata
 8000762:	490d      	ldr	r1, [pc, #52]	; (8000798 <LoopForever+0xa>)
  ldr r2, =_sidata
 8000764:	4a0d      	ldr	r2, [pc, #52]	; (800079c <LoopForever+0xe>)
  movs r3, #0
 8000766:	2300      	movs	r3, #0
  b LoopCopyDataInit
 8000768:	e002      	b.n	8000770 <LoopCopyDataInit>

0800076a <CopyDataInit>:

CopyDataInit:
  ldr r4, [r2, r3]
 800076a:	58d4      	ldr	r4, [r2, r3]
  str r4, [r0, r3]
 800076c:	50c4      	str	r4, [r0, r3]
  adds r3, r3, #4
 800076e:	3304      	adds	r3, #4

08000770 <LoopCopyDataInit>:

LoopCopyDataInit:
  adds r4, r0, r3
 8000770:	18c4      	adds	r4, r0, r3
  cmp r4, r1
 8000772:	428c      	cmp	r4, r1
  bcc CopyDataInit
 8000774:	d3f9      	bcc.n	800076a <CopyDataInit>
  
/* Zero fill the bss segment. */
  ldr r2, =_sbss
 8000776:	4a0a      	ldr	r2, [pc, #40]	; (80007a0 <LoopForever+0x12>)
  ldr r4, =_ebss
 8000778:	4c0a      	ldr	r4, [pc, #40]	; (80007a4 <LoopForever+0x16>)
  movs r3, #0
 800077a:	2300      	movs	r3, #0
  b LoopFillZerobss
 800077c:	e001      	b.n	8000782 <LoopFillZerobss>

0800077e <FillZerobss>:

FillZerobss:
  str  r3, [r2]
 800077e:	6013      	str	r3, [r2, #0]
  adds r2, r2, #4
 8000780:	3204      	adds	r2, #4

08000782 <LoopFillZerobss>:

LoopFillZerobss:
  cmp r2, r4
 8000782:	42a2      	cmp	r2, r4
  bcc FillZerobss
 8000784:	d3fb      	bcc.n	800077e <FillZerobss>

/* Call static constructors */
    bl __libc_init_array
 8000786:	f001 ffe7 	bl	8002758 <__libc_init_array>
/* Call the application's entry point.*/
  bl  main
 800078a:	f7ff fe8d 	bl	80004a8 <main>

0800078e <LoopForever>:

LoopForever:
    b LoopForever
 800078e:	e7fe      	b.n	800078e <LoopForever>
   ldr   r0, =_estack
 8000790:	20005000 	.word	0x20005000
  ldr r0, =_sdata
 8000794:	20000000 	.word	0x20000000
  ldr r1, =_edata
 8000798:	2000000c 	.word	0x2000000c
  ldr r2, =_sidata
 800079c:	08002858 	.word	0x08002858
  ldr r2, =_sbss
 80007a0:	2000000c 	.word	0x2000000c
  ldr r4, =_ebss
 80007a4:	200000b4 	.word	0x200000b4

080007a8 <ADC1_COMP_IRQHandler>:
 * @retval : None
*/
    .section  .text.Default_Handler,"ax",%progbits
Default_Handler:
Infinite_Loop:
  b  Infinite_Loop
 80007a8:	e7fe      	b.n	80007a8 <ADC1_COMP_IRQHandler>
	...

080007ac <HAL_Init>:
  *        In the default implementation,Systick is used as source of time base.
  *        the tick variable is incremented each 1ms in its ISR.
  * @retval HAL status
  */
HAL_StatusTypeDef HAL_Init(void)
{
 80007ac:	b580      	push	{r7, lr}
 80007ae:	b082      	sub	sp, #8
 80007b0:	af00      	add	r7, sp, #0
  HAL_StatusTypeDef  status = HAL_OK;
 80007b2:	1dfb      	adds	r3, r7, #7
 80007b4:	2200      	movs	r2, #0
 80007b6:	701a      	strb	r2, [r3, #0]
#if (BUFFER_CACHE_DISABLE != 0)
  __HAL_FLASH_BUFFER_CACHE_DISABLE();
#endif /* BUFFER_CACHE_DISABLE */

#if (PREREAD_ENABLE != 0)
  __HAL_FLASH_PREREAD_BUFFER_ENABLE();
 80007b8:	4b0b      	ldr	r3, [pc, #44]	; (80007e8 <HAL_Init+0x3c>)
 80007ba:	681a      	ldr	r2, [r3, #0]
 80007bc:	4b0a      	ldr	r3, [pc, #40]	; (80007e8 <HAL_Init+0x3c>)
 80007be:	2140      	movs	r1, #64	; 0x40
 80007c0:	430a      	orrs	r2, r1
 80007c2:	601a      	str	r2, [r3, #0]
#if (PREFETCH_ENABLE != 0)
  __HAL_FLASH_PREFETCH_BUFFER_ENABLE();
#endif /* PREFETCH_ENABLE */

  /* Use SysTick as time base source and configure 1ms tick (default clock after Reset is MSI) */
  if (HAL_InitTick(TICK_INT_PRIORITY) != HAL_OK)
 80007c4:	2000      	movs	r0, #0
 80007c6:	f000 f811 	bl	80007ec <HAL_InitTick>
 80007ca:	1e03      	subs	r3, r0, #0
 80007cc:	d003      	beq.n	80007d6 <HAL_Init+0x2a>
  {
    status = HAL_ERROR;
 80007ce:	1dfb      	adds	r3, r7, #7
 80007d0:	2201      	movs	r2, #1
 80007d2:	701a      	strb	r2, [r3, #0]
 80007d4:	e001      	b.n	80007da <HAL_Init+0x2e>
  }
  else
  {
    /* Init the low level hardware */
    HAL_MspInit();
 80007d6:	f7ff ff49 	bl	800066c <HAL_MspInit>
  }

  /* Return function status */
  return status;
 80007da:	1dfb      	adds	r3, r7, #7
 80007dc:	781b      	ldrb	r3, [r3, #0]
}
 80007de:	0018      	movs	r0, r3
 80007e0:	46bd      	mov	sp, r7
 80007e2:	b002      	add	sp, #8
 80007e4:	bd80      	pop	{r7, pc}
 80007e6:	46c0      	nop			; (mov r8, r8)
 80007e8:	40022000 	.word	0x40022000

080007ec <HAL_InitTick>:
  *       implementation  in user file.
  * @param TickPriority Tick interrupt priority.
  * @retval HAL status
  */
__weak HAL_StatusTypeDef HAL_InitTick(uint32_t TickPriority)
{
 80007ec:	b590      	push	{r4, r7, lr}
 80007ee:	b083      	sub	sp, #12
 80007f0:	af00      	add	r7, sp, #0
 80007f2:	6078      	str	r0, [r7, #4]
  /* Configure the SysTick to have interrupt in 1ms time basis*/
  if (HAL_SYSTICK_Config(SystemCoreClock / (1000U / uwTickFreq)) > 0U)
 80007f4:	4b14      	ldr	r3, [pc, #80]	; (8000848 <HAL_InitTick+0x5c>)
 80007f6:	681c      	ldr	r4, [r3, #0]
 80007f8:	4b14      	ldr	r3, [pc, #80]	; (800084c <HAL_InitTick+0x60>)
 80007fa:	781b      	ldrb	r3, [r3, #0]
 80007fc:	0019      	movs	r1, r3
 80007fe:	23fa      	movs	r3, #250	; 0xfa
 8000800:	0098      	lsls	r0, r3, #2
 8000802:	f7ff fc81 	bl	8000108 <__udivsi3>
 8000806:	0003      	movs	r3, r0
 8000808:	0019      	movs	r1, r3
 800080a:	0020      	movs	r0, r4
 800080c:	f7ff fc7c 	bl	8000108 <__udivsi3>
 8000810:	0003      	movs	r3, r0
 8000812:	0018      	movs	r0, r3
 8000814:	f000 f905 	bl	8000a22 <HAL_SYSTICK_Config>
 8000818:	1e03      	subs	r3, r0, #0
 800081a:	d001      	beq.n	8000820 <HAL_InitTick+0x34>
  {
    return HAL_ERROR;
 800081c:	2301      	movs	r3, #1
 800081e:	e00f      	b.n	8000840 <HAL_InitTick+0x54>
  }

  /* Configure the SysTick IRQ priority */
  if (TickPriority < (1UL << __NVIC_PRIO_BITS))
 8000820:	687b      	ldr	r3, [r7, #4]
 8000822:	2b03      	cmp	r3, #3
 8000824:	d80b      	bhi.n	800083e <HAL_InitTick+0x52>
  {
    HAL_NVIC_SetPriority(SysTick_IRQn, TickPriority, 0U);
 8000826:	6879      	ldr	r1, [r7, #4]
 8000828:	2301      	movs	r3, #1
 800082a:	425b      	negs	r3, r3
 800082c:	2200      	movs	r2, #0
 800082e:	0018      	movs	r0, r3
 8000830:	f000 f8e2 	bl	80009f8 <HAL_NVIC_SetPriority>
    uwTickPrio = TickPriority;
 8000834:	4b06      	ldr	r3, [pc, #24]	; (8000850 <HAL_InitTick+0x64>)
 8000836:	687a      	ldr	r2, [r7, #4]
 8000838:	601a      	str	r2, [r3, #0]
  {
    return HAL_ERROR;
  }

  /* Return function status */
  return HAL_OK;
 800083a:	2300      	movs	r3, #0
 800083c:	e000      	b.n	8000840 <HAL_InitTick+0x54>
    return HAL_ERROR;
 800083e:	2301      	movs	r3, #1
}
 8000840:	0018      	movs	r0, r3
 8000842:	46bd      	mov	sp, r7
 8000844:	b003      	add	sp, #12
 8000846:	bd90      	pop	{r4, r7, pc}
 8000848:	20000000 	.word	0x20000000
 800084c:	20000008 	.word	0x20000008
 8000850:	20000004 	.word	0x20000004

08000854 <HAL_IncTick>:
 * @note This function is declared as __weak to be overwritten in case of other
  *      implementations in user file.
  * @retval None
  */
__weak void HAL_IncTick(void)
{
 8000854:	b580      	push	{r7, lr}
 8000856:	af00      	add	r7, sp, #0
  uwTick += uwTickFreq;
 8000858:	4b05      	ldr	r3, [pc, #20]	; (8000870 <HAL_IncTick+0x1c>)
 800085a:	781b      	ldrb	r3, [r3, #0]
 800085c:	001a      	movs	r2, r3
 800085e:	4b05      	ldr	r3, [pc, #20]	; (8000874 <HAL_IncTick+0x20>)
 8000860:	681b      	ldr	r3, [r3, #0]
 8000862:	18d2      	adds	r2, r2, r3
 8000864:	4b03      	ldr	r3, [pc, #12]	; (8000874 <HAL_IncTick+0x20>)
 8000866:	601a      	str	r2, [r3, #0]
}
 8000868:	46c0      	nop			; (mov r8, r8)
 800086a:	46bd      	mov	sp, r7
 800086c:	bd80      	pop	{r7, pc}
 800086e:	46c0      	nop			; (mov r8, r8)
 8000870:	20000008 	.word	0x20000008
 8000874:	200000b0 	.word	0x200000b0

08000878 <HAL_GetTick>:
  * @note This function is declared as __weak to be overwritten in case of other
  *       implementations in user file.
  * @retval tick value
  */
__weak uint32_t HAL_GetTick(void)
{
 8000878:	b580      	push	{r7, lr}
 800087a:	af00      	add	r7, sp, #0
  return uwTick;
 800087c:	4b02      	ldr	r3, [pc, #8]	; (8000888 <HAL_GetTick+0x10>)
 800087e:	681b      	ldr	r3, [r3, #0]
}
 8000880:	0018      	movs	r0, r3
 8000882:	46bd      	mov	sp, r7
 8000884:	bd80      	pop	{r7, pc}
 8000886:	46c0      	nop			; (mov r8, r8)
 8000888:	200000b0 	.word	0x200000b0

0800088c <HAL_Delay>:
  *       implementations in user file.
  * @param Delay specifies the delay time length, in milliseconds.
  * @retval None
  */
__weak void HAL_Delay(uint32_t Delay)
{
 800088c:	b580      	push	{r7, lr}
 800088e:	b084      	sub	sp, #16
 8000890:	af00      	add	r7, sp, #0
 8000892:	6078      	str	r0, [r7, #4]
  uint32_t tickstart = HAL_GetTick();
 8000894:	f7ff fff0 	bl	8000878 <HAL_GetTick>
 8000898:	0003      	movs	r3, r0
 800089a:	60bb      	str	r3, [r7, #8]
  uint32_t wait = Delay;
 800089c:	687b      	ldr	r3, [r7, #4]
 800089e:	60fb      	str	r3, [r7, #12]

  /* Add a freq to guarantee minimum wait */
  if (wait < HAL_MAX_DELAY)
 80008a0:	68fb      	ldr	r3, [r7, #12]
 80008a2:	3301      	adds	r3, #1
 80008a4:	d005      	beq.n	80008b2 <HAL_Delay+0x26>
  {
    wait += (uint32_t)(uwTickFreq);
 80008a6:	4b0a      	ldr	r3, [pc, #40]	; (80008d0 <HAL_Delay+0x44>)
 80008a8:	781b      	ldrb	r3, [r3, #0]
 80008aa:	001a      	movs	r2, r3
 80008ac:	68fb      	ldr	r3, [r7, #12]
 80008ae:	189b      	adds	r3, r3, r2
 80008b0:	60fb      	str	r3, [r7, #12]
  }

  while((HAL_GetTick() - tickstart) < wait)
 80008b2:	46c0      	nop			; (mov r8, r8)
 80008b4:	f7ff ffe0 	bl	8000878 <HAL_GetTick>
 80008b8:	0002      	movs	r2, r0
 80008ba:	68bb      	ldr	r3, [r7, #8]
 80008bc:	1ad3      	subs	r3, r2, r3
 80008be:	68fa      	ldr	r2, [r7, #12]
 80008c0:	429a      	cmp	r2, r3
 80008c2:	d8f7      	bhi.n	80008b4 <HAL_Delay+0x28>
  {
  }
}
 80008c4:	46c0      	nop			; (mov r8, r8)
 80008c6:	46c0      	nop			; (mov r8, r8)
 80008c8:	46bd      	mov	sp, r7
 80008ca:	b004      	add	sp, #16
 80008cc:	bd80      	pop	{r7, pc}
 80008ce:	46c0      	nop			; (mov r8, r8)
 80008d0:	20000008 	.word	0x20000008

080008d4 <__NVIC_SetPriority>:
  \param [in]      IRQn  Interrupt number.
  \param [in]  priority  Priority to set.
  \note    The priority cannot be set for every processor exception.
 */
__STATIC_INLINE void __NVIC_SetPriority(IRQn_Type IRQn, uint32_t priority)
{
 80008d4:	b590      	push	{r4, r7, lr}
 80008d6:	b083      	sub	sp, #12
 80008d8:	af00      	add	r7, sp, #0
 80008da:	0002      	movs	r2, r0
 80008dc:	6039      	str	r1, [r7, #0]
 80008de:	1dfb      	adds	r3, r7, #7
 80008e0:	701a      	strb	r2, [r3, #0]
  if ((int32_t)(IRQn) >= 0)
 80008e2:	1dfb      	adds	r3, r7, #7
 80008e4:	781b      	ldrb	r3, [r3, #0]
 80008e6:	2b7f      	cmp	r3, #127	; 0x7f
 80008e8:	d828      	bhi.n	800093c <__NVIC_SetPriority+0x68>
  {
    NVIC->IP[_IP_IDX(IRQn)]  = ((uint32_t)(NVIC->IP[_IP_IDX(IRQn)]  & ~(0xFFUL << _BIT_SHIFT(IRQn))) |
 80008ea:	4a2f      	ldr	r2, [pc, #188]	; (80009a8 <__NVIC_SetPriority+0xd4>)
 80008ec:	1dfb      	adds	r3, r7, #7
 80008ee:	781b      	ldrb	r3, [r3, #0]
 80008f0:	b25b      	sxtb	r3, r3
 80008f2:	089b      	lsrs	r3, r3, #2
 80008f4:	33c0      	adds	r3, #192	; 0xc0
 80008f6:	009b      	lsls	r3, r3, #2
 80008f8:	589b      	ldr	r3, [r3, r2]
 80008fa:	1dfa      	adds	r2, r7, #7
 80008fc:	7812      	ldrb	r2, [r2, #0]
 80008fe:	0011      	movs	r1, r2
 8000900:	2203      	movs	r2, #3
 8000902:	400a      	ands	r2, r1
 8000904:	00d2      	lsls	r2, r2, #3
 8000906:	21ff      	movs	r1, #255	; 0xff
 8000908:	4091      	lsls	r1, r2
 800090a:	000a      	movs	r2, r1
 800090c:	43d2      	mvns	r2, r2
 800090e:	401a      	ands	r2, r3
 8000910:	0011      	movs	r1, r2
       (((priority << (8U - __NVIC_PRIO_BITS)) & (uint32_t)0xFFUL) << _BIT_SHIFT(IRQn)));
 8000912:	683b      	ldr	r3, [r7, #0]
 8000914:	019b      	lsls	r3, r3, #6
 8000916:	22ff      	movs	r2, #255	; 0xff
 8000918:	401a      	ands	r2, r3
 800091a:	1dfb      	adds	r3, r7, #7
 800091c:	781b      	ldrb	r3, [r3, #0]
 800091e:	0018      	movs	r0, r3
 8000920:	2303      	movs	r3, #3
 8000922:	4003      	ands	r3, r0
 8000924:	00db      	lsls	r3, r3, #3
 8000926:	409a      	lsls	r2, r3
    NVIC->IP[_IP_IDX(IRQn)]  = ((uint32_t)(NVIC->IP[_IP_IDX(IRQn)]  & ~(0xFFUL << _BIT_SHIFT(IRQn))) |
 8000928:	481f      	ldr	r0, [pc, #124]	; (80009a8 <__NVIC_SetPriority+0xd4>)
 800092a:	1dfb      	adds	r3, r7, #7
 800092c:	781b      	ldrb	r3, [r3, #0]
 800092e:	b25b      	sxtb	r3, r3
 8000930:	089b      	lsrs	r3, r3, #2
 8000932:	430a      	orrs	r2, r1
 8000934:	33c0      	adds	r3, #192	; 0xc0
 8000936:	009b      	lsls	r3, r3, #2
 8000938:	501a      	str	r2, [r3, r0]
  else
  {
    SCB->SHP[_SHP_IDX(IRQn)] = ((uint32_t)(SCB->SHP[_SHP_IDX(IRQn)] & ~(0xFFUL << _BIT_SHIFT(IRQn))) |
       (((priority << (8U - __NVIC_PRIO_BITS)) & (uint32_t)0xFFUL) << _BIT_SHIFT(IRQn)));
  }
}
 800093a:	e031      	b.n	80009a0 <__NVIC_SetPriority+0xcc>
    SCB->SHP[_SHP_IDX(IRQn)] = ((uint32_t)(SCB->SHP[_SHP_IDX(IRQn)] & ~(0xFFUL << _BIT_SHIFT(IRQn))) |
 800093c:	4a1b      	ldr	r2, [pc, #108]	; (80009ac <__NVIC_SetPriority+0xd8>)
 800093e:	1dfb      	adds	r3, r7, #7
 8000940:	781b      	ldrb	r3, [r3, #0]
 8000942:	0019      	movs	r1, r3
 8000944:	230f      	movs	r3, #15
 8000946:	400b      	ands	r3, r1
 8000948:	3b08      	subs	r3, #8
 800094a:	089b      	lsrs	r3, r3, #2
 800094c:	3306      	adds	r3, #6
 800094e:	009b      	lsls	r3, r3, #2
 8000950:	18d3      	adds	r3, r2, r3
 8000952:	3304      	adds	r3, #4
 8000954:	681b      	ldr	r3, [r3, #0]
 8000956:	1dfa      	adds	r2, r7, #7
 8000958:	7812      	ldrb	r2, [r2, #0]
 800095a:	0011      	movs	r1, r2
 800095c:	2203      	movs	r2, #3
 800095e:	400a      	ands	r2, r1
 8000960:	00d2      	lsls	r2, r2, #3
 8000962:	21ff      	movs	r1, #255	; 0xff
 8000964:	4091      	lsls	r1, r2
 8000966:	000a      	movs	r2, r1
 8000968:	43d2      	mvns	r2, r2
 800096a:	401a      	ands	r2, r3
 800096c:	0011      	movs	r1, r2
       (((priority << (8U - __NVIC_PRIO_BITS)) & (uint32_t)0xFFUL) << _BIT_SHIFT(IRQn)));
 800096e:	683b      	ldr	r3, [r7, #0]
 8000970:	019b      	lsls	r3, r3, #6
 8000972:	22ff      	movs	r2, #255	; 0xff
 8000974:	401a      	ands	r2, r3
 8000976:	1dfb      	adds	r3, r7, #7
 8000978:	781b      	ldrb	r3, [r3, #0]
 800097a:	0018      	movs	r0, r3
 800097c:	2303      	movs	r3, #3
 800097e:	4003      	ands	r3, r0
 8000980:	00db      	lsls	r3, r3, #3
 8000982:	409a      	lsls	r2, r3
    SCB->SHP[_SHP_IDX(IRQn)] = ((uint32_t)(SCB->SHP[_SHP_IDX(IRQn)] & ~(0xFFUL << _BIT_SHIFT(IRQn))) |
 8000984:	4809      	ldr	r0, [pc, #36]	; (80009ac <__NVIC_SetPriority+0xd8>)
 8000986:	1dfb      	adds	r3, r7, #7
 8000988:	781b      	ldrb	r3, [r3, #0]
 800098a:	001c      	movs	r4, r3
 800098c:	230f      	movs	r3, #15
 800098e:	4023      	ands	r3, r4
 8000990:	3b08      	subs	r3, #8
 8000992:	089b      	lsrs	r3, r3, #2
 8000994:	430a      	orrs	r2, r1
 8000996:	3306      	adds	r3, #6
 8000998:	009b      	lsls	r3, r3, #2
 800099a:	18c3      	adds	r3, r0, r3
 800099c:	3304      	adds	r3, #4
 800099e:	601a      	str	r2, [r3, #0]
}
 80009a0:	46c0      	nop			; (mov r8, r8)
 80009a2:	46bd      	mov	sp, r7
 80009a4:	b003      	add	sp, #12
 80009a6:	bd90      	pop	{r4, r7, pc}
 80009a8:	e000e100 	.word	0xe000e100
 80009ac:	e000ed00 	.word	0xe000ed00

080009b0 <SysTick_Config>:
  \note    When the variable <b>__Vendor_SysTickConfig</b> is set to 1, then the
           function <b>SysTick_Config</b> is not included. In this case, the file <b><i>device</i>.h</b>
           must contain a vendor-specific implementation of this function.
 */
__STATIC_INLINE uint32_t SysTick_Config(uint32_t ticks)
{
 80009b0:	b580      	push	{r7, lr}
 80009b2:	b082      	sub	sp, #8
 80009b4:	af00      	add	r7, sp, #0
 80009b6:	6078      	str	r0, [r7, #4]
  if ((ticks - 1UL) > SysTick_LOAD_RELOAD_Msk)
 80009b8:	687b      	ldr	r3, [r7, #4]
 80009ba:	1e5a      	subs	r2, r3, #1
 80009bc:	2380      	movs	r3, #128	; 0x80
 80009be:	045b      	lsls	r3, r3, #17
 80009c0:	429a      	cmp	r2, r3
 80009c2:	d301      	bcc.n	80009c8 <SysTick_Config+0x18>
  {
    return (1UL);                                                   /* Reload value impossible */
 80009c4:	2301      	movs	r3, #1
 80009c6:	e010      	b.n	80009ea <SysTick_Config+0x3a>
  }

  SysTick->LOAD  = (uint32_t)(ticks - 1UL);                         /* set reload register */
 80009c8:	4b0a      	ldr	r3, [pc, #40]	; (80009f4 <SysTick_Config+0x44>)
 80009ca:	687a      	ldr	r2, [r7, #4]
 80009cc:	3a01      	subs	r2, #1
 80009ce:	605a      	str	r2, [r3, #4]
  NVIC_SetPriority (SysTick_IRQn, (1UL << __NVIC_PRIO_BITS) - 1UL); /* set Priority for Systick Interrupt */
 80009d0:	2301      	movs	r3, #1
 80009d2:	425b      	negs	r3, r3
 80009d4:	2103      	movs	r1, #3
 80009d6:	0018      	movs	r0, r3
 80009d8:	f7ff ff7c 	bl	80008d4 <__NVIC_SetPriority>
  SysTick->VAL   = 0UL;                                             /* Load the SysTick Counter Value */
 80009dc:	4b05      	ldr	r3, [pc, #20]	; (80009f4 <SysTick_Config+0x44>)
 80009de:	2200      	movs	r2, #0
 80009e0:	609a      	str	r2, [r3, #8]
  SysTick->CTRL  = SysTick_CTRL_CLKSOURCE_Msk |
 80009e2:	4b04      	ldr	r3, [pc, #16]	; (80009f4 <SysTick_Config+0x44>)
 80009e4:	2207      	movs	r2, #7
 80009e6:	601a      	str	r2, [r3, #0]
                   SysTick_CTRL_TICKINT_Msk   |
                   SysTick_CTRL_ENABLE_Msk;                         /* Enable SysTick IRQ and SysTick Timer */
  return (0UL);                                                     /* Function successful */
 80009e8:	2300      	movs	r3, #0
}
 80009ea:	0018      	movs	r0, r3
 80009ec:	46bd      	mov	sp, r7
 80009ee:	b002      	add	sp, #8
 80009f0:	bd80      	pop	{r7, pc}
 80009f2:	46c0      	nop			; (mov r8, r8)
 80009f4:	e000e010 	.word	0xe000e010

080009f8 <HAL_NVIC_SetPriority>:
  *         with stm32l0xx devices, this parameter is a dummy value and it is ignored, because 
  *         no subpriority supported in Cortex M0+ based products.   
  * @retval None
  */
void HAL_NVIC_SetPriority(IRQn_Type IRQn, uint32_t PreemptPriority, uint32_t SubPriority)
{ 
 80009f8:	b580      	push	{r7, lr}
 80009fa:	b084      	sub	sp, #16
 80009fc:	af00      	add	r7, sp, #0
 80009fe:	60b9      	str	r1, [r7, #8]
 8000a00:	607a      	str	r2, [r7, #4]
 8000a02:	210f      	movs	r1, #15
 8000a04:	187b      	adds	r3, r7, r1
 8000a06:	1c02      	adds	r2, r0, #0
 8000a08:	701a      	strb	r2, [r3, #0]
    /* Check the parameters */
  assert_param(IS_NVIC_PREEMPTION_PRIORITY(PreemptPriority));
  NVIC_SetPriority(IRQn,PreemptPriority);
 8000a0a:	68ba      	ldr	r2, [r7, #8]
 8000a0c:	187b      	adds	r3, r7, r1
 8000a0e:	781b      	ldrb	r3, [r3, #0]
 8000a10:	b25b      	sxtb	r3, r3
 8000a12:	0011      	movs	r1, r2
 8000a14:	0018      	movs	r0, r3
 8000a16:	f7ff ff5d 	bl	80008d4 <__NVIC_SetPriority>
}
 8000a1a:	46c0      	nop			; (mov r8, r8)
 8000a1c:	46bd      	mov	sp, r7
 8000a1e:	b004      	add	sp, #16
 8000a20:	bd80      	pop	{r7, pc}

08000a22 <HAL_SYSTICK_Config>:
  * @param  TicksNumb Specifies the ticks Number of ticks between two interrupts.
  * @retval status:  - 0  Function succeeded.
  *                  - 1  Function failed.
  */
uint32_t HAL_SYSTICK_Config(uint32_t TicksNumb)
{
 8000a22:	b580      	push	{r7, lr}
 8000a24:	b082      	sub	sp, #8
 8000a26:	af00      	add	r7, sp, #0
 8000a28:	6078      	str	r0, [r7, #4]
   return SysTick_Config(TicksNumb);
 8000a2a:	687b      	ldr	r3, [r7, #4]
 8000a2c:	0018      	movs	r0, r3
 8000a2e:	f7ff ffbf 	bl	80009b0 <SysTick_Config>
 8000a32:	0003      	movs	r3, r0
}
 8000a34:	0018      	movs	r0, r3
 8000a36:	46bd      	mov	sp, r7
 8000a38:	b002      	add	sp, #8
 8000a3a:	bd80      	pop	{r7, pc}

08000a3c <HAL_GPIO_Init>:
  * @param  GPIO_Init pointer to a GPIO_InitTypeDef structure that contains
  *                    the configuration information for the specified GPIO peripheral.
  * @retval None
  */
void HAL_GPIO_Init(GPIO_TypeDef  *GPIOx, GPIO_InitTypeDef *GPIO_Init)
{
 8000a3c:	b580      	push	{r7, lr}
 8000a3e:	b086      	sub	sp, #24
 8000a40:	af00      	add	r7, sp, #0
 8000a42:	6078      	str	r0, [r7, #4]
 8000a44:	6039      	str	r1, [r7, #0]
  uint32_t position = 0x00U;
 8000a46:	2300      	movs	r3, #0
 8000a48:	617b      	str	r3, [r7, #20]
  uint32_t iocurrent = 0x00U;
 8000a4a:	2300      	movs	r3, #0
 8000a4c:	60fb      	str	r3, [r7, #12]
  uint32_t temp = 0x00U;
 8000a4e:	2300      	movs	r3, #0
 8000a50:	613b      	str	r3, [r7, #16]
  /* Check the parameters */
  assert_param(IS_GPIO_MODE(GPIO_Init->Mode));
  assert_param(IS_GPIO_PIN_AVAILABLE(GPIOx, (GPIO_Init->Pin)));

  /* Configure the port pins */
  while (((GPIO_Init->Pin) >> position) != 0)
 8000a52:	e155      	b.n	8000d00 <HAL_GPIO_Init+0x2c4>
  {
    /* Get the IO position */
    iocurrent = (GPIO_Init->Pin) & (1U << position);
 8000a54:	683b      	ldr	r3, [r7, #0]
 8000a56:	681b      	ldr	r3, [r3, #0]
 8000a58:	2101      	movs	r1, #1
 8000a5a:	697a      	ldr	r2, [r7, #20]
 8000a5c:	4091      	lsls	r1, r2
 8000a5e:	000a      	movs	r2, r1
 8000a60:	4013      	ands	r3, r2
 8000a62:	60fb      	str	r3, [r7, #12]

    if (iocurrent)
 8000a64:	68fb      	ldr	r3, [r7, #12]
 8000a66:	2b00      	cmp	r3, #0
 8000a68:	d100      	bne.n	8000a6c <HAL_GPIO_Init+0x30>
 8000a6a:	e146      	b.n	8000cfa <HAL_GPIO_Init+0x2be>
    {
      /*--------------------- GPIO Mode Configuration ------------------------*/
      /* In case of Output or Alternate function mode selection */
      if (((GPIO_Init->Mode & GPIO_MODE) == MODE_OUTPUT) ||
 8000a6c:	683b      	ldr	r3, [r7, #0]
 8000a6e:	685b      	ldr	r3, [r3, #4]
 8000a70:	2203      	movs	r2, #3
 8000a72:	4013      	ands	r3, r2
 8000a74:	2b01      	cmp	r3, #1
 8000a76:	d005      	beq.n	8000a84 <HAL_GPIO_Init+0x48>
          ((GPIO_Init->Mode & GPIO_MODE) == MODE_AF))
 8000a78:	683b      	ldr	r3, [r7, #0]
 8000a7a:	685b      	ldr	r3, [r3, #4]
 8000a7c:	2203      	movs	r2, #3
 8000a7e:	4013      	ands	r3, r2
      if (((GPIO_Init->Mode & GPIO_MODE) == MODE_OUTPUT) ||
 8000a80:	2b02      	cmp	r3, #2
 8000a82:	d130      	bne.n	8000ae6 <HAL_GPIO_Init+0xaa>
      {
        /* Check the Speed parameter */
        assert_param(IS_GPIO_SPEED(GPIO_Init->Speed));
        /* Configure the IO Speed */
        temp = GPIOx->OSPEEDR;
 8000a84:	687b      	ldr	r3, [r7, #4]
 8000a86:	689b      	ldr	r3, [r3, #8]
 8000a88:	613b      	str	r3, [r7, #16]
        temp &= ~(GPIO_OSPEEDER_OSPEED0 << (position * 2U));
 8000a8a:	697b      	ldr	r3, [r7, #20]
 8000a8c:	005b      	lsls	r3, r3, #1
 8000a8e:	2203      	movs	r2, #3
 8000a90:	409a      	lsls	r2, r3
 8000a92:	0013      	movs	r3, r2
 8000a94:	43da      	mvns	r2, r3
 8000a96:	693b      	ldr	r3, [r7, #16]
 8000a98:	4013      	ands	r3, r2
 8000a9a:	613b      	str	r3, [r7, #16]
        temp |= (GPIO_Init->Speed << (position * 2U));
 8000a9c:	683b      	ldr	r3, [r7, #0]
 8000a9e:	68da      	ldr	r2, [r3, #12]
 8000aa0:	697b      	ldr	r3, [r7, #20]
 8000aa2:	005b      	lsls	r3, r3, #1
 8000aa4:	409a      	lsls	r2, r3
 8000aa6:	0013      	movs	r3, r2
 8000aa8:	693a      	ldr	r2, [r7, #16]
 8000aaa:	4313      	orrs	r3, r2
 8000aac:	613b      	str	r3, [r7, #16]
        GPIOx->OSPEEDR = temp;
 8000aae:	687b      	ldr	r3, [r7, #4]
 8000ab0:	693a      	ldr	r2, [r7, #16]
 8000ab2:	609a      	str	r2, [r3, #8]

        /* Configure the IO Output Type */
        temp = GPIOx->OTYPER;
 8000ab4:	687b      	ldr	r3, [r7, #4]
 8000ab6:	685b      	ldr	r3, [r3, #4]
 8000ab8:	613b      	str	r3, [r7, #16]
        temp &= ~(GPIO_OTYPER_OT_0 << position) ;
 8000aba:	2201      	movs	r2, #1
 8000abc:	697b      	ldr	r3, [r7, #20]
 8000abe:	409a      	lsls	r2, r3
 8000ac0:	0013      	movs	r3, r2
 8000ac2:	43da      	mvns	r2, r3
 8000ac4:	693b      	ldr	r3, [r7, #16]
 8000ac6:	4013      	ands	r3, r2
 8000ac8:	613b      	str	r3, [r7, #16]
        temp |= (((GPIO_Init->Mode & OUTPUT_TYPE) >> OUTPUT_TYPE_Pos) << position);
 8000aca:	683b      	ldr	r3, [r7, #0]
 8000acc:	685b      	ldr	r3, [r3, #4]
 8000ace:	091b      	lsrs	r3, r3, #4
 8000ad0:	2201      	movs	r2, #1
 8000ad2:	401a      	ands	r2, r3
 8000ad4:	697b      	ldr	r3, [r7, #20]
 8000ad6:	409a      	lsls	r2, r3
 8000ad8:	0013      	movs	r3, r2
 8000ada:	693a      	ldr	r2, [r7, #16]
 8000adc:	4313      	orrs	r3, r2
 8000ade:	613b      	str	r3, [r7, #16]
        GPIOx->OTYPER = temp;
 8000ae0:	687b      	ldr	r3, [r7, #4]
 8000ae2:	693a      	ldr	r2, [r7, #16]
 8000ae4:	605a      	str	r2, [r3, #4]
      }

      if ((GPIO_Init->Mode & GPIO_MODE) != MODE_ANALOG)
 8000ae6:	683b      	ldr	r3, [r7, #0]
 8000ae8:	685b      	ldr	r3, [r3, #4]
 8000aea:	2203      	movs	r2, #3
 8000aec:	4013      	ands	r3, r2
 8000aee:	2b03      	cmp	r3, #3
 8000af0:	d017      	beq.n	8000b22 <HAL_GPIO_Init+0xe6>
      {
        /* Check the Pull parameter */
        assert_param(IS_GPIO_PULL(GPIO_Init->Pull));

        /* Activate the Pull-up or Pull down resistor for the current IO */
        temp = GPIOx->PUPDR;
 8000af2:	687b      	ldr	r3, [r7, #4]
 8000af4:	68db      	ldr	r3, [r3, #12]
 8000af6:	613b      	str	r3, [r7, #16]
        temp &= ~(GPIO_PUPDR_PUPD0 << (position * 2U));
 8000af8:	697b      	ldr	r3, [r7, #20]
 8000afa:	005b      	lsls	r3, r3, #1
 8000afc:	2203      	movs	r2, #3
 8000afe:	409a      	lsls	r2, r3
 8000b00:	0013      	movs	r3, r2
 8000b02:	43da      	mvns	r2, r3
 8000b04:	693b      	ldr	r3, [r7, #16]
 8000b06:	4013      	ands	r3, r2
 8000b08:	613b      	str	r3, [r7, #16]
        temp |= ((GPIO_Init->Pull) << (position * 2U));
 8000b0a:	683b      	ldr	r3, [r7, #0]
 8000b0c:	689a      	ldr	r2, [r3, #8]
 8000b0e:	697b      	ldr	r3, [r7, #20]
 8000b10:	005b      	lsls	r3, r3, #1
 8000b12:	409a      	lsls	r2, r3
 8000b14:	0013      	movs	r3, r2
 8000b16:	693a      	ldr	r2, [r7, #16]
 8000b18:	4313      	orrs	r3, r2
 8000b1a:	613b      	str	r3, [r7, #16]
        GPIOx->PUPDR = temp;
 8000b1c:	687b      	ldr	r3, [r7, #4]
 8000b1e:	693a      	ldr	r2, [r7, #16]
 8000b20:	60da      	str	r2, [r3, #12]
      }

      /* In case of Alternate function mode selection */
      if ((GPIO_Init->Mode & GPIO_MODE) == MODE_AF)
 8000b22:	683b      	ldr	r3, [r7, #0]
 8000b24:	685b      	ldr	r3, [r3, #4]
 8000b26:	2203      	movs	r2, #3
 8000b28:	4013      	ands	r3, r2
 8000b2a:	2b02      	cmp	r3, #2
 8000b2c:	d123      	bne.n	8000b76 <HAL_GPIO_Init+0x13a>
        /* Check the Alternate function parameters */
        assert_param(IS_GPIO_AF_INSTANCE(GPIOx));
        assert_param(IS_GPIO_AF(GPIO_Init->Alternate));

        /* Configure Alternate function mapped with the current IO */
        temp = GPIOx->AFR[position >> 3U];
 8000b2e:	697b      	ldr	r3, [r7, #20]
 8000b30:	08da      	lsrs	r2, r3, #3
 8000b32:	687b      	ldr	r3, [r7, #4]
 8000b34:	3208      	adds	r2, #8
 8000b36:	0092      	lsls	r2, r2, #2
 8000b38:	58d3      	ldr	r3, [r2, r3]
 8000b3a:	613b      	str	r3, [r7, #16]
        temp &= ~(0xFUL << ((uint32_t)(position & 0x07UL) * 4U));
 8000b3c:	697b      	ldr	r3, [r7, #20]
 8000b3e:	2207      	movs	r2, #7
 8000b40:	4013      	ands	r3, r2
 8000b42:	009b      	lsls	r3, r3, #2
 8000b44:	220f      	movs	r2, #15
 8000b46:	409a      	lsls	r2, r3
 8000b48:	0013      	movs	r3, r2
 8000b4a:	43da      	mvns	r2, r3
 8000b4c:	693b      	ldr	r3, [r7, #16]
 8000b4e:	4013      	ands	r3, r2
 8000b50:	613b      	str	r3, [r7, #16]
        temp |= ((uint32_t)(GPIO_Init->Alternate) << (((uint32_t)position & (uint32_t)0x07U) * 4U));
 8000b52:	683b      	ldr	r3, [r7, #0]
 8000b54:	691a      	ldr	r2, [r3, #16]
 8000b56:	697b      	ldr	r3, [r7, #20]
 8000b58:	2107      	movs	r1, #7
 8000b5a:	400b      	ands	r3, r1
 8000b5c:	009b      	lsls	r3, r3, #2
 8000b5e:	409a      	lsls	r2, r3
 8000b60:	0013      	movs	r3, r2
 8000b62:	693a      	ldr	r2, [r7, #16]
 8000b64:	4313      	orrs	r3, r2
 8000b66:	613b      	str	r3, [r7, #16]
        GPIOx->AFR[position >> 3U] = temp;
 8000b68:	697b      	ldr	r3, [r7, #20]
 8000b6a:	08da      	lsrs	r2, r3, #3
 8000b6c:	687b      	ldr	r3, [r7, #4]
 8000b6e:	3208      	adds	r2, #8
 8000b70:	0092      	lsls	r2, r2, #2
 8000b72:	6939      	ldr	r1, [r7, #16]
 8000b74:	50d1      	str	r1, [r2, r3]
      }

      /* Configure IO Direction mode (Input, Output, Alternate or Analog) */
      temp = GPIOx->MODER;
 8000b76:	687b      	ldr	r3, [r7, #4]
 8000b78:	681b      	ldr	r3, [r3, #0]
 8000b7a:	613b      	str	r3, [r7, #16]
      temp &= ~(GPIO_MODER_MODE0 << (position * 2U));
 8000b7c:	697b      	ldr	r3, [r7, #20]
 8000b7e:	005b      	lsls	r3, r3, #1
 8000b80:	2203      	movs	r2, #3
 8000b82:	409a      	lsls	r2, r3
 8000b84:	0013      	movs	r3, r2
 8000b86:	43da      	mvns	r2, r3
 8000b88:	693b      	ldr	r3, [r7, #16]
 8000b8a:	4013      	ands	r3, r2
 8000b8c:	613b      	str	r3, [r7, #16]
      temp |= ((GPIO_Init->Mode & GPIO_MODE) << (position * 2U));
 8000b8e:	683b      	ldr	r3, [r7, #0]
 8000b90:	685b      	ldr	r3, [r3, #4]
 8000b92:	2203      	movs	r2, #3
 8000b94:	401a      	ands	r2, r3
 8000b96:	697b      	ldr	r3, [r7, #20]
 8000b98:	005b      	lsls	r3, r3, #1
 8000b9a:	409a      	lsls	r2, r3
 8000b9c:	0013      	movs	r3, r2
 8000b9e:	693a      	ldr	r2, [r7, #16]
 8000ba0:	4313      	orrs	r3, r2
 8000ba2:	613b      	str	r3, [r7, #16]
      GPIOx->MODER = temp;
 8000ba4:	687b      	ldr	r3, [r7, #4]
 8000ba6:	693a      	ldr	r2, [r7, #16]
 8000ba8:	601a      	str	r2, [r3, #0]

      /*--------------------- EXTI Mode Configuration ------------------------*/
      /* Configure the External Interrupt or event for the current IO */
      if ((GPIO_Init->Mode & EXTI_MODE) != 0x00U)
 8000baa:	683b      	ldr	r3, [r7, #0]
 8000bac:	685a      	ldr	r2, [r3, #4]
 8000bae:	23c0      	movs	r3, #192	; 0xc0
 8000bb0:	029b      	lsls	r3, r3, #10
 8000bb2:	4013      	ands	r3, r2
 8000bb4:	d100      	bne.n	8000bb8 <HAL_GPIO_Init+0x17c>
 8000bb6:	e0a0      	b.n	8000cfa <HAL_GPIO_Init+0x2be>
      {
        /* Enable SYSCFG Clock */
        __HAL_RCC_SYSCFG_CLK_ENABLE();
 8000bb8:	4b57      	ldr	r3, [pc, #348]	; (8000d18 <HAL_GPIO_Init+0x2dc>)
 8000bba:	6b5a      	ldr	r2, [r3, #52]	; 0x34
 8000bbc:	4b56      	ldr	r3, [pc, #344]	; (8000d18 <HAL_GPIO_Init+0x2dc>)
 8000bbe:	2101      	movs	r1, #1
 8000bc0:	430a      	orrs	r2, r1
 8000bc2:	635a      	str	r2, [r3, #52]	; 0x34

        temp = SYSCFG->EXTICR[position >> 2U];
 8000bc4:	4a55      	ldr	r2, [pc, #340]	; (8000d1c <HAL_GPIO_Init+0x2e0>)
 8000bc6:	697b      	ldr	r3, [r7, #20]
 8000bc8:	089b      	lsrs	r3, r3, #2
 8000bca:	3302      	adds	r3, #2
 8000bcc:	009b      	lsls	r3, r3, #2
 8000bce:	589b      	ldr	r3, [r3, r2]
 8000bd0:	613b      	str	r3, [r7, #16]
        CLEAR_BIT(temp, (0x0FUL) << (4U * (position & 0x03U)));
 8000bd2:	697b      	ldr	r3, [r7, #20]
 8000bd4:	2203      	movs	r2, #3
 8000bd6:	4013      	ands	r3, r2
 8000bd8:	009b      	lsls	r3, r3, #2
 8000bda:	220f      	movs	r2, #15
 8000bdc:	409a      	lsls	r2, r3
 8000bde:	0013      	movs	r3, r2
 8000be0:	43da      	mvns	r2, r3
 8000be2:	693b      	ldr	r3, [r7, #16]
 8000be4:	4013      	ands	r3, r2
 8000be6:	613b      	str	r3, [r7, #16]
        SET_BIT(temp, (GPIO_GET_INDEX(GPIOx)) << (4 * (position & 0x03U)));
 8000be8:	687a      	ldr	r2, [r7, #4]
 8000bea:	23a0      	movs	r3, #160	; 0xa0
 8000bec:	05db      	lsls	r3, r3, #23
 8000bee:	429a      	cmp	r2, r3
 8000bf0:	d01f      	beq.n	8000c32 <HAL_GPIO_Init+0x1f6>
 8000bf2:	687b      	ldr	r3, [r7, #4]
 8000bf4:	4a4a      	ldr	r2, [pc, #296]	; (8000d20 <HAL_GPIO_Init+0x2e4>)
 8000bf6:	4293      	cmp	r3, r2
 8000bf8:	d019      	beq.n	8000c2e <HAL_GPIO_Init+0x1f2>
 8000bfa:	687b      	ldr	r3, [r7, #4]
 8000bfc:	4a49      	ldr	r2, [pc, #292]	; (8000d24 <HAL_GPIO_Init+0x2e8>)
 8000bfe:	4293      	cmp	r3, r2
 8000c00:	d013      	beq.n	8000c2a <HAL_GPIO_Init+0x1ee>
 8000c02:	687b      	ldr	r3, [r7, #4]
 8000c04:	4a48      	ldr	r2, [pc, #288]	; (8000d28 <HAL_GPIO_Init+0x2ec>)
 8000c06:	4293      	cmp	r3, r2
 8000c08:	d00d      	beq.n	8000c26 <HAL_GPIO_Init+0x1ea>
 8000c0a:	687b      	ldr	r3, [r7, #4]
 8000c0c:	4a47      	ldr	r2, [pc, #284]	; (8000d2c <HAL_GPIO_Init+0x2f0>)
 8000c0e:	4293      	cmp	r3, r2
 8000c10:	d007      	beq.n	8000c22 <HAL_GPIO_Init+0x1e6>
 8000c12:	687b      	ldr	r3, [r7, #4]
 8000c14:	4a46      	ldr	r2, [pc, #280]	; (8000d30 <HAL_GPIO_Init+0x2f4>)
 8000c16:	4293      	cmp	r3, r2
 8000c18:	d101      	bne.n	8000c1e <HAL_GPIO_Init+0x1e2>
 8000c1a:	2305      	movs	r3, #5
 8000c1c:	e00a      	b.n	8000c34 <HAL_GPIO_Init+0x1f8>
 8000c1e:	2306      	movs	r3, #6
 8000c20:	e008      	b.n	8000c34 <HAL_GPIO_Init+0x1f8>
 8000c22:	2304      	movs	r3, #4
 8000c24:	e006      	b.n	8000c34 <HAL_GPIO_Init+0x1f8>
 8000c26:	2303      	movs	r3, #3
 8000c28:	e004      	b.n	8000c34 <HAL_GPIO_Init+0x1f8>
 8000c2a:	2302      	movs	r3, #2
 8000c2c:	e002      	b.n	8000c34 <HAL_GPIO_Init+0x1f8>
 8000c2e:	2301      	movs	r3, #1
 8000c30:	e000      	b.n	8000c34 <HAL_GPIO_Init+0x1f8>
 8000c32:	2300      	movs	r3, #0
 8000c34:	697a      	ldr	r2, [r7, #20]
 8000c36:	2103      	movs	r1, #3
 8000c38:	400a      	ands	r2, r1
 8000c3a:	0092      	lsls	r2, r2, #2
 8000c3c:	4093      	lsls	r3, r2
 8000c3e:	693a      	ldr	r2, [r7, #16]
 8000c40:	4313      	orrs	r3, r2
 8000c42:	613b      	str	r3, [r7, #16]
        SYSCFG->EXTICR[position >> 2U] = temp;
 8000c44:	4935      	ldr	r1, [pc, #212]	; (8000d1c <HAL_GPIO_Init+0x2e0>)
 8000c46:	697b      	ldr	r3, [r7, #20]
 8000c48:	089b      	lsrs	r3, r3, #2
 8000c4a:	3302      	adds	r3, #2
 8000c4c:	009b      	lsls	r3, r3, #2
 8000c4e:	693a      	ldr	r2, [r7, #16]
 8000c50:	505a      	str	r2, [r3, r1]

        /* Clear Rising Falling edge configuration */
        temp = EXTI->RTSR;
 8000c52:	4b38      	ldr	r3, [pc, #224]	; (8000d34 <HAL_GPIO_Init+0x2f8>)
 8000c54:	689b      	ldr	r3, [r3, #8]
 8000c56:	613b      	str	r3, [r7, #16]
        temp &= ~((uint32_t)iocurrent);
 8000c58:	68fb      	ldr	r3, [r7, #12]
 8000c5a:	43da      	mvns	r2, r3
 8000c5c:	693b      	ldr	r3, [r7, #16]
 8000c5e:	4013      	ands	r3, r2
 8000c60:	613b      	str	r3, [r7, #16]
        if ((GPIO_Init->Mode & TRIGGER_RISING) != 0x00U)
 8000c62:	683b      	ldr	r3, [r7, #0]
 8000c64:	685a      	ldr	r2, [r3, #4]
 8000c66:	2380      	movs	r3, #128	; 0x80
 8000c68:	035b      	lsls	r3, r3, #13
 8000c6a:	4013      	ands	r3, r2
 8000c6c:	d003      	beq.n	8000c76 <HAL_GPIO_Init+0x23a>
        {
          temp |= iocurrent;
 8000c6e:	693a      	ldr	r2, [r7, #16]
 8000c70:	68fb      	ldr	r3, [r7, #12]
 8000c72:	4313      	orrs	r3, r2
 8000c74:	613b      	str	r3, [r7, #16]
        }
        EXTI->RTSR = temp;
 8000c76:	4b2f      	ldr	r3, [pc, #188]	; (8000d34 <HAL_GPIO_Init+0x2f8>)
 8000c78:	693a      	ldr	r2, [r7, #16]
 8000c7a:	609a      	str	r2, [r3, #8]

        temp = EXTI->FTSR;
 8000c7c:	4b2d      	ldr	r3, [pc, #180]	; (8000d34 <HAL_GPIO_Init+0x2f8>)
 8000c7e:	68db      	ldr	r3, [r3, #12]
 8000c80:	613b      	str	r3, [r7, #16]
        temp &= ~((uint32_t)iocurrent);
 8000c82:	68fb      	ldr	r3, [r7, #12]
 8000c84:	43da      	mvns	r2, r3
 8000c86:	693b      	ldr	r3, [r7, #16]
 8000c88:	4013      	ands	r3, r2
 8000c8a:	613b      	str	r3, [r7, #16]
        if ((GPIO_Init->Mode & TRIGGER_FALLING) != 0x00U)
 8000c8c:	683b      	ldr	r3, [r7, #0]
 8000c8e:	685a      	ldr	r2, [r3, #4]
 8000c90:	2380      	movs	r3, #128	; 0x80
 8000c92:	039b      	lsls	r3, r3, #14
 8000c94:	4013      	ands	r3, r2
 8000c96:	d003      	beq.n	8000ca0 <HAL_GPIO_Init+0x264>
        {
          temp |= iocurrent;
 8000c98:	693a      	ldr	r2, [r7, #16]
 8000c9a:	68fb      	ldr	r3, [r7, #12]
 8000c9c:	4313      	orrs	r3, r2
 8000c9e:	613b      	str	r3, [r7, #16]
        }
        EXTI->FTSR = temp;
 8000ca0:	4b24      	ldr	r3, [pc, #144]	; (8000d34 <HAL_GPIO_Init+0x2f8>)
 8000ca2:	693a      	ldr	r2, [r7, #16]
 8000ca4:	60da      	str	r2, [r3, #12]

        temp = EXTI->EMR;
 8000ca6:	4b23      	ldr	r3, [pc, #140]	; (8000d34 <HAL_GPIO_Init+0x2f8>)
 8000ca8:	685b      	ldr	r3, [r3, #4]
 8000caa:	613b      	str	r3, [r7, #16]
        temp &= ~((uint32_t)iocurrent);
 8000cac:	68fb      	ldr	r3, [r7, #12]
 8000cae:	43da      	mvns	r2, r3
 8000cb0:	693b      	ldr	r3, [r7, #16]
 8000cb2:	4013      	ands	r3, r2
 8000cb4:	613b      	str	r3, [r7, #16]
        if ((GPIO_Init->Mode & EXTI_EVT) != 0x00U)
 8000cb6:	683b      	ldr	r3, [r7, #0]
 8000cb8:	685a      	ldr	r2, [r3, #4]
 8000cba:	2380      	movs	r3, #128	; 0x80
 8000cbc:	029b      	lsls	r3, r3, #10
 8000cbe:	4013      	ands	r3, r2
 8000cc0:	d003      	beq.n	8000cca <HAL_GPIO_Init+0x28e>
        {
          temp |= iocurrent;
 8000cc2:	693a      	ldr	r2, [r7, #16]
 8000cc4:	68fb      	ldr	r3, [r7, #12]
 8000cc6:	4313      	orrs	r3, r2
 8000cc8:	613b      	str	r3, [r7, #16]
        }
        EXTI->EMR = temp;
 8000cca:	4b1a      	ldr	r3, [pc, #104]	; (8000d34 <HAL_GPIO_Init+0x2f8>)
 8000ccc:	693a      	ldr	r2, [r7, #16]
 8000cce:	605a      	str	r2, [r3, #4]

        /* Clear EXTI line configuration */
        temp = EXTI->IMR;
 8000cd0:	4b18      	ldr	r3, [pc, #96]	; (8000d34 <HAL_GPIO_Init+0x2f8>)
 8000cd2:	681b      	ldr	r3, [r3, #0]
 8000cd4:	613b      	str	r3, [r7, #16]
        temp &= ~((uint32_t)iocurrent);
 8000cd6:	68fb      	ldr	r3, [r7, #12]
 8000cd8:	43da      	mvns	r2, r3
 8000cda:	693b      	ldr	r3, [r7, #16]
 8000cdc:	4013      	ands	r3, r2
 8000cde:	613b      	str	r3, [r7, #16]
        if ((GPIO_Init->Mode & EXTI_IT) != 0x00U)
 8000ce0:	683b      	ldr	r3, [r7, #0]
 8000ce2:	685a      	ldr	r2, [r3, #4]
 8000ce4:	2380      	movs	r3, #128	; 0x80
 8000ce6:	025b      	lsls	r3, r3, #9
 8000ce8:	4013      	ands	r3, r2
 8000cea:	d003      	beq.n	8000cf4 <HAL_GPIO_Init+0x2b8>
        {
          temp |= iocurrent;
 8000cec:	693a      	ldr	r2, [r7, #16]
 8000cee:	68fb      	ldr	r3, [r7, #12]
 8000cf0:	4313      	orrs	r3, r2
 8000cf2:	613b      	str	r3, [r7, #16]
        }
        EXTI->IMR = temp;
 8000cf4:	4b0f      	ldr	r3, [pc, #60]	; (8000d34 <HAL_GPIO_Init+0x2f8>)
 8000cf6:	693a      	ldr	r2, [r7, #16]
 8000cf8:	601a      	str	r2, [r3, #0]
      }
    }
    position++;
 8000cfa:	697b      	ldr	r3, [r7, #20]
 8000cfc:	3301      	adds	r3, #1
 8000cfe:	617b      	str	r3, [r7, #20]
  while (((GPIO_Init->Pin) >> position) != 0)
 8000d00:	683b      	ldr	r3, [r7, #0]
 8000d02:	681a      	ldr	r2, [r3, #0]
 8000d04:	697b      	ldr	r3, [r7, #20]
 8000d06:	40da      	lsrs	r2, r3
 8000d08:	1e13      	subs	r3, r2, #0
 8000d0a:	d000      	beq.n	8000d0e <HAL_GPIO_Init+0x2d2>
 8000d0c:	e6a2      	b.n	8000a54 <HAL_GPIO_Init+0x18>
  }
}
 8000d0e:	46c0      	nop			; (mov r8, r8)
 8000d10:	46c0      	nop			; (mov r8, r8)
 8000d12:	46bd      	mov	sp, r7
 8000d14:	b006      	add	sp, #24
 8000d16:	bd80      	pop	{r7, pc}
 8000d18:	40021000 	.word	0x40021000
 8000d1c:	40010000 	.word	0x40010000
 8000d20:	50000400 	.word	0x50000400
 8000d24:	50000800 	.word	0x50000800
 8000d28:	50000c00 	.word	0x50000c00
 8000d2c:	50001000 	.word	0x50001000
 8000d30:	50001c00 	.word	0x50001c00
 8000d34:	40010400 	.word	0x40010400

08000d38 <HAL_RCC_OscConfig>:
  *         supported by this macro. User should request a transition to HSE Off
  *         first and then HSE On or HSE Bypass.
  * @retval HAL status
  */
HAL_StatusTypeDef HAL_RCC_OscConfig(RCC_OscInitTypeDef  *RCC_OscInitStruct)
{
 8000d38:	b5b0      	push	{r4, r5, r7, lr}
 8000d3a:	b08a      	sub	sp, #40	; 0x28
 8000d3c:	af00      	add	r7, sp, #0
 8000d3e:	6078      	str	r0, [r7, #4]
  uint32_t hsi_state;
  HAL_StatusTypeDef status;
  uint32_t sysclk_source, pll_config;

  /* Check Null pointer */
  if(RCC_OscInitStruct == NULL)
 8000d40:	687b      	ldr	r3, [r7, #4]
 8000d42:	2b00      	cmp	r3, #0
 8000d44:	d102      	bne.n	8000d4c <HAL_RCC_OscConfig+0x14>
  {
    return HAL_ERROR;
 8000d46:	2301      	movs	r3, #1
 8000d48:	f000 fbbf 	bl	80014ca <HAL_RCC_OscConfig+0x792>
  }

  /* Check the parameters */
  assert_param(IS_RCC_OSCILLATORTYPE(RCC_OscInitStruct->OscillatorType));

  sysclk_source = __HAL_RCC_GET_SYSCLK_SOURCE();
 8000d4c:	4bc9      	ldr	r3, [pc, #804]	; (8001074 <HAL_RCC_OscConfig+0x33c>)
 8000d4e:	68db      	ldr	r3, [r3, #12]
 8000d50:	220c      	movs	r2, #12
 8000d52:	4013      	ands	r3, r2
 8000d54:	61fb      	str	r3, [r7, #28]
  pll_config = __HAL_RCC_GET_PLL_OSCSOURCE();
 8000d56:	4bc7      	ldr	r3, [pc, #796]	; (8001074 <HAL_RCC_OscConfig+0x33c>)
 8000d58:	68da      	ldr	r2, [r3, #12]
 8000d5a:	2380      	movs	r3, #128	; 0x80
 8000d5c:	025b      	lsls	r3, r3, #9
 8000d5e:	4013      	ands	r3, r2
 8000d60:	61bb      	str	r3, [r7, #24]

  /*------------------------------- HSE Configuration ------------------------*/
  if(((RCC_OscInitStruct->OscillatorType) & RCC_OSCILLATORTYPE_HSE) == RCC_OSCILLATORTYPE_HSE)
 8000d62:	687b      	ldr	r3, [r7, #4]
 8000d64:	681b      	ldr	r3, [r3, #0]
 8000d66:	2201      	movs	r2, #1
 8000d68:	4013      	ands	r3, r2
 8000d6a:	d100      	bne.n	8000d6e <HAL_RCC_OscConfig+0x36>
 8000d6c:	e07e      	b.n	8000e6c <HAL_RCC_OscConfig+0x134>
  {
    /* Check the parameters */
    assert_param(IS_RCC_HSE(RCC_OscInitStruct->HSEState));

    /* When the HSE is used as system clock or clock source for PLL in these cases it is not allowed to be disabled */
    if((sysclk_source == RCC_SYSCLKSOURCE_STATUS_HSE)
 8000d6e:	69fb      	ldr	r3, [r7, #28]
 8000d70:	2b08      	cmp	r3, #8
 8000d72:	d007      	beq.n	8000d84 <HAL_RCC_OscConfig+0x4c>
       || ((sysclk_source == RCC_SYSCLKSOURCE_STATUS_PLLCLK) && (pll_config == RCC_PLLSOURCE_HSE)))
 8000d74:	69fb      	ldr	r3, [r7, #28]
 8000d76:	2b0c      	cmp	r3, #12
 8000d78:	d112      	bne.n	8000da0 <HAL_RCC_OscConfig+0x68>
 8000d7a:	69ba      	ldr	r2, [r7, #24]
 8000d7c:	2380      	movs	r3, #128	; 0x80
 8000d7e:	025b      	lsls	r3, r3, #9
 8000d80:	429a      	cmp	r2, r3
 8000d82:	d10d      	bne.n	8000da0 <HAL_RCC_OscConfig+0x68>
    {
      if((__HAL_RCC_GET_FLAG(RCC_FLAG_HSERDY) != 0U) && (RCC_OscInitStruct->HSEState == RCC_HSE_OFF))
 8000d84:	4bbb      	ldr	r3, [pc, #748]	; (8001074 <HAL_RCC_OscConfig+0x33c>)
 8000d86:	681a      	ldr	r2, [r3, #0]
 8000d88:	2380      	movs	r3, #128	; 0x80
 8000d8a:	029b      	lsls	r3, r3, #10
 8000d8c:	4013      	ands	r3, r2
 8000d8e:	d100      	bne.n	8000d92 <HAL_RCC_OscConfig+0x5a>
 8000d90:	e06b      	b.n	8000e6a <HAL_RCC_OscConfig+0x132>
 8000d92:	687b      	ldr	r3, [r7, #4]
 8000d94:	685b      	ldr	r3, [r3, #4]
 8000d96:	2b00      	cmp	r3, #0
 8000d98:	d167      	bne.n	8000e6a <HAL_RCC_OscConfig+0x132>
      {
        return HAL_ERROR;
 8000d9a:	2301      	movs	r3, #1
 8000d9c:	f000 fb95 	bl	80014ca <HAL_RCC_OscConfig+0x792>
      }
    }
    else
    {
      /* Set the new HSE configuration ---------------------------------------*/
      __HAL_RCC_HSE_CONFIG(RCC_OscInitStruct->HSEState);
 8000da0:	687b      	ldr	r3, [r7, #4]
 8000da2:	685a      	ldr	r2, [r3, #4]
 8000da4:	2380      	movs	r3, #128	; 0x80
 8000da6:	025b      	lsls	r3, r3, #9
 8000da8:	429a      	cmp	r2, r3
 8000daa:	d107      	bne.n	8000dbc <HAL_RCC_OscConfig+0x84>
 8000dac:	4bb1      	ldr	r3, [pc, #708]	; (8001074 <HAL_RCC_OscConfig+0x33c>)
 8000dae:	681a      	ldr	r2, [r3, #0]
 8000db0:	4bb0      	ldr	r3, [pc, #704]	; (8001074 <HAL_RCC_OscConfig+0x33c>)
 8000db2:	2180      	movs	r1, #128	; 0x80
 8000db4:	0249      	lsls	r1, r1, #9
 8000db6:	430a      	orrs	r2, r1
 8000db8:	601a      	str	r2, [r3, #0]
 8000dba:	e027      	b.n	8000e0c <HAL_RCC_OscConfig+0xd4>
 8000dbc:	687b      	ldr	r3, [r7, #4]
 8000dbe:	685a      	ldr	r2, [r3, #4]
 8000dc0:	23a0      	movs	r3, #160	; 0xa0
 8000dc2:	02db      	lsls	r3, r3, #11
 8000dc4:	429a      	cmp	r2, r3
 8000dc6:	d10e      	bne.n	8000de6 <HAL_RCC_OscConfig+0xae>
 8000dc8:	4baa      	ldr	r3, [pc, #680]	; (8001074 <HAL_RCC_OscConfig+0x33c>)
 8000dca:	681a      	ldr	r2, [r3, #0]
 8000dcc:	4ba9      	ldr	r3, [pc, #676]	; (8001074 <HAL_RCC_OscConfig+0x33c>)
 8000dce:	2180      	movs	r1, #128	; 0x80
 8000dd0:	02c9      	lsls	r1, r1, #11
 8000dd2:	430a      	orrs	r2, r1
 8000dd4:	601a      	str	r2, [r3, #0]
 8000dd6:	4ba7      	ldr	r3, [pc, #668]	; (8001074 <HAL_RCC_OscConfig+0x33c>)
 8000dd8:	681a      	ldr	r2, [r3, #0]
 8000dda:	4ba6      	ldr	r3, [pc, #664]	; (8001074 <HAL_RCC_OscConfig+0x33c>)
 8000ddc:	2180      	movs	r1, #128	; 0x80
 8000dde:	0249      	lsls	r1, r1, #9
 8000de0:	430a      	orrs	r2, r1
 8000de2:	601a      	str	r2, [r3, #0]
 8000de4:	e012      	b.n	8000e0c <HAL_RCC_OscConfig+0xd4>
 8000de6:	4ba3      	ldr	r3, [pc, #652]	; (8001074 <HAL_RCC_OscConfig+0x33c>)
 8000de8:	681a      	ldr	r2, [r3, #0]
 8000dea:	4ba2      	ldr	r3, [pc, #648]	; (8001074 <HAL_RCC_OscConfig+0x33c>)
 8000dec:	49a2      	ldr	r1, [pc, #648]	; (8001078 <HAL_RCC_OscConfig+0x340>)
 8000dee:	400a      	ands	r2, r1
 8000df0:	601a      	str	r2, [r3, #0]
 8000df2:	4ba0      	ldr	r3, [pc, #640]	; (8001074 <HAL_RCC_OscConfig+0x33c>)
 8000df4:	681a      	ldr	r2, [r3, #0]
 8000df6:	2380      	movs	r3, #128	; 0x80
 8000df8:	025b      	lsls	r3, r3, #9
 8000dfa:	4013      	ands	r3, r2
 8000dfc:	60fb      	str	r3, [r7, #12]
 8000dfe:	68fb      	ldr	r3, [r7, #12]
 8000e00:	4b9c      	ldr	r3, [pc, #624]	; (8001074 <HAL_RCC_OscConfig+0x33c>)
 8000e02:	681a      	ldr	r2, [r3, #0]
 8000e04:	4b9b      	ldr	r3, [pc, #620]	; (8001074 <HAL_RCC_OscConfig+0x33c>)
 8000e06:	499d      	ldr	r1, [pc, #628]	; (800107c <HAL_RCC_OscConfig+0x344>)
 8000e08:	400a      	ands	r2, r1
 8000e0a:	601a      	str	r2, [r3, #0]

      /* Check the HSE State */
      if(RCC_OscInitStruct->HSEState != RCC_HSE_OFF)
 8000e0c:	687b      	ldr	r3, [r7, #4]
 8000e0e:	685b      	ldr	r3, [r3, #4]
 8000e10:	2b00      	cmp	r3, #0
 8000e12:	d015      	beq.n	8000e40 <HAL_RCC_OscConfig+0x108>
      {
        /* Get Start Tick */
        tickstart = HAL_GetTick();
 8000e14:	f7ff fd30 	bl	8000878 <HAL_GetTick>
 8000e18:	0003      	movs	r3, r0
 8000e1a:	617b      	str	r3, [r7, #20]

        /* Wait till HSE is ready */
        while(__HAL_RCC_GET_FLAG(RCC_FLAG_HSERDY) == 0U)
 8000e1c:	e009      	b.n	8000e32 <HAL_RCC_OscConfig+0xfa>
        {
          if((HAL_GetTick() - tickstart ) > HSE_TIMEOUT_VALUE)
 8000e1e:	f7ff fd2b 	bl	8000878 <HAL_GetTick>
 8000e22:	0002      	movs	r2, r0
 8000e24:	697b      	ldr	r3, [r7, #20]
 8000e26:	1ad3      	subs	r3, r2, r3
 8000e28:	2b64      	cmp	r3, #100	; 0x64
 8000e2a:	d902      	bls.n	8000e32 <HAL_RCC_OscConfig+0xfa>
          {
            return HAL_TIMEOUT;
 8000e2c:	2303      	movs	r3, #3
 8000e2e:	f000 fb4c 	bl	80014ca <HAL_RCC_OscConfig+0x792>
        while(__HAL_RCC_GET_FLAG(RCC_FLAG_HSERDY) == 0U)
 8000e32:	4b90      	ldr	r3, [pc, #576]	; (8001074 <HAL_RCC_OscConfig+0x33c>)
 8000e34:	681a      	ldr	r2, [r3, #0]
 8000e36:	2380      	movs	r3, #128	; 0x80
 8000e38:	029b      	lsls	r3, r3, #10
 8000e3a:	4013      	ands	r3, r2
 8000e3c:	d0ef      	beq.n	8000e1e <HAL_RCC_OscConfig+0xe6>
 8000e3e:	e015      	b.n	8000e6c <HAL_RCC_OscConfig+0x134>
        }
      }
      else
      {
        /* Get Start Tick */
        tickstart = HAL_GetTick();
 8000e40:	f7ff fd1a 	bl	8000878 <HAL_GetTick>
 8000e44:	0003      	movs	r3, r0
 8000e46:	617b      	str	r3, [r7, #20]

        /* Wait till HSE is disabled */
        while(__HAL_RCC_GET_FLAG(RCC_FLAG_HSERDY) != 0U)
 8000e48:	e008      	b.n	8000e5c <HAL_RCC_OscConfig+0x124>
        {
           if((HAL_GetTick() - tickstart ) > HSE_TIMEOUT_VALUE)
 8000e4a:	f7ff fd15 	bl	8000878 <HAL_GetTick>
 8000e4e:	0002      	movs	r2, r0
 8000e50:	697b      	ldr	r3, [r7, #20]
 8000e52:	1ad3      	subs	r3, r2, r3
 8000e54:	2b64      	cmp	r3, #100	; 0x64
 8000e56:	d901      	bls.n	8000e5c <HAL_RCC_OscConfig+0x124>
          {
            return HAL_TIMEOUT;
 8000e58:	2303      	movs	r3, #3
 8000e5a:	e336      	b.n	80014ca <HAL_RCC_OscConfig+0x792>
        while(__HAL_RCC_GET_FLAG(RCC_FLAG_HSERDY) != 0U)
 8000e5c:	4b85      	ldr	r3, [pc, #532]	; (8001074 <HAL_RCC_OscConfig+0x33c>)
 8000e5e:	681a      	ldr	r2, [r3, #0]
 8000e60:	2380      	movs	r3, #128	; 0x80
 8000e62:	029b      	lsls	r3, r3, #10
 8000e64:	4013      	ands	r3, r2
 8000e66:	d1f0      	bne.n	8000e4a <HAL_RCC_OscConfig+0x112>
 8000e68:	e000      	b.n	8000e6c <HAL_RCC_OscConfig+0x134>
      if((__HAL_RCC_GET_FLAG(RCC_FLAG_HSERDY) != 0U) && (RCC_OscInitStruct->HSEState == RCC_HSE_OFF))
 8000e6a:	46c0      	nop			; (mov r8, r8)
        }
      }
    }
  }
  /*----------------------------- HSI Configuration --------------------------*/
  if(((RCC_OscInitStruct->OscillatorType) & RCC_OSCILLATORTYPE_HSI) == RCC_OSCILLATORTYPE_HSI)
 8000e6c:	687b      	ldr	r3, [r7, #4]
 8000e6e:	681b      	ldr	r3, [r3, #0]
 8000e70:	2202      	movs	r2, #2
 8000e72:	4013      	ands	r3, r2
 8000e74:	d100      	bne.n	8000e78 <HAL_RCC_OscConfig+0x140>
 8000e76:	e099      	b.n	8000fac <HAL_RCC_OscConfig+0x274>
  {
    /* Check the parameters */
    assert_param(IS_RCC_HSI(RCC_OscInitStruct->HSIState));
    assert_param(IS_RCC_CALIBRATION_VALUE(RCC_OscInitStruct->HSICalibrationValue));

    hsi_state = RCC_OscInitStruct->HSIState;
 8000e78:	687b      	ldr	r3, [r7, #4]
 8000e7a:	68db      	ldr	r3, [r3, #12]
 8000e7c:	627b      	str	r3, [r7, #36]	; 0x24

#if defined(RCC_CR_HSIOUTEN)
    if((hsi_state & RCC_HSI_OUTEN) != 0U)
 8000e7e:	6a7b      	ldr	r3, [r7, #36]	; 0x24
 8000e80:	2220      	movs	r2, #32
 8000e82:	4013      	ands	r3, r2
 8000e84:	d009      	beq.n	8000e9a <HAL_RCC_OscConfig+0x162>
    {
      /* HSI Output enable for timer requested */
      SET_BIT(RCC->CR, RCC_CR_HSIOUTEN);
 8000e86:	4b7b      	ldr	r3, [pc, #492]	; (8001074 <HAL_RCC_OscConfig+0x33c>)
 8000e88:	681a      	ldr	r2, [r3, #0]
 8000e8a:	4b7a      	ldr	r3, [pc, #488]	; (8001074 <HAL_RCC_OscConfig+0x33c>)
 8000e8c:	2120      	movs	r1, #32
 8000e8e:	430a      	orrs	r2, r1
 8000e90:	601a      	str	r2, [r3, #0]

      hsi_state &= ~RCC_CR_HSIOUTEN;
 8000e92:	6a7b      	ldr	r3, [r7, #36]	; 0x24
 8000e94:	2220      	movs	r2, #32
 8000e96:	4393      	bics	r3, r2
 8000e98:	627b      	str	r3, [r7, #36]	; 0x24
    }
#endif

    /* Check if HSI is used as system clock or as PLL source when PLL is selected as system clock */
    if((sysclk_source == RCC_SYSCLKSOURCE_STATUS_HSI)
 8000e9a:	69fb      	ldr	r3, [r7, #28]
 8000e9c:	2b04      	cmp	r3, #4
 8000e9e:	d005      	beq.n	8000eac <HAL_RCC_OscConfig+0x174>
       || ((sysclk_source == RCC_SYSCLKSOURCE_STATUS_PLLCLK) && (pll_config == RCC_PLLSOURCE_HSI)))
 8000ea0:	69fb      	ldr	r3, [r7, #28]
 8000ea2:	2b0c      	cmp	r3, #12
 8000ea4:	d13e      	bne.n	8000f24 <HAL_RCC_OscConfig+0x1ec>
 8000ea6:	69bb      	ldr	r3, [r7, #24]
 8000ea8:	2b00      	cmp	r3, #0
 8000eaa:	d13b      	bne.n	8000f24 <HAL_RCC_OscConfig+0x1ec>
    {
      /* When HSI is used as system clock it will not disabled */
      if((__HAL_RCC_GET_FLAG(RCC_FLAG_HSIRDY) != 0U) && (hsi_state == RCC_HSI_OFF))
 8000eac:	4b71      	ldr	r3, [pc, #452]	; (8001074 <HAL_RCC_OscConfig+0x33c>)
 8000eae:	681b      	ldr	r3, [r3, #0]
 8000eb0:	2204      	movs	r2, #4
 8000eb2:	4013      	ands	r3, r2
 8000eb4:	d004      	beq.n	8000ec0 <HAL_RCC_OscConfig+0x188>
 8000eb6:	6a7b      	ldr	r3, [r7, #36]	; 0x24
 8000eb8:	2b00      	cmp	r3, #0
 8000eba:	d101      	bne.n	8000ec0 <HAL_RCC_OscConfig+0x188>
      {
        return HAL_ERROR;
 8000ebc:	2301      	movs	r3, #1
 8000ebe:	e304      	b.n	80014ca <HAL_RCC_OscConfig+0x792>
      }
      /* Otherwise, just the calibration and HSI or HSIdiv4 are allowed */
      else
      {
        /* Adjusts the Internal High Speed oscillator (HSI) calibration value.*/
        __HAL_RCC_HSI_CALIBRATIONVALUE_ADJUST(RCC_OscInitStruct->HSICalibrationValue);
 8000ec0:	4b6c      	ldr	r3, [pc, #432]	; (8001074 <HAL_RCC_OscConfig+0x33c>)
 8000ec2:	685b      	ldr	r3, [r3, #4]
 8000ec4:	4a6e      	ldr	r2, [pc, #440]	; (8001080 <HAL_RCC_OscConfig+0x348>)
 8000ec6:	4013      	ands	r3, r2
 8000ec8:	0019      	movs	r1, r3
 8000eca:	687b      	ldr	r3, [r7, #4]
 8000ecc:	691b      	ldr	r3, [r3, #16]
 8000ece:	021a      	lsls	r2, r3, #8
 8000ed0:	4b68      	ldr	r3, [pc, #416]	; (8001074 <HAL_RCC_OscConfig+0x33c>)
 8000ed2:	430a      	orrs	r2, r1
 8000ed4:	605a      	str	r2, [r3, #4]

        /* Enable the Internal High Speed oscillator (HSI or HSIdiv4) */
        __HAL_RCC_HSI_CONFIG(hsi_state);
 8000ed6:	4b67      	ldr	r3, [pc, #412]	; (8001074 <HAL_RCC_OscConfig+0x33c>)
 8000ed8:	681b      	ldr	r3, [r3, #0]
 8000eda:	2209      	movs	r2, #9
 8000edc:	4393      	bics	r3, r2
 8000ede:	0019      	movs	r1, r3
 8000ee0:	4b64      	ldr	r3, [pc, #400]	; (8001074 <HAL_RCC_OscConfig+0x33c>)
 8000ee2:	6a7a      	ldr	r2, [r7, #36]	; 0x24
 8000ee4:	430a      	orrs	r2, r1
 8000ee6:	601a      	str	r2, [r3, #0]
      }

      /* Update the SystemCoreClock global variable */
      SystemCoreClock = HAL_RCC_GetSysClockFreq() >> AHBPrescTable[(RCC->CFGR & RCC_CFGR_HPRE)>> RCC_CFGR_HPRE_Pos];
 8000ee8:	f000 fc42 	bl	8001770 <HAL_RCC_GetSysClockFreq>
 8000eec:	0001      	movs	r1, r0
 8000eee:	4b61      	ldr	r3, [pc, #388]	; (8001074 <HAL_RCC_OscConfig+0x33c>)
 8000ef0:	68db      	ldr	r3, [r3, #12]
 8000ef2:	091b      	lsrs	r3, r3, #4
 8000ef4:	220f      	movs	r2, #15
 8000ef6:	4013      	ands	r3, r2
 8000ef8:	4a62      	ldr	r2, [pc, #392]	; (8001084 <HAL_RCC_OscConfig+0x34c>)
 8000efa:	5cd3      	ldrb	r3, [r2, r3]
 8000efc:	000a      	movs	r2, r1
 8000efe:	40da      	lsrs	r2, r3
 8000f00:	4b61      	ldr	r3, [pc, #388]	; (8001088 <HAL_RCC_OscConfig+0x350>)
 8000f02:	601a      	str	r2, [r3, #0]

      /* Configure the source of time base considering new system clocks settings*/
      status = HAL_InitTick (uwTickPrio);
 8000f04:	4b61      	ldr	r3, [pc, #388]	; (800108c <HAL_RCC_OscConfig+0x354>)
 8000f06:	681b      	ldr	r3, [r3, #0]
 8000f08:	2513      	movs	r5, #19
 8000f0a:	197c      	adds	r4, r7, r5
 8000f0c:	0018      	movs	r0, r3
 8000f0e:	f7ff fc6d 	bl	80007ec <HAL_InitTick>
 8000f12:	0003      	movs	r3, r0
 8000f14:	7023      	strb	r3, [r4, #0]
      if(status != HAL_OK)
 8000f16:	197b      	adds	r3, r7, r5
 8000f18:	781b      	ldrb	r3, [r3, #0]
 8000f1a:	2b00      	cmp	r3, #0
 8000f1c:	d046      	beq.n	8000fac <HAL_RCC_OscConfig+0x274>
      {
        return status;
 8000f1e:	197b      	adds	r3, r7, r5
 8000f20:	781b      	ldrb	r3, [r3, #0]
 8000f22:	e2d2      	b.n	80014ca <HAL_RCC_OscConfig+0x792>
      }
    }
    else
    {
      /* Check the HSI State */
      if(hsi_state != RCC_HSI_OFF)
 8000f24:	6a7b      	ldr	r3, [r7, #36]	; 0x24
 8000f26:	2b00      	cmp	r3, #0
 8000f28:	d027      	beq.n	8000f7a <HAL_RCC_OscConfig+0x242>
      {
        /* Enable the Internal High Speed oscillator (HSI or HSIdiv4) */
        __HAL_RCC_HSI_CONFIG(hsi_state);
 8000f2a:	4b52      	ldr	r3, [pc, #328]	; (8001074 <HAL_RCC_OscConfig+0x33c>)
 8000f2c:	681b      	ldr	r3, [r3, #0]
 8000f2e:	2209      	movs	r2, #9
 8000f30:	4393      	bics	r3, r2
 8000f32:	0019      	movs	r1, r3
 8000f34:	4b4f      	ldr	r3, [pc, #316]	; (8001074 <HAL_RCC_OscConfig+0x33c>)
 8000f36:	6a7a      	ldr	r2, [r7, #36]	; 0x24
 8000f38:	430a      	orrs	r2, r1
 8000f3a:	601a      	str	r2, [r3, #0]

        /* Get Start Tick */
        tickstart = HAL_GetTick();
 8000f3c:	f7ff fc9c 	bl	8000878 <HAL_GetTick>
 8000f40:	0003      	movs	r3, r0
 8000f42:	617b      	str	r3, [r7, #20]

        /* Wait till HSI is ready */
        while(__HAL_RCC_GET_FLAG(RCC_FLAG_HSIRDY) == 0U)
 8000f44:	e008      	b.n	8000f58 <HAL_RCC_OscConfig+0x220>
        {
          if((HAL_GetTick() - tickstart ) > HSI_TIMEOUT_VALUE)
 8000f46:	f7ff fc97 	bl	8000878 <HAL_GetTick>
 8000f4a:	0002      	movs	r2, r0
 8000f4c:	697b      	ldr	r3, [r7, #20]
 8000f4e:	1ad3      	subs	r3, r2, r3
 8000f50:	2b02      	cmp	r3, #2
 8000f52:	d901      	bls.n	8000f58 <HAL_RCC_OscConfig+0x220>
          {
            return HAL_TIMEOUT;
 8000f54:	2303      	movs	r3, #3
 8000f56:	e2b8      	b.n	80014ca <HAL_RCC_OscConfig+0x792>
        while(__HAL_RCC_GET_FLAG(RCC_FLAG_HSIRDY) == 0U)
 8000f58:	4b46      	ldr	r3, [pc, #280]	; (8001074 <HAL_RCC_OscConfig+0x33c>)
 8000f5a:	681b      	ldr	r3, [r3, #0]
 8000f5c:	2204      	movs	r2, #4
 8000f5e:	4013      	ands	r3, r2
 8000f60:	d0f1      	beq.n	8000f46 <HAL_RCC_OscConfig+0x20e>
          }
        }

        /* Adjusts the Internal High Speed oscillator (HSI) calibration value.*/
        __HAL_RCC_HSI_CALIBRATIONVALUE_ADJUST(RCC_OscInitStruct->HSICalibrationValue);
 8000f62:	4b44      	ldr	r3, [pc, #272]	; (8001074 <HAL_RCC_OscConfig+0x33c>)
 8000f64:	685b      	ldr	r3, [r3, #4]
 8000f66:	4a46      	ldr	r2, [pc, #280]	; (8001080 <HAL_RCC_OscConfig+0x348>)
 8000f68:	4013      	ands	r3, r2
 8000f6a:	0019      	movs	r1, r3
 8000f6c:	687b      	ldr	r3, [r7, #4]
 8000f6e:	691b      	ldr	r3, [r3, #16]
 8000f70:	021a      	lsls	r2, r3, #8
 8000f72:	4b40      	ldr	r3, [pc, #256]	; (8001074 <HAL_RCC_OscConfig+0x33c>)
 8000f74:	430a      	orrs	r2, r1
 8000f76:	605a      	str	r2, [r3, #4]
 8000f78:	e018      	b.n	8000fac <HAL_RCC_OscConfig+0x274>
      }
      else
      {
        /* Disable the Internal High Speed oscillator (HSI). */
        __HAL_RCC_HSI_DISABLE();
 8000f7a:	4b3e      	ldr	r3, [pc, #248]	; (8001074 <HAL_RCC_OscConfig+0x33c>)
 8000f7c:	681a      	ldr	r2, [r3, #0]
 8000f7e:	4b3d      	ldr	r3, [pc, #244]	; (8001074 <HAL_RCC_OscConfig+0x33c>)
 8000f80:	2101      	movs	r1, #1
 8000f82:	438a      	bics	r2, r1
 8000f84:	601a      	str	r2, [r3, #0]

        /* Get Start Tick */
        tickstart = HAL_GetTick();
 8000f86:	f7ff fc77 	bl	8000878 <HAL_GetTick>
 8000f8a:	0003      	movs	r3, r0
 8000f8c:	617b      	str	r3, [r7, #20]

        /* Wait till HSI is disabled */
        while(__HAL_RCC_GET_FLAG(RCC_FLAG_HSIRDY) != 0U)
 8000f8e:	e008      	b.n	8000fa2 <HAL_RCC_OscConfig+0x26a>
        {
          if((HAL_GetTick() - tickstart ) > HSI_TIMEOUT_VALUE)
 8000f90:	f7ff fc72 	bl	8000878 <HAL_GetTick>
 8000f94:	0002      	movs	r2, r0
 8000f96:	697b      	ldr	r3, [r7, #20]
 8000f98:	1ad3      	subs	r3, r2, r3
 8000f9a:	2b02      	cmp	r3, #2
 8000f9c:	d901      	bls.n	8000fa2 <HAL_RCC_OscConfig+0x26a>
          {
            return HAL_TIMEOUT;
 8000f9e:	2303      	movs	r3, #3
 8000fa0:	e293      	b.n	80014ca <HAL_RCC_OscConfig+0x792>
        while(__HAL_RCC_GET_FLAG(RCC_FLAG_HSIRDY) != 0U)
 8000fa2:	4b34      	ldr	r3, [pc, #208]	; (8001074 <HAL_RCC_OscConfig+0x33c>)
 8000fa4:	681b      	ldr	r3, [r3, #0]
 8000fa6:	2204      	movs	r2, #4
 8000fa8:	4013      	ands	r3, r2
 8000faa:	d1f1      	bne.n	8000f90 <HAL_RCC_OscConfig+0x258>
        }
      }
    }
  }
  /*----------------------------- MSI Configuration --------------------------*/
  if(((RCC_OscInitStruct->OscillatorType) & RCC_OSCILLATORTYPE_MSI) == RCC_OSCILLATORTYPE_MSI)
 8000fac:	687b      	ldr	r3, [r7, #4]
 8000fae:	681b      	ldr	r3, [r3, #0]
 8000fb0:	2210      	movs	r2, #16
 8000fb2:	4013      	ands	r3, r2
 8000fb4:	d100      	bne.n	8000fb8 <HAL_RCC_OscConfig+0x280>
 8000fb6:	e0a2      	b.n	80010fe <HAL_RCC_OscConfig+0x3c6>
  {
    /* When the MSI is used as system clock it will not be disabled */
    if(sysclk_source == RCC_CFGR_SWS_MSI)
 8000fb8:	69fb      	ldr	r3, [r7, #28]
 8000fba:	2b00      	cmp	r3, #0
 8000fbc:	d140      	bne.n	8001040 <HAL_RCC_OscConfig+0x308>
    {
      if((__HAL_RCC_GET_FLAG(RCC_FLAG_MSIRDY) != 0U) && (RCC_OscInitStruct->MSIState == RCC_MSI_OFF))
 8000fbe:	4b2d      	ldr	r3, [pc, #180]	; (8001074 <HAL_RCC_OscConfig+0x33c>)
 8000fc0:	681a      	ldr	r2, [r3, #0]
 8000fc2:	2380      	movs	r3, #128	; 0x80
 8000fc4:	009b      	lsls	r3, r3, #2
 8000fc6:	4013      	ands	r3, r2
 8000fc8:	d005      	beq.n	8000fd6 <HAL_RCC_OscConfig+0x29e>
 8000fca:	687b      	ldr	r3, [r7, #4]
 8000fcc:	69db      	ldr	r3, [r3, #28]
 8000fce:	2b00      	cmp	r3, #0
 8000fd0:	d101      	bne.n	8000fd6 <HAL_RCC_OscConfig+0x29e>
      {
        return HAL_ERROR;
 8000fd2:	2301      	movs	r3, #1
 8000fd4:	e279      	b.n	80014ca <HAL_RCC_OscConfig+0x792>
        /* Check MSICalibrationValue and MSIClockRange input parameters */
        assert_param(IS_RCC_MSICALIBRATION_VALUE(RCC_OscInitStruct->MSICalibrationValue));
        assert_param(IS_RCC_MSI_CLOCK_RANGE(RCC_OscInitStruct->MSIClockRange));

        /* Selects the Multiple Speed oscillator (MSI) clock range .*/
        __HAL_RCC_MSI_RANGE_CONFIG(RCC_OscInitStruct->MSIClockRange);
 8000fd6:	4b27      	ldr	r3, [pc, #156]	; (8001074 <HAL_RCC_OscConfig+0x33c>)
 8000fd8:	685b      	ldr	r3, [r3, #4]
 8000fda:	4a2d      	ldr	r2, [pc, #180]	; (8001090 <HAL_RCC_OscConfig+0x358>)
 8000fdc:	4013      	ands	r3, r2
 8000fde:	0019      	movs	r1, r3
 8000fe0:	687b      	ldr	r3, [r7, #4]
 8000fe2:	6a5a      	ldr	r2, [r3, #36]	; 0x24
 8000fe4:	4b23      	ldr	r3, [pc, #140]	; (8001074 <HAL_RCC_OscConfig+0x33c>)
 8000fe6:	430a      	orrs	r2, r1
 8000fe8:	605a      	str	r2, [r3, #4]
        /* Adjusts the Multiple Speed oscillator (MSI) calibration value.*/
        __HAL_RCC_MSI_CALIBRATIONVALUE_ADJUST(RCC_OscInitStruct->MSICalibrationValue);
 8000fea:	4b22      	ldr	r3, [pc, #136]	; (8001074 <HAL_RCC_OscConfig+0x33c>)
 8000fec:	685b      	ldr	r3, [r3, #4]
 8000fee:	021b      	lsls	r3, r3, #8
 8000ff0:	0a19      	lsrs	r1, r3, #8
 8000ff2:	687b      	ldr	r3, [r7, #4]
 8000ff4:	6a1b      	ldr	r3, [r3, #32]
 8000ff6:	061a      	lsls	r2, r3, #24
 8000ff8:	4b1e      	ldr	r3, [pc, #120]	; (8001074 <HAL_RCC_OscConfig+0x33c>)
 8000ffa:	430a      	orrs	r2, r1
 8000ffc:	605a      	str	r2, [r3, #4]


        /* Update the SystemCoreClock global variable */
        SystemCoreClock =  (32768U * (1UL << ((RCC_OscInitStruct->MSIClockRange >> RCC_ICSCR_MSIRANGE_Pos) + 1U)))
 8000ffe:	687b      	ldr	r3, [r7, #4]
 8001000:	6a5b      	ldr	r3, [r3, #36]	; 0x24
 8001002:	0b5b      	lsrs	r3, r3, #13
 8001004:	3301      	adds	r3, #1
 8001006:	2280      	movs	r2, #128	; 0x80
 8001008:	0212      	lsls	r2, r2, #8
 800100a:	409a      	lsls	r2, r3
                           >> AHBPrescTable[((RCC->CFGR & RCC_CFGR_HPRE) >> RCC_CFGR_HPRE_Pos)];
 800100c:	4b19      	ldr	r3, [pc, #100]	; (8001074 <HAL_RCC_OscConfig+0x33c>)
 800100e:	68db      	ldr	r3, [r3, #12]
 8001010:	091b      	lsrs	r3, r3, #4
 8001012:	210f      	movs	r1, #15
 8001014:	400b      	ands	r3, r1
 8001016:	491b      	ldr	r1, [pc, #108]	; (8001084 <HAL_RCC_OscConfig+0x34c>)
 8001018:	5ccb      	ldrb	r3, [r1, r3]
 800101a:	40da      	lsrs	r2, r3
        SystemCoreClock =  (32768U * (1UL << ((RCC_OscInitStruct->MSIClockRange >> RCC_ICSCR_MSIRANGE_Pos) + 1U)))
 800101c:	4b1a      	ldr	r3, [pc, #104]	; (8001088 <HAL_RCC_OscConfig+0x350>)
 800101e:	601a      	str	r2, [r3, #0]

        /* Configure the source of time base considering new system clocks settings*/
        status = HAL_InitTick (uwTickPrio);
 8001020:	4b1a      	ldr	r3, [pc, #104]	; (800108c <HAL_RCC_OscConfig+0x354>)
 8001022:	681b      	ldr	r3, [r3, #0]
 8001024:	2513      	movs	r5, #19
 8001026:	197c      	adds	r4, r7, r5
 8001028:	0018      	movs	r0, r3
 800102a:	f7ff fbdf 	bl	80007ec <HAL_InitTick>
 800102e:	0003      	movs	r3, r0
 8001030:	7023      	strb	r3, [r4, #0]
        if(status != HAL_OK)
 8001032:	197b      	adds	r3, r7, r5
 8001034:	781b      	ldrb	r3, [r3, #0]
 8001036:	2b00      	cmp	r3, #0
 8001038:	d061      	beq.n	80010fe <HAL_RCC_OscConfig+0x3c6>
        {
          return status;
 800103a:	197b      	adds	r3, r7, r5
 800103c:	781b      	ldrb	r3, [r3, #0]
 800103e:	e244      	b.n	80014ca <HAL_RCC_OscConfig+0x792>
    {
      /* Check MSI State */
      assert_param(IS_RCC_MSI(RCC_OscInitStruct->MSIState));

      /* Check the MSI State */
      if(RCC_OscInitStruct->MSIState != RCC_MSI_OFF)
 8001040:	687b      	ldr	r3, [r7, #4]
 8001042:	69db      	ldr	r3, [r3, #28]
 8001044:	2b00      	cmp	r3, #0
 8001046:	d040      	beq.n	80010ca <HAL_RCC_OscConfig+0x392>
      {
        /* Enable the Multi Speed oscillator (MSI). */
        __HAL_RCC_MSI_ENABLE();
 8001048:	4b0a      	ldr	r3, [pc, #40]	; (8001074 <HAL_RCC_OscConfig+0x33c>)
 800104a:	681a      	ldr	r2, [r3, #0]
 800104c:	4b09      	ldr	r3, [pc, #36]	; (8001074 <HAL_RCC_OscConfig+0x33c>)
 800104e:	2180      	movs	r1, #128	; 0x80
 8001050:	0049      	lsls	r1, r1, #1
 8001052:	430a      	orrs	r2, r1
 8001054:	601a      	str	r2, [r3, #0]

        /* Get Start Tick */
        tickstart = HAL_GetTick();
 8001056:	f7ff fc0f 	bl	8000878 <HAL_GetTick>
 800105a:	0003      	movs	r3, r0
 800105c:	617b      	str	r3, [r7, #20]

        /* Wait till MSI is ready */
        while(__HAL_RCC_GET_FLAG(RCC_FLAG_MSIRDY) == 0U)
 800105e:	e019      	b.n	8001094 <HAL_RCC_OscConfig+0x35c>
        {
          if((HAL_GetTick() - tickstart) > MSI_TIMEOUT_VALUE)
 8001060:	f7ff fc0a 	bl	8000878 <HAL_GetTick>
 8001064:	0002      	movs	r2, r0
 8001066:	697b      	ldr	r3, [r7, #20]
 8001068:	1ad3      	subs	r3, r2, r3
 800106a:	2b02      	cmp	r3, #2
 800106c:	d912      	bls.n	8001094 <HAL_RCC_OscConfig+0x35c>
          {
            return HAL_TIMEOUT;
 800106e:	2303      	movs	r3, #3
 8001070:	e22b      	b.n	80014ca <HAL_RCC_OscConfig+0x792>
 8001072:	46c0      	nop			; (mov r8, r8)
 8001074:	40021000 	.word	0x40021000
 8001078:	fffeffff 	.word	0xfffeffff
 800107c:	fffbffff 	.word	0xfffbffff
 8001080:	ffffe0ff 	.word	0xffffe0ff
 8001084:	080027dc 	.word	0x080027dc
 8001088:	20000000 	.word	0x20000000
 800108c:	20000004 	.word	0x20000004
 8001090:	ffff1fff 	.word	0xffff1fff
        while(__HAL_RCC_GET_FLAG(RCC_FLAG_MSIRDY) == 0U)
 8001094:	4bca      	ldr	r3, [pc, #808]	; (80013c0 <HAL_RCC_OscConfig+0x688>)
 8001096:	681a      	ldr	r2, [r3, #0]
 8001098:	2380      	movs	r3, #128	; 0x80
 800109a:	009b      	lsls	r3, r3, #2
 800109c:	4013      	ands	r3, r2
 800109e:	d0df      	beq.n	8001060 <HAL_RCC_OscConfig+0x328>
        /* Check MSICalibrationValue and MSIClockRange input parameters */
        assert_param(IS_RCC_MSICALIBRATION_VALUE(RCC_OscInitStruct->MSICalibrationValue));
        assert_param(IS_RCC_MSI_CLOCK_RANGE(RCC_OscInitStruct->MSIClockRange));

        /* Selects the Multiple Speed oscillator (MSI) clock range .*/
        __HAL_RCC_MSI_RANGE_CONFIG(RCC_OscInitStruct->MSIClockRange);
 80010a0:	4bc7      	ldr	r3, [pc, #796]	; (80013c0 <HAL_RCC_OscConfig+0x688>)
 80010a2:	685b      	ldr	r3, [r3, #4]
 80010a4:	4ac7      	ldr	r2, [pc, #796]	; (80013c4 <HAL_RCC_OscConfig+0x68c>)
 80010a6:	4013      	ands	r3, r2
 80010a8:	0019      	movs	r1, r3
 80010aa:	687b      	ldr	r3, [r7, #4]
 80010ac:	6a5a      	ldr	r2, [r3, #36]	; 0x24
 80010ae:	4bc4      	ldr	r3, [pc, #784]	; (80013c0 <HAL_RCC_OscConfig+0x688>)
 80010b0:	430a      	orrs	r2, r1
 80010b2:	605a      	str	r2, [r3, #4]
         /* Adjusts the Multiple Speed oscillator (MSI) calibration value.*/
        __HAL_RCC_MSI_CALIBRATIONVALUE_ADJUST(RCC_OscInitStruct->MSICalibrationValue);
 80010b4:	4bc2      	ldr	r3, [pc, #776]	; (80013c0 <HAL_RCC_OscConfig+0x688>)
 80010b6:	685b      	ldr	r3, [r3, #4]
 80010b8:	021b      	lsls	r3, r3, #8
 80010ba:	0a19      	lsrs	r1, r3, #8
 80010bc:	687b      	ldr	r3, [r7, #4]
 80010be:	6a1b      	ldr	r3, [r3, #32]
 80010c0:	061a      	lsls	r2, r3, #24
 80010c2:	4bbf      	ldr	r3, [pc, #764]	; (80013c0 <HAL_RCC_OscConfig+0x688>)
 80010c4:	430a      	orrs	r2, r1
 80010c6:	605a      	str	r2, [r3, #4]
 80010c8:	e019      	b.n	80010fe <HAL_RCC_OscConfig+0x3c6>
      }
      else
      {
        /* Disable the Multi Speed oscillator (MSI). */
        __HAL_RCC_MSI_DISABLE();
 80010ca:	4bbd      	ldr	r3, [pc, #756]	; (80013c0 <HAL_RCC_OscConfig+0x688>)
 80010cc:	681a      	ldr	r2, [r3, #0]
 80010ce:	4bbc      	ldr	r3, [pc, #752]	; (80013c0 <HAL_RCC_OscConfig+0x688>)
 80010d0:	49bd      	ldr	r1, [pc, #756]	; (80013c8 <HAL_RCC_OscConfig+0x690>)
 80010d2:	400a      	ands	r2, r1
 80010d4:	601a      	str	r2, [r3, #0]

        /* Get Start Tick */
        tickstart = HAL_GetTick();
 80010d6:	f7ff fbcf 	bl	8000878 <HAL_GetTick>
 80010da:	0003      	movs	r3, r0
 80010dc:	617b      	str	r3, [r7, #20]

        /* Wait till MSI is ready */
        while(__HAL_RCC_GET_FLAG(RCC_FLAG_MSIRDY) != 0U)
 80010de:	e008      	b.n	80010f2 <HAL_RCC_OscConfig+0x3ba>
        {
          if((HAL_GetTick() - tickstart) > MSI_TIMEOUT_VALUE)
 80010e0:	f7ff fbca 	bl	8000878 <HAL_GetTick>
 80010e4:	0002      	movs	r2, r0
 80010e6:	697b      	ldr	r3, [r7, #20]
 80010e8:	1ad3      	subs	r3, r2, r3
 80010ea:	2b02      	cmp	r3, #2
 80010ec:	d901      	bls.n	80010f2 <HAL_RCC_OscConfig+0x3ba>
          {
            return HAL_TIMEOUT;
 80010ee:	2303      	movs	r3, #3
 80010f0:	e1eb      	b.n	80014ca <HAL_RCC_OscConfig+0x792>
        while(__HAL_RCC_GET_FLAG(RCC_FLAG_MSIRDY) != 0U)
 80010f2:	4bb3      	ldr	r3, [pc, #716]	; (80013c0 <HAL_RCC_OscConfig+0x688>)
 80010f4:	681a      	ldr	r2, [r3, #0]
 80010f6:	2380      	movs	r3, #128	; 0x80
 80010f8:	009b      	lsls	r3, r3, #2
 80010fa:	4013      	ands	r3, r2
 80010fc:	d1f0      	bne.n	80010e0 <HAL_RCC_OscConfig+0x3a8>
        }
      }
    }
  }
  /*------------------------------ LSI Configuration -------------------------*/
  if(((RCC_OscInitStruct->OscillatorType) & RCC_OSCILLATORTYPE_LSI) == RCC_OSCILLATORTYPE_LSI)
 80010fe:	687b      	ldr	r3, [r7, #4]
 8001100:	681b      	ldr	r3, [r3, #0]
 8001102:	2208      	movs	r2, #8
 8001104:	4013      	ands	r3, r2
 8001106:	d036      	beq.n	8001176 <HAL_RCC_OscConfig+0x43e>
  {
    /* Check the parameters */
    assert_param(IS_RCC_LSI(RCC_OscInitStruct->LSIState));

    /* Check the LSI State */
    if(RCC_OscInitStruct->LSIState != RCC_LSI_OFF)
 8001108:	687b      	ldr	r3, [r7, #4]
 800110a:	695b      	ldr	r3, [r3, #20]
 800110c:	2b00      	cmp	r3, #0
 800110e:	d019      	beq.n	8001144 <HAL_RCC_OscConfig+0x40c>
    {
      /* Enable the Internal Low Speed oscillator (LSI). */
      __HAL_RCC_LSI_ENABLE();
 8001110:	4bab      	ldr	r3, [pc, #684]	; (80013c0 <HAL_RCC_OscConfig+0x688>)
 8001112:	6d1a      	ldr	r2, [r3, #80]	; 0x50
 8001114:	4baa      	ldr	r3, [pc, #680]	; (80013c0 <HAL_RCC_OscConfig+0x688>)
 8001116:	2101      	movs	r1, #1
 8001118:	430a      	orrs	r2, r1
 800111a:	651a      	str	r2, [r3, #80]	; 0x50

      /* Get Start Tick */
      tickstart = HAL_GetTick();
 800111c:	f7ff fbac 	bl	8000878 <HAL_GetTick>
 8001120:	0003      	movs	r3, r0
 8001122:	617b      	str	r3, [r7, #20]

      /* Wait till LSI is ready */
      while(__HAL_RCC_GET_FLAG(RCC_FLAG_LSIRDY) == 0U)
 8001124:	e008      	b.n	8001138 <HAL_RCC_OscConfig+0x400>
      {
        if((HAL_GetTick() - tickstart ) > LSI_TIMEOUT_VALUE)
 8001126:	f7ff fba7 	bl	8000878 <HAL_GetTick>
 800112a:	0002      	movs	r2, r0
 800112c:	697b      	ldr	r3, [r7, #20]
 800112e:	1ad3      	subs	r3, r2, r3
 8001130:	2b02      	cmp	r3, #2
 8001132:	d901      	bls.n	8001138 <HAL_RCC_OscConfig+0x400>
        {
          return HAL_TIMEOUT;
 8001134:	2303      	movs	r3, #3
 8001136:	e1c8      	b.n	80014ca <HAL_RCC_OscConfig+0x792>
      while(__HAL_RCC_GET_FLAG(RCC_FLAG_LSIRDY) == 0U)
 8001138:	4ba1      	ldr	r3, [pc, #644]	; (80013c0 <HAL_RCC_OscConfig+0x688>)
 800113a:	6d1b      	ldr	r3, [r3, #80]	; 0x50
 800113c:	2202      	movs	r2, #2
 800113e:	4013      	ands	r3, r2
 8001140:	d0f1      	beq.n	8001126 <HAL_RCC_OscConfig+0x3ee>
 8001142:	e018      	b.n	8001176 <HAL_RCC_OscConfig+0x43e>
      }
    }
    else
    {
      /* Disable the Internal Low Speed oscillator (LSI). */
      __HAL_RCC_LSI_DISABLE();
 8001144:	4b9e      	ldr	r3, [pc, #632]	; (80013c0 <HAL_RCC_OscConfig+0x688>)
 8001146:	6d1a      	ldr	r2, [r3, #80]	; 0x50
 8001148:	4b9d      	ldr	r3, [pc, #628]	; (80013c0 <HAL_RCC_OscConfig+0x688>)
 800114a:	2101      	movs	r1, #1
 800114c:	438a      	bics	r2, r1
 800114e:	651a      	str	r2, [r3, #80]	; 0x50

      /* Get Start Tick */
      tickstart = HAL_GetTick();
 8001150:	f7ff fb92 	bl	8000878 <HAL_GetTick>
 8001154:	0003      	movs	r3, r0
 8001156:	617b      	str	r3, [r7, #20]

      /* Wait till LSI is disabled */
      while(__HAL_RCC_GET_FLAG(RCC_FLAG_LSIRDY) != 0U)
 8001158:	e008      	b.n	800116c <HAL_RCC_OscConfig+0x434>
      {
        if((HAL_GetTick() - tickstart ) > LSI_TIMEOUT_VALUE)
 800115a:	f7ff fb8d 	bl	8000878 <HAL_GetTick>
 800115e:	0002      	movs	r2, r0
 8001160:	697b      	ldr	r3, [r7, #20]
 8001162:	1ad3      	subs	r3, r2, r3
 8001164:	2b02      	cmp	r3, #2
 8001166:	d901      	bls.n	800116c <HAL_RCC_OscConfig+0x434>
        {
          return HAL_TIMEOUT;
 8001168:	2303      	movs	r3, #3
 800116a:	e1ae      	b.n	80014ca <HAL_RCC_OscConfig+0x792>
      while(__HAL_RCC_GET_FLAG(RCC_FLAG_LSIRDY) != 0U)
 800116c:	4b94      	ldr	r3, [pc, #592]	; (80013c0 <HAL_RCC_OscConfig+0x688>)
 800116e:	6d1b      	ldr	r3, [r3, #80]	; 0x50
 8001170:	2202      	movs	r2, #2
 8001172:	4013      	ands	r3, r2
 8001174:	d1f1      	bne.n	800115a <HAL_RCC_OscConfig+0x422>
        }
      }
    }
  }
  /*------------------------------ LSE Configuration -------------------------*/
  if(((RCC_OscInitStruct->OscillatorType) & RCC_OSCILLATORTYPE_LSE) == RCC_OSCILLATORTYPE_LSE)
 8001176:	687b      	ldr	r3, [r7, #4]
 8001178:	681b      	ldr	r3, [r3, #0]
 800117a:	2204      	movs	r2, #4
 800117c:	4013      	ands	r3, r2
 800117e:	d100      	bne.n	8001182 <HAL_RCC_OscConfig+0x44a>
 8001180:	e0ae      	b.n	80012e0 <HAL_RCC_OscConfig+0x5a8>
  {
    FlagStatus       pwrclkchanged = RESET;
 8001182:	2023      	movs	r0, #35	; 0x23
 8001184:	183b      	adds	r3, r7, r0
 8001186:	2200      	movs	r2, #0
 8001188:	701a      	strb	r2, [r3, #0]
    /* Check the parameters */
    assert_param(IS_RCC_LSE(RCC_OscInitStruct->LSEState));

    /* Update LSE configuration in Backup Domain control register    */
    /* Requires to enable write access to Backup Domain of necessary */
    if(__HAL_RCC_PWR_IS_CLK_DISABLED())
 800118a:	4b8d      	ldr	r3, [pc, #564]	; (80013c0 <HAL_RCC_OscConfig+0x688>)
 800118c:	6b9a      	ldr	r2, [r3, #56]	; 0x38
 800118e:	2380      	movs	r3, #128	; 0x80
 8001190:	055b      	lsls	r3, r3, #21
 8001192:	4013      	ands	r3, r2
 8001194:	d109      	bne.n	80011aa <HAL_RCC_OscConfig+0x472>
    {
      __HAL_RCC_PWR_CLK_ENABLE();
 8001196:	4b8a      	ldr	r3, [pc, #552]	; (80013c0 <HAL_RCC_OscConfig+0x688>)
 8001198:	6b9a      	ldr	r2, [r3, #56]	; 0x38
 800119a:	4b89      	ldr	r3, [pc, #548]	; (80013c0 <HAL_RCC_OscConfig+0x688>)
 800119c:	2180      	movs	r1, #128	; 0x80
 800119e:	0549      	lsls	r1, r1, #21
 80011a0:	430a      	orrs	r2, r1
 80011a2:	639a      	str	r2, [r3, #56]	; 0x38
      pwrclkchanged = SET;
 80011a4:	183b      	adds	r3, r7, r0
 80011a6:	2201      	movs	r2, #1
 80011a8:	701a      	strb	r2, [r3, #0]
    }

    if(HAL_IS_BIT_CLR(PWR->CR, PWR_CR_DBP))
 80011aa:	4b88      	ldr	r3, [pc, #544]	; (80013cc <HAL_RCC_OscConfig+0x694>)
 80011ac:	681a      	ldr	r2, [r3, #0]
 80011ae:	2380      	movs	r3, #128	; 0x80
 80011b0:	005b      	lsls	r3, r3, #1
 80011b2:	4013      	ands	r3, r2
 80011b4:	d11a      	bne.n	80011ec <HAL_RCC_OscConfig+0x4b4>
    {
      /* Enable write access to Backup domain */
      SET_BIT(PWR->CR, PWR_CR_DBP);
 80011b6:	4b85      	ldr	r3, [pc, #532]	; (80013cc <HAL_RCC_OscConfig+0x694>)
 80011b8:	681a      	ldr	r2, [r3, #0]
 80011ba:	4b84      	ldr	r3, [pc, #528]	; (80013cc <HAL_RCC_OscConfig+0x694>)
 80011bc:	2180      	movs	r1, #128	; 0x80
 80011be:	0049      	lsls	r1, r1, #1
 80011c0:	430a      	orrs	r2, r1
 80011c2:	601a      	str	r2, [r3, #0]

      /* Wait for Backup domain Write protection disable */
      tickstart = HAL_GetTick();
 80011c4:	f7ff fb58 	bl	8000878 <HAL_GetTick>
 80011c8:	0003      	movs	r3, r0
 80011ca:	617b      	str	r3, [r7, #20]

      while(HAL_IS_BIT_CLR(PWR->CR, PWR_CR_DBP))
 80011cc:	e008      	b.n	80011e0 <HAL_RCC_OscConfig+0x4a8>
      {
        if((HAL_GetTick() - tickstart) > RCC_DBP_TIMEOUT_VALUE)
 80011ce:	f7ff fb53 	bl	8000878 <HAL_GetTick>
 80011d2:	0002      	movs	r2, r0
 80011d4:	697b      	ldr	r3, [r7, #20]
 80011d6:	1ad3      	subs	r3, r2, r3
 80011d8:	2b64      	cmp	r3, #100	; 0x64
 80011da:	d901      	bls.n	80011e0 <HAL_RCC_OscConfig+0x4a8>
        {
          return HAL_TIMEOUT;
 80011dc:	2303      	movs	r3, #3
 80011de:	e174      	b.n	80014ca <HAL_RCC_OscConfig+0x792>
      while(HAL_IS_BIT_CLR(PWR->CR, PWR_CR_DBP))
 80011e0:	4b7a      	ldr	r3, [pc, #488]	; (80013cc <HAL_RCC_OscConfig+0x694>)
 80011e2:	681a      	ldr	r2, [r3, #0]
 80011e4:	2380      	movs	r3, #128	; 0x80
 80011e6:	005b      	lsls	r3, r3, #1
 80011e8:	4013      	ands	r3, r2
 80011ea:	d0f0      	beq.n	80011ce <HAL_RCC_OscConfig+0x496>
        }
      }
    }

    /* Set the new LSE configuration -----------------------------------------*/
    __HAL_RCC_LSE_CONFIG(RCC_OscInitStruct->LSEState);
 80011ec:	687b      	ldr	r3, [r7, #4]
 80011ee:	689a      	ldr	r2, [r3, #8]
 80011f0:	2380      	movs	r3, #128	; 0x80
 80011f2:	005b      	lsls	r3, r3, #1
 80011f4:	429a      	cmp	r2, r3
 80011f6:	d107      	bne.n	8001208 <HAL_RCC_OscConfig+0x4d0>
 80011f8:	4b71      	ldr	r3, [pc, #452]	; (80013c0 <HAL_RCC_OscConfig+0x688>)
 80011fa:	6d1a      	ldr	r2, [r3, #80]	; 0x50
 80011fc:	4b70      	ldr	r3, [pc, #448]	; (80013c0 <HAL_RCC_OscConfig+0x688>)
 80011fe:	2180      	movs	r1, #128	; 0x80
 8001200:	0049      	lsls	r1, r1, #1
 8001202:	430a      	orrs	r2, r1
 8001204:	651a      	str	r2, [r3, #80]	; 0x50
 8001206:	e031      	b.n	800126c <HAL_RCC_OscConfig+0x534>
 8001208:	687b      	ldr	r3, [r7, #4]
 800120a:	689b      	ldr	r3, [r3, #8]
 800120c:	2b00      	cmp	r3, #0
 800120e:	d10c      	bne.n	800122a <HAL_RCC_OscConfig+0x4f2>
 8001210:	4b6b      	ldr	r3, [pc, #428]	; (80013c0 <HAL_RCC_OscConfig+0x688>)
 8001212:	6d1a      	ldr	r2, [r3, #80]	; 0x50
 8001214:	4b6a      	ldr	r3, [pc, #424]	; (80013c0 <HAL_RCC_OscConfig+0x688>)
 8001216:	496c      	ldr	r1, [pc, #432]	; (80013c8 <HAL_RCC_OscConfig+0x690>)
 8001218:	400a      	ands	r2, r1
 800121a:	651a      	str	r2, [r3, #80]	; 0x50
 800121c:	4b68      	ldr	r3, [pc, #416]	; (80013c0 <HAL_RCC_OscConfig+0x688>)
 800121e:	6d1a      	ldr	r2, [r3, #80]	; 0x50
 8001220:	4b67      	ldr	r3, [pc, #412]	; (80013c0 <HAL_RCC_OscConfig+0x688>)
 8001222:	496b      	ldr	r1, [pc, #428]	; (80013d0 <HAL_RCC_OscConfig+0x698>)
 8001224:	400a      	ands	r2, r1
 8001226:	651a      	str	r2, [r3, #80]	; 0x50
 8001228:	e020      	b.n	800126c <HAL_RCC_OscConfig+0x534>
 800122a:	687b      	ldr	r3, [r7, #4]
 800122c:	689a      	ldr	r2, [r3, #8]
 800122e:	23a0      	movs	r3, #160	; 0xa0
 8001230:	00db      	lsls	r3, r3, #3
 8001232:	429a      	cmp	r2, r3
 8001234:	d10e      	bne.n	8001254 <HAL_RCC_OscConfig+0x51c>
 8001236:	4b62      	ldr	r3, [pc, #392]	; (80013c0 <HAL_RCC_OscConfig+0x688>)
 8001238:	6d1a      	ldr	r2, [r3, #80]	; 0x50
 800123a:	4b61      	ldr	r3, [pc, #388]	; (80013c0 <HAL_RCC_OscConfig+0x688>)
 800123c:	2180      	movs	r1, #128	; 0x80
 800123e:	00c9      	lsls	r1, r1, #3
 8001240:	430a      	orrs	r2, r1
 8001242:	651a      	str	r2, [r3, #80]	; 0x50
 8001244:	4b5e      	ldr	r3, [pc, #376]	; (80013c0 <HAL_RCC_OscConfig+0x688>)
 8001246:	6d1a      	ldr	r2, [r3, #80]	; 0x50
 8001248:	4b5d      	ldr	r3, [pc, #372]	; (80013c0 <HAL_RCC_OscConfig+0x688>)
 800124a:	2180      	movs	r1, #128	; 0x80
 800124c:	0049      	lsls	r1, r1, #1
 800124e:	430a      	orrs	r2, r1
 8001250:	651a      	str	r2, [r3, #80]	; 0x50
 8001252:	e00b      	b.n	800126c <HAL_RCC_OscConfig+0x534>
 8001254:	4b5a      	ldr	r3, [pc, #360]	; (80013c0 <HAL_RCC_OscConfig+0x688>)
 8001256:	6d1a      	ldr	r2, [r3, #80]	; 0x50
 8001258:	4b59      	ldr	r3, [pc, #356]	; (80013c0 <HAL_RCC_OscConfig+0x688>)
 800125a:	495b      	ldr	r1, [pc, #364]	; (80013c8 <HAL_RCC_OscConfig+0x690>)
 800125c:	400a      	ands	r2, r1
 800125e:	651a      	str	r2, [r3, #80]	; 0x50
 8001260:	4b57      	ldr	r3, [pc, #348]	; (80013c0 <HAL_RCC_OscConfig+0x688>)
 8001262:	6d1a      	ldr	r2, [r3, #80]	; 0x50
 8001264:	4b56      	ldr	r3, [pc, #344]	; (80013c0 <HAL_RCC_OscConfig+0x688>)
 8001266:	495a      	ldr	r1, [pc, #360]	; (80013d0 <HAL_RCC_OscConfig+0x698>)
 8001268:	400a      	ands	r2, r1
 800126a:	651a      	str	r2, [r3, #80]	; 0x50

    /* Check the LSE State */
    if(RCC_OscInitStruct->LSEState != RCC_LSE_OFF)
 800126c:	687b      	ldr	r3, [r7, #4]
 800126e:	689b      	ldr	r3, [r3, #8]
 8001270:	2b00      	cmp	r3, #0
 8001272:	d015      	beq.n	80012a0 <HAL_RCC_OscConfig+0x568>
    {
      /* Get Start Tick */
      tickstart = HAL_GetTick();
 8001274:	f7ff fb00 	bl	8000878 <HAL_GetTick>
 8001278:	0003      	movs	r3, r0
 800127a:	617b      	str	r3, [r7, #20]

      /* Wait till LSE is ready */
      while(__HAL_RCC_GET_FLAG(RCC_FLAG_LSERDY) == 0U)
 800127c:	e009      	b.n	8001292 <HAL_RCC_OscConfig+0x55a>
      {
        if((HAL_GetTick() - tickstart ) > RCC_LSE_TIMEOUT_VALUE)
 800127e:	f7ff fafb 	bl	8000878 <HAL_GetTick>
 8001282:	0002      	movs	r2, r0
 8001284:	697b      	ldr	r3, [r7, #20]
 8001286:	1ad3      	subs	r3, r2, r3
 8001288:	4a52      	ldr	r2, [pc, #328]	; (80013d4 <HAL_RCC_OscConfig+0x69c>)
 800128a:	4293      	cmp	r3, r2
 800128c:	d901      	bls.n	8001292 <HAL_RCC_OscConfig+0x55a>
        {
          return HAL_TIMEOUT;
 800128e:	2303      	movs	r3, #3
 8001290:	e11b      	b.n	80014ca <HAL_RCC_OscConfig+0x792>
      while(__HAL_RCC_GET_FLAG(RCC_FLAG_LSERDY) == 0U)
 8001292:	4b4b      	ldr	r3, [pc, #300]	; (80013c0 <HAL_RCC_OscConfig+0x688>)
 8001294:	6d1a      	ldr	r2, [r3, #80]	; 0x50
 8001296:	2380      	movs	r3, #128	; 0x80
 8001298:	009b      	lsls	r3, r3, #2
 800129a:	4013      	ands	r3, r2
 800129c:	d0ef      	beq.n	800127e <HAL_RCC_OscConfig+0x546>
 800129e:	e014      	b.n	80012ca <HAL_RCC_OscConfig+0x592>
      }
    }
    else
    {
      /* Get Start Tick */
      tickstart = HAL_GetTick();
 80012a0:	f7ff faea 	bl	8000878 <HAL_GetTick>
 80012a4:	0003      	movs	r3, r0
 80012a6:	617b      	str	r3, [r7, #20]

      /* Wait till LSE is disabled */
      while(__HAL_RCC_GET_FLAG(RCC_FLAG_LSERDY) != 0U)
 80012a8:	e009      	b.n	80012be <HAL_RCC_OscConfig+0x586>
      {
        if((HAL_GetTick() - tickstart ) > RCC_LSE_TIMEOUT_VALUE)
 80012aa:	f7ff fae5 	bl	8000878 <HAL_GetTick>
 80012ae:	0002      	movs	r2, r0
 80012b0:	697b      	ldr	r3, [r7, #20]
 80012b2:	1ad3      	subs	r3, r2, r3
 80012b4:	4a47      	ldr	r2, [pc, #284]	; (80013d4 <HAL_RCC_OscConfig+0x69c>)
 80012b6:	4293      	cmp	r3, r2
 80012b8:	d901      	bls.n	80012be <HAL_RCC_OscConfig+0x586>
        {
          return HAL_TIMEOUT;
 80012ba:	2303      	movs	r3, #3
 80012bc:	e105      	b.n	80014ca <HAL_RCC_OscConfig+0x792>
      while(__HAL_RCC_GET_FLAG(RCC_FLAG_LSERDY) != 0U)
 80012be:	4b40      	ldr	r3, [pc, #256]	; (80013c0 <HAL_RCC_OscConfig+0x688>)
 80012c0:	6d1a      	ldr	r2, [r3, #80]	; 0x50
 80012c2:	2380      	movs	r3, #128	; 0x80
 80012c4:	009b      	lsls	r3, r3, #2
 80012c6:	4013      	ands	r3, r2
 80012c8:	d1ef      	bne.n	80012aa <HAL_RCC_OscConfig+0x572>
        }
      }
    }

    /* Require to disable power clock if necessary */
    if(pwrclkchanged == SET)
 80012ca:	2323      	movs	r3, #35	; 0x23
 80012cc:	18fb      	adds	r3, r7, r3
 80012ce:	781b      	ldrb	r3, [r3, #0]
 80012d0:	2b01      	cmp	r3, #1
 80012d2:	d105      	bne.n	80012e0 <HAL_RCC_OscConfig+0x5a8>
    {
      __HAL_RCC_PWR_CLK_DISABLE();
 80012d4:	4b3a      	ldr	r3, [pc, #232]	; (80013c0 <HAL_RCC_OscConfig+0x688>)
 80012d6:	6b9a      	ldr	r2, [r3, #56]	; 0x38
 80012d8:	4b39      	ldr	r3, [pc, #228]	; (80013c0 <HAL_RCC_OscConfig+0x688>)
 80012da:	493f      	ldr	r1, [pc, #252]	; (80013d8 <HAL_RCC_OscConfig+0x6a0>)
 80012dc:	400a      	ands	r2, r1
 80012de:	639a      	str	r2, [r3, #56]	; 0x38
    }
  }

#if defined(RCC_HSI48_SUPPORT)
  /*----------------------------- HSI48 Configuration --------------------------*/
  if(((RCC_OscInitStruct->OscillatorType) & RCC_OSCILLATORTYPE_HSI48) == RCC_OSCILLATORTYPE_HSI48)
 80012e0:	687b      	ldr	r3, [r7, #4]
 80012e2:	681b      	ldr	r3, [r3, #0]
 80012e4:	2220      	movs	r2, #32
 80012e6:	4013      	ands	r3, r2
 80012e8:	d049      	beq.n	800137e <HAL_RCC_OscConfig+0x646>
  {
    /* Check the parameters */
    assert_param(IS_RCC_HSI48(RCC_OscInitStruct->HSI48State));

      /* Check the HSI48 State */
      if(RCC_OscInitStruct->HSI48State != RCC_HSI48_OFF)
 80012ea:	687b      	ldr	r3, [r7, #4]
 80012ec:	699b      	ldr	r3, [r3, #24]
 80012ee:	2b00      	cmp	r3, #0
 80012f0:	d026      	beq.n	8001340 <HAL_RCC_OscConfig+0x608>
      {
        /* Enable the Internal High Speed oscillator (HSI48). */
        __HAL_RCC_HSI48_ENABLE();
 80012f2:	4b33      	ldr	r3, [pc, #204]	; (80013c0 <HAL_RCC_OscConfig+0x688>)
 80012f4:	689a      	ldr	r2, [r3, #8]
 80012f6:	4b32      	ldr	r3, [pc, #200]	; (80013c0 <HAL_RCC_OscConfig+0x688>)
 80012f8:	2101      	movs	r1, #1
 80012fa:	430a      	orrs	r2, r1
 80012fc:	609a      	str	r2, [r3, #8]
 80012fe:	4b30      	ldr	r3, [pc, #192]	; (80013c0 <HAL_RCC_OscConfig+0x688>)
 8001300:	6b5a      	ldr	r2, [r3, #52]	; 0x34
 8001302:	4b2f      	ldr	r3, [pc, #188]	; (80013c0 <HAL_RCC_OscConfig+0x688>)
 8001304:	2101      	movs	r1, #1
 8001306:	430a      	orrs	r2, r1
 8001308:	635a      	str	r2, [r3, #52]	; 0x34
 800130a:	4b34      	ldr	r3, [pc, #208]	; (80013dc <HAL_RCC_OscConfig+0x6a4>)
 800130c:	6a1a      	ldr	r2, [r3, #32]
 800130e:	4b33      	ldr	r3, [pc, #204]	; (80013dc <HAL_RCC_OscConfig+0x6a4>)
 8001310:	2180      	movs	r1, #128	; 0x80
 8001312:	0189      	lsls	r1, r1, #6
 8001314:	430a      	orrs	r2, r1
 8001316:	621a      	str	r2, [r3, #32]

        /* Get Start Tick */
        tickstart = HAL_GetTick();
 8001318:	f7ff faae 	bl	8000878 <HAL_GetTick>
 800131c:	0003      	movs	r3, r0
 800131e:	617b      	str	r3, [r7, #20]

        /* Wait till HSI48 is ready */
        while(__HAL_RCC_GET_FLAG(RCC_FLAG_HSI48RDY) == 0U)
 8001320:	e008      	b.n	8001334 <HAL_RCC_OscConfig+0x5fc>
        {
          if((HAL_GetTick() - tickstart) > HSI48_TIMEOUT_VALUE)
 8001322:	f7ff faa9 	bl	8000878 <HAL_GetTick>
 8001326:	0002      	movs	r2, r0
 8001328:	697b      	ldr	r3, [r7, #20]
 800132a:	1ad3      	subs	r3, r2, r3
 800132c:	2b02      	cmp	r3, #2
 800132e:	d901      	bls.n	8001334 <HAL_RCC_OscConfig+0x5fc>
          {
            return HAL_TIMEOUT;
 8001330:	2303      	movs	r3, #3
 8001332:	e0ca      	b.n	80014ca <HAL_RCC_OscConfig+0x792>
        while(__HAL_RCC_GET_FLAG(RCC_FLAG_HSI48RDY) == 0U)
 8001334:	4b22      	ldr	r3, [pc, #136]	; (80013c0 <HAL_RCC_OscConfig+0x688>)
 8001336:	689b      	ldr	r3, [r3, #8]
 8001338:	2202      	movs	r2, #2
 800133a:	4013      	ands	r3, r2
 800133c:	d0f1      	beq.n	8001322 <HAL_RCC_OscConfig+0x5ea>
 800133e:	e01e      	b.n	800137e <HAL_RCC_OscConfig+0x646>
        }
      }
      else
      {
        /* Disable the Internal High Speed oscillator (HSI48). */
        __HAL_RCC_HSI48_DISABLE();
 8001340:	4b1f      	ldr	r3, [pc, #124]	; (80013c0 <HAL_RCC_OscConfig+0x688>)
 8001342:	689a      	ldr	r2, [r3, #8]
 8001344:	4b1e      	ldr	r3, [pc, #120]	; (80013c0 <HAL_RCC_OscConfig+0x688>)
 8001346:	2101      	movs	r1, #1
 8001348:	438a      	bics	r2, r1
 800134a:	609a      	str	r2, [r3, #8]
 800134c:	4b23      	ldr	r3, [pc, #140]	; (80013dc <HAL_RCC_OscConfig+0x6a4>)
 800134e:	6a1a      	ldr	r2, [r3, #32]
 8001350:	4b22      	ldr	r3, [pc, #136]	; (80013dc <HAL_RCC_OscConfig+0x6a4>)
 8001352:	4923      	ldr	r1, [pc, #140]	; (80013e0 <HAL_RCC_OscConfig+0x6a8>)
 8001354:	400a      	ands	r2, r1
 8001356:	621a      	str	r2, [r3, #32]

        /* Get Start Tick */
        tickstart = HAL_GetTick();
 8001358:	f7ff fa8e 	bl	8000878 <HAL_GetTick>
 800135c:	0003      	movs	r3, r0
 800135e:	617b      	str	r3, [r7, #20]

        /* Wait till HSI48 is ready */
        while(__HAL_RCC_GET_FLAG(RCC_FLAG_HSI48RDY) != 0U)
 8001360:	e008      	b.n	8001374 <HAL_RCC_OscConfig+0x63c>
        {
          if((HAL_GetTick() - tickstart) > HSI48_TIMEOUT_VALUE)
 8001362:	f7ff fa89 	bl	8000878 <HAL_GetTick>
 8001366:	0002      	movs	r2, r0
 8001368:	697b      	ldr	r3, [r7, #20]
 800136a:	1ad3      	subs	r3, r2, r3
 800136c:	2b02      	cmp	r3, #2
 800136e:	d901      	bls.n	8001374 <HAL_RCC_OscConfig+0x63c>
          {
            return HAL_TIMEOUT;
 8001370:	2303      	movs	r3, #3
 8001372:	e0aa      	b.n	80014ca <HAL_RCC_OscConfig+0x792>
        while(__HAL_RCC_GET_FLAG(RCC_FLAG_HSI48RDY) != 0U)
 8001374:	4b12      	ldr	r3, [pc, #72]	; (80013c0 <HAL_RCC_OscConfig+0x688>)
 8001376:	689b      	ldr	r3, [r3, #8]
 8001378:	2202      	movs	r2, #2
 800137a:	4013      	ands	r3, r2
 800137c:	d1f1      	bne.n	8001362 <HAL_RCC_OscConfig+0x62a>
#endif /* RCC_HSI48_SUPPORT */

  /*-------------------------------- PLL Configuration -----------------------*/
  /* Check the parameters */
  assert_param(IS_RCC_PLL(RCC_OscInitStruct->PLL.PLLState));
  if ((RCC_OscInitStruct->PLL.PLLState) != RCC_PLL_NONE)
 800137e:	687b      	ldr	r3, [r7, #4]
 8001380:	6a9b      	ldr	r3, [r3, #40]	; 0x28
 8001382:	2b00      	cmp	r3, #0
 8001384:	d100      	bne.n	8001388 <HAL_RCC_OscConfig+0x650>
 8001386:	e09f      	b.n	80014c8 <HAL_RCC_OscConfig+0x790>
  {
    /* Check if the PLL is used as system clock or not */
    if(sysclk_source != RCC_SYSCLKSOURCE_STATUS_PLLCLK)
 8001388:	69fb      	ldr	r3, [r7, #28]
 800138a:	2b0c      	cmp	r3, #12
 800138c:	d100      	bne.n	8001390 <HAL_RCC_OscConfig+0x658>
 800138e:	e078      	b.n	8001482 <HAL_RCC_OscConfig+0x74a>
    {
      if((RCC_OscInitStruct->PLL.PLLState) == RCC_PLL_ON)
 8001390:	687b      	ldr	r3, [r7, #4]
 8001392:	6a9b      	ldr	r3, [r3, #40]	; 0x28
 8001394:	2b02      	cmp	r3, #2
 8001396:	d159      	bne.n	800144c <HAL_RCC_OscConfig+0x714>
        assert_param(IS_RCC_PLLSOURCE(RCC_OscInitStruct->PLL.PLLSource));
        assert_param(IS_RCC_PLL_MUL(RCC_OscInitStruct->PLL.PLLMUL));
        assert_param(IS_RCC_PLL_DIV(RCC_OscInitStruct->PLL.PLLDIV));

        /* Disable the main PLL. */
        __HAL_RCC_PLL_DISABLE();
 8001398:	4b09      	ldr	r3, [pc, #36]	; (80013c0 <HAL_RCC_OscConfig+0x688>)
 800139a:	681a      	ldr	r2, [r3, #0]
 800139c:	4b08      	ldr	r3, [pc, #32]	; (80013c0 <HAL_RCC_OscConfig+0x688>)
 800139e:	4911      	ldr	r1, [pc, #68]	; (80013e4 <HAL_RCC_OscConfig+0x6ac>)
 80013a0:	400a      	ands	r2, r1
 80013a2:	601a      	str	r2, [r3, #0]

        /* Get Start Tick */
        tickstart = HAL_GetTick();
 80013a4:	f7ff fa68 	bl	8000878 <HAL_GetTick>
 80013a8:	0003      	movs	r3, r0
 80013aa:	617b      	str	r3, [r7, #20]

        /* Wait till PLL is ready */
        while(__HAL_RCC_GET_FLAG(RCC_FLAG_PLLRDY)  != 0U)
 80013ac:	e01c      	b.n	80013e8 <HAL_RCC_OscConfig+0x6b0>
        {
          if((HAL_GetTick() - tickstart ) > PLL_TIMEOUT_VALUE)
 80013ae:	f7ff fa63 	bl	8000878 <HAL_GetTick>
 80013b2:	0002      	movs	r2, r0
 80013b4:	697b      	ldr	r3, [r7, #20]
 80013b6:	1ad3      	subs	r3, r2, r3
 80013b8:	2b02      	cmp	r3, #2
 80013ba:	d915      	bls.n	80013e8 <HAL_RCC_OscConfig+0x6b0>
          {
            return HAL_TIMEOUT;
 80013bc:	2303      	movs	r3, #3
 80013be:	e084      	b.n	80014ca <HAL_RCC_OscConfig+0x792>
 80013c0:	40021000 	.word	0x40021000
 80013c4:	ffff1fff 	.word	0xffff1fff
 80013c8:	fffffeff 	.word	0xfffffeff
 80013cc:	40007000 	.word	0x40007000
 80013d0:	fffffbff 	.word	0xfffffbff
 80013d4:	00001388 	.word	0x00001388
 80013d8:	efffffff 	.word	0xefffffff
 80013dc:	40010000 	.word	0x40010000
 80013e0:	ffffdfff 	.word	0xffffdfff
 80013e4:	feffffff 	.word	0xfeffffff
        while(__HAL_RCC_GET_FLAG(RCC_FLAG_PLLRDY)  != 0U)
 80013e8:	4b3a      	ldr	r3, [pc, #232]	; (80014d4 <HAL_RCC_OscConfig+0x79c>)
 80013ea:	681a      	ldr	r2, [r3, #0]
 80013ec:	2380      	movs	r3, #128	; 0x80
 80013ee:	049b      	lsls	r3, r3, #18
 80013f0:	4013      	ands	r3, r2
 80013f2:	d1dc      	bne.n	80013ae <HAL_RCC_OscConfig+0x676>
          }
        }

        /* Configure the main PLL clock source, multiplication and division factors. */
        __HAL_RCC_PLL_CONFIG(RCC_OscInitStruct->PLL.PLLSource,
 80013f4:	4b37      	ldr	r3, [pc, #220]	; (80014d4 <HAL_RCC_OscConfig+0x79c>)
 80013f6:	68db      	ldr	r3, [r3, #12]
 80013f8:	4a37      	ldr	r2, [pc, #220]	; (80014d8 <HAL_RCC_OscConfig+0x7a0>)
 80013fa:	4013      	ands	r3, r2
 80013fc:	0019      	movs	r1, r3
 80013fe:	687b      	ldr	r3, [r7, #4]
 8001400:	6ada      	ldr	r2, [r3, #44]	; 0x2c
 8001402:	687b      	ldr	r3, [r7, #4]
 8001404:	6b1b      	ldr	r3, [r3, #48]	; 0x30
 8001406:	431a      	orrs	r2, r3
 8001408:	687b      	ldr	r3, [r7, #4]
 800140a:	6b5b      	ldr	r3, [r3, #52]	; 0x34
 800140c:	431a      	orrs	r2, r3
 800140e:	4b31      	ldr	r3, [pc, #196]	; (80014d4 <HAL_RCC_OscConfig+0x79c>)
 8001410:	430a      	orrs	r2, r1
 8001412:	60da      	str	r2, [r3, #12]
                             RCC_OscInitStruct->PLL.PLLMUL,
                             RCC_OscInitStruct->PLL.PLLDIV);
        /* Enable the main PLL. */
        __HAL_RCC_PLL_ENABLE();
 8001414:	4b2f      	ldr	r3, [pc, #188]	; (80014d4 <HAL_RCC_OscConfig+0x79c>)
 8001416:	681a      	ldr	r2, [r3, #0]
 8001418:	4b2e      	ldr	r3, [pc, #184]	; (80014d4 <HAL_RCC_OscConfig+0x79c>)
 800141a:	2180      	movs	r1, #128	; 0x80
 800141c:	0449      	lsls	r1, r1, #17
 800141e:	430a      	orrs	r2, r1
 8001420:	601a      	str	r2, [r3, #0]

        /* Get Start Tick */
        tickstart = HAL_GetTick();
 8001422:	f7ff fa29 	bl	8000878 <HAL_GetTick>
 8001426:	0003      	movs	r3, r0
 8001428:	617b      	str	r3, [r7, #20]

        /* Wait till PLL is ready */
        while(__HAL_RCC_GET_FLAG(RCC_FLAG_PLLRDY)  == 0U)
 800142a:	e008      	b.n	800143e <HAL_RCC_OscConfig+0x706>
        {
          if((HAL_GetTick() - tickstart ) > PLL_TIMEOUT_VALUE)
 800142c:	f7ff fa24 	bl	8000878 <HAL_GetTick>
 8001430:	0002      	movs	r2, r0
 8001432:	697b      	ldr	r3, [r7, #20]
 8001434:	1ad3      	subs	r3, r2, r3
 8001436:	2b02      	cmp	r3, #2
 8001438:	d901      	bls.n	800143e <HAL_RCC_OscConfig+0x706>
          {
            return HAL_TIMEOUT;
 800143a:	2303      	movs	r3, #3
 800143c:	e045      	b.n	80014ca <HAL_RCC_OscConfig+0x792>
        while(__HAL_RCC_GET_FLAG(RCC_FLAG_PLLRDY)  == 0U)
 800143e:	4b25      	ldr	r3, [pc, #148]	; (80014d4 <HAL_RCC_OscConfig+0x79c>)
 8001440:	681a      	ldr	r2, [r3, #0]
 8001442:	2380      	movs	r3, #128	; 0x80
 8001444:	049b      	lsls	r3, r3, #18
 8001446:	4013      	ands	r3, r2
 8001448:	d0f0      	beq.n	800142c <HAL_RCC_OscConfig+0x6f4>
 800144a:	e03d      	b.n	80014c8 <HAL_RCC_OscConfig+0x790>
        }
      }
      else
      {
        /* Disable the main PLL. */
        __HAL_RCC_PLL_DISABLE();
 800144c:	4b21      	ldr	r3, [pc, #132]	; (80014d4 <HAL_RCC_OscConfig+0x79c>)
 800144e:	681a      	ldr	r2, [r3, #0]
 8001450:	4b20      	ldr	r3, [pc, #128]	; (80014d4 <HAL_RCC_OscConfig+0x79c>)
 8001452:	4922      	ldr	r1, [pc, #136]	; (80014dc <HAL_RCC_OscConfig+0x7a4>)
 8001454:	400a      	ands	r2, r1
 8001456:	601a      	str	r2, [r3, #0]

        /* Get Start Tick */
        tickstart = HAL_GetTick();
 8001458:	f7ff fa0e 	bl	8000878 <HAL_GetTick>
 800145c:	0003      	movs	r3, r0
 800145e:	617b      	str	r3, [r7, #20]

        /* Wait till PLL is disabled */
        while(__HAL_RCC_GET_FLAG(RCC_FLAG_PLLRDY)  != 0U)
 8001460:	e008      	b.n	8001474 <HAL_RCC_OscConfig+0x73c>
        {
          if((HAL_GetTick() - tickstart ) > PLL_TIMEOUT_VALUE)
 8001462:	f7ff fa09 	bl	8000878 <HAL_GetTick>
 8001466:	0002      	movs	r2, r0
 8001468:	697b      	ldr	r3, [r7, #20]
 800146a:	1ad3      	subs	r3, r2, r3
 800146c:	2b02      	cmp	r3, #2
 800146e:	d901      	bls.n	8001474 <HAL_RCC_OscConfig+0x73c>
          {
            return HAL_TIMEOUT;
 8001470:	2303      	movs	r3, #3
 8001472:	e02a      	b.n	80014ca <HAL_RCC_OscConfig+0x792>
        while(__HAL_RCC_GET_FLAG(RCC_FLAG_PLLRDY)  != 0U)
 8001474:	4b17      	ldr	r3, [pc, #92]	; (80014d4 <HAL_RCC_OscConfig+0x79c>)
 8001476:	681a      	ldr	r2, [r3, #0]
 8001478:	2380      	movs	r3, #128	; 0x80
 800147a:	049b      	lsls	r3, r3, #18
 800147c:	4013      	ands	r3, r2
 800147e:	d1f0      	bne.n	8001462 <HAL_RCC_OscConfig+0x72a>
 8001480:	e022      	b.n	80014c8 <HAL_RCC_OscConfig+0x790>
      }
    }
    else
    {
      /* Check if there is a request to disable the PLL used as System clock source */
      if((RCC_OscInitStruct->PLL.PLLState) == RCC_PLL_OFF)
 8001482:	687b      	ldr	r3, [r7, #4]
 8001484:	6a9b      	ldr	r3, [r3, #40]	; 0x28
 8001486:	2b01      	cmp	r3, #1
 8001488:	d101      	bne.n	800148e <HAL_RCC_OscConfig+0x756>
      {
        return HAL_ERROR;
 800148a:	2301      	movs	r3, #1
 800148c:	e01d      	b.n	80014ca <HAL_RCC_OscConfig+0x792>
      }
      else
      {
        /* Do not return HAL_ERROR if request repeats the current configuration */
        pll_config = RCC->CFGR;
 800148e:	4b11      	ldr	r3, [pc, #68]	; (80014d4 <HAL_RCC_OscConfig+0x79c>)
 8001490:	68db      	ldr	r3, [r3, #12]
 8001492:	61bb      	str	r3, [r7, #24]
        if((READ_BIT(pll_config, RCC_CFGR_PLLSRC) != RCC_OscInitStruct->PLL.PLLSource) ||
 8001494:	69ba      	ldr	r2, [r7, #24]
 8001496:	2380      	movs	r3, #128	; 0x80
 8001498:	025b      	lsls	r3, r3, #9
 800149a:	401a      	ands	r2, r3
 800149c:	687b      	ldr	r3, [r7, #4]
 800149e:	6adb      	ldr	r3, [r3, #44]	; 0x2c
 80014a0:	429a      	cmp	r2, r3
 80014a2:	d10f      	bne.n	80014c4 <HAL_RCC_OscConfig+0x78c>
           (READ_BIT(pll_config, RCC_CFGR_PLLMUL) != RCC_OscInitStruct->PLL.PLLMUL) ||
 80014a4:	69ba      	ldr	r2, [r7, #24]
 80014a6:	23f0      	movs	r3, #240	; 0xf0
 80014a8:	039b      	lsls	r3, r3, #14
 80014aa:	401a      	ands	r2, r3
 80014ac:	687b      	ldr	r3, [r7, #4]
 80014ae:	6b1b      	ldr	r3, [r3, #48]	; 0x30
        if((READ_BIT(pll_config, RCC_CFGR_PLLSRC) != RCC_OscInitStruct->PLL.PLLSource) ||
 80014b0:	429a      	cmp	r2, r3
 80014b2:	d107      	bne.n	80014c4 <HAL_RCC_OscConfig+0x78c>
           (READ_BIT(pll_config, RCC_CFGR_PLLDIV) != RCC_OscInitStruct->PLL.PLLDIV))
 80014b4:	69ba      	ldr	r2, [r7, #24]
 80014b6:	23c0      	movs	r3, #192	; 0xc0
 80014b8:	041b      	lsls	r3, r3, #16
 80014ba:	401a      	ands	r2, r3
 80014bc:	687b      	ldr	r3, [r7, #4]
 80014be:	6b5b      	ldr	r3, [r3, #52]	; 0x34
           (READ_BIT(pll_config, RCC_CFGR_PLLMUL) != RCC_OscInitStruct->PLL.PLLMUL) ||
 80014c0:	429a      	cmp	r2, r3
 80014c2:	d001      	beq.n	80014c8 <HAL_RCC_OscConfig+0x790>
        {
          return HAL_ERROR;
 80014c4:	2301      	movs	r3, #1
 80014c6:	e000      	b.n	80014ca <HAL_RCC_OscConfig+0x792>
        }
      }
    }
  }
  return HAL_OK;
 80014c8:	2300      	movs	r3, #0
}
 80014ca:	0018      	movs	r0, r3
 80014cc:	46bd      	mov	sp, r7
 80014ce:	b00a      	add	sp, #40	; 0x28
 80014d0:	bdb0      	pop	{r4, r5, r7, pc}
 80014d2:	46c0      	nop			; (mov r8, r8)
 80014d4:	40021000 	.word	0x40021000
 80014d8:	ff02ffff 	.word	0xff02ffff
 80014dc:	feffffff 	.word	0xfeffffff

080014e0 <HAL_RCC_ClockConfig>:
  *         HPRE[3:0] bits to ensure that HCLK not exceed the maximum allowed frequency
  *         (for more details refer to section above "Initialization/de-initialization functions")
  * @retval HAL status
  */
HAL_StatusTypeDef HAL_RCC_ClockConfig(RCC_ClkInitTypeDef  *RCC_ClkInitStruct, uint32_t FLatency)
{
 80014e0:	b5b0      	push	{r4, r5, r7, lr}
 80014e2:	b084      	sub	sp, #16
 80014e4:	af00      	add	r7, sp, #0
 80014e6:	6078      	str	r0, [r7, #4]
 80014e8:	6039      	str	r1, [r7, #0]
  uint32_t tickstart;
  HAL_StatusTypeDef status;

  /* Check Null pointer */
  if(RCC_ClkInitStruct == NULL)
 80014ea:	687b      	ldr	r3, [r7, #4]
 80014ec:	2b00      	cmp	r3, #0
 80014ee:	d101      	bne.n	80014f4 <HAL_RCC_ClockConfig+0x14>
  {
    return HAL_ERROR;
 80014f0:	2301      	movs	r3, #1
 80014f2:	e128      	b.n	8001746 <HAL_RCC_ClockConfig+0x266>
  /* To correctly read data from FLASH memory, the number of wait states (LATENCY)
  must be correctly programmed according to the frequency of the CPU clock
  (HCLK) and the supply voltage of the device. */

  /* Increasing the number of wait states because of higher CPU frequency */
  if(FLatency > __HAL_FLASH_GET_LATENCY())
 80014f4:	4b96      	ldr	r3, [pc, #600]	; (8001750 <HAL_RCC_ClockConfig+0x270>)
 80014f6:	681b      	ldr	r3, [r3, #0]
 80014f8:	2201      	movs	r2, #1
 80014fa:	4013      	ands	r3, r2
 80014fc:	683a      	ldr	r2, [r7, #0]
 80014fe:	429a      	cmp	r2, r3
 8001500:	d91e      	bls.n	8001540 <HAL_RCC_ClockConfig+0x60>
  {
    /* Program the new number of wait states to the LATENCY bits in the FLASH_ACR register */
    __HAL_FLASH_SET_LATENCY(FLatency);
 8001502:	4b93      	ldr	r3, [pc, #588]	; (8001750 <HAL_RCC_ClockConfig+0x270>)
 8001504:	681b      	ldr	r3, [r3, #0]
 8001506:	2201      	movs	r2, #1
 8001508:	4393      	bics	r3, r2
 800150a:	0019      	movs	r1, r3
 800150c:	4b90      	ldr	r3, [pc, #576]	; (8001750 <HAL_RCC_ClockConfig+0x270>)
 800150e:	683a      	ldr	r2, [r7, #0]
 8001510:	430a      	orrs	r2, r1
 8001512:	601a      	str	r2, [r3, #0]

    /* Check that the new number of wait states is taken into account to access the Flash
    memory by polling the FLASH_ACR register */
    tickstart = HAL_GetTick();
 8001514:	f7ff f9b0 	bl	8000878 <HAL_GetTick>
 8001518:	0003      	movs	r3, r0
 800151a:	60fb      	str	r3, [r7, #12]

    while (__HAL_FLASH_GET_LATENCY() != FLatency)
 800151c:	e009      	b.n	8001532 <HAL_RCC_ClockConfig+0x52>
    {
      if ((HAL_GetTick() - tickstart) > CLOCKSWITCH_TIMEOUT_VALUE)
 800151e:	f7ff f9ab 	bl	8000878 <HAL_GetTick>
 8001522:	0002      	movs	r2, r0
 8001524:	68fb      	ldr	r3, [r7, #12]
 8001526:	1ad3      	subs	r3, r2, r3
 8001528:	4a8a      	ldr	r2, [pc, #552]	; (8001754 <HAL_RCC_ClockConfig+0x274>)
 800152a:	4293      	cmp	r3, r2
 800152c:	d901      	bls.n	8001532 <HAL_RCC_ClockConfig+0x52>
      {
        return HAL_TIMEOUT;
 800152e:	2303      	movs	r3, #3
 8001530:	e109      	b.n	8001746 <HAL_RCC_ClockConfig+0x266>
    while (__HAL_FLASH_GET_LATENCY() != FLatency)
 8001532:	4b87      	ldr	r3, [pc, #540]	; (8001750 <HAL_RCC_ClockConfig+0x270>)
 8001534:	681b      	ldr	r3, [r3, #0]
 8001536:	2201      	movs	r2, #1
 8001538:	4013      	ands	r3, r2
 800153a:	683a      	ldr	r2, [r7, #0]
 800153c:	429a      	cmp	r2, r3
 800153e:	d1ee      	bne.n	800151e <HAL_RCC_ClockConfig+0x3e>
      }
    }
  }

  /*-------------------------- HCLK Configuration --------------------------*/
  if(((RCC_ClkInitStruct->ClockType) & RCC_CLOCKTYPE_HCLK) == RCC_CLOCKTYPE_HCLK)
 8001540:	687b      	ldr	r3, [r7, #4]
 8001542:	681b      	ldr	r3, [r3, #0]
 8001544:	2202      	movs	r2, #2
 8001546:	4013      	ands	r3, r2
 8001548:	d009      	beq.n	800155e <HAL_RCC_ClockConfig+0x7e>
  {
    assert_param(IS_RCC_HCLK(RCC_ClkInitStruct->AHBCLKDivider));
    MODIFY_REG(RCC->CFGR, RCC_CFGR_HPRE, RCC_ClkInitStruct->AHBCLKDivider);
 800154a:	4b83      	ldr	r3, [pc, #524]	; (8001758 <HAL_RCC_ClockConfig+0x278>)
 800154c:	68db      	ldr	r3, [r3, #12]
 800154e:	22f0      	movs	r2, #240	; 0xf0
 8001550:	4393      	bics	r3, r2
 8001552:	0019      	movs	r1, r3
 8001554:	687b      	ldr	r3, [r7, #4]
 8001556:	689a      	ldr	r2, [r3, #8]
 8001558:	4b7f      	ldr	r3, [pc, #508]	; (8001758 <HAL_RCC_ClockConfig+0x278>)
 800155a:	430a      	orrs	r2, r1
 800155c:	60da      	str	r2, [r3, #12]
  }

  /*------------------------- SYSCLK Configuration ---------------------------*/
  if(((RCC_ClkInitStruct->ClockType) & RCC_CLOCKTYPE_SYSCLK) == RCC_CLOCKTYPE_SYSCLK)
 800155e:	687b      	ldr	r3, [r7, #4]
 8001560:	681b      	ldr	r3, [r3, #0]
 8001562:	2201      	movs	r2, #1
 8001564:	4013      	ands	r3, r2
 8001566:	d100      	bne.n	800156a <HAL_RCC_ClockConfig+0x8a>
 8001568:	e089      	b.n	800167e <HAL_RCC_ClockConfig+0x19e>
  {
    assert_param(IS_RCC_SYSCLKSOURCE(RCC_ClkInitStruct->SYSCLKSource));

    /* HSE is selected as System Clock Source */
    if(RCC_ClkInitStruct->SYSCLKSource == RCC_SYSCLKSOURCE_HSE)
 800156a:	687b      	ldr	r3, [r7, #4]
 800156c:	685b      	ldr	r3, [r3, #4]
 800156e:	2b02      	cmp	r3, #2
 8001570:	d107      	bne.n	8001582 <HAL_RCC_ClockConfig+0xa2>
    {
      /* Check the HSE ready flag */
      if(__HAL_RCC_GET_FLAG(RCC_FLAG_HSERDY) == 0U)
 8001572:	4b79      	ldr	r3, [pc, #484]	; (8001758 <HAL_RCC_ClockConfig+0x278>)
 8001574:	681a      	ldr	r2, [r3, #0]
 8001576:	2380      	movs	r3, #128	; 0x80
 8001578:	029b      	lsls	r3, r3, #10
 800157a:	4013      	ands	r3, r2
 800157c:	d120      	bne.n	80015c0 <HAL_RCC_ClockConfig+0xe0>
      {
        return HAL_ERROR;
 800157e:	2301      	movs	r3, #1
 8001580:	e0e1      	b.n	8001746 <HAL_RCC_ClockConfig+0x266>
      }
    }
    /* PLL is selected as System Clock Source */
    else if(RCC_ClkInitStruct->SYSCLKSource == RCC_SYSCLKSOURCE_PLLCLK)
 8001582:	687b      	ldr	r3, [r7, #4]
 8001584:	685b      	ldr	r3, [r3, #4]
 8001586:	2b03      	cmp	r3, #3
 8001588:	d107      	bne.n	800159a <HAL_RCC_ClockConfig+0xba>
    {
      /* Check the PLL ready flag */
      if(__HAL_RCC_GET_FLAG(RCC_FLAG_PLLRDY) == 0U)
 800158a:	4b73      	ldr	r3, [pc, #460]	; (8001758 <HAL_RCC_ClockConfig+0x278>)
 800158c:	681a      	ldr	r2, [r3, #0]
 800158e:	2380      	movs	r3, #128	; 0x80
 8001590:	049b      	lsls	r3, r3, #18
 8001592:	4013      	ands	r3, r2
 8001594:	d114      	bne.n	80015c0 <HAL_RCC_ClockConfig+0xe0>
      {
        return HAL_ERROR;
 8001596:	2301      	movs	r3, #1
 8001598:	e0d5      	b.n	8001746 <HAL_RCC_ClockConfig+0x266>
      }
    }
    /* HSI is selected as System Clock Source */
    else if(RCC_ClkInitStruct->SYSCLKSource == RCC_SYSCLKSOURCE_HSI)
 800159a:	687b      	ldr	r3, [r7, #4]
 800159c:	685b      	ldr	r3, [r3, #4]
 800159e:	2b01      	cmp	r3, #1
 80015a0:	d106      	bne.n	80015b0 <HAL_RCC_ClockConfig+0xd0>
    {
      /* Check the HSI ready flag */
      if(__HAL_RCC_GET_FLAG(RCC_FLAG_HSIRDY) == 0U)
 80015a2:	4b6d      	ldr	r3, [pc, #436]	; (8001758 <HAL_RCC_ClockConfig+0x278>)
 80015a4:	681b      	ldr	r3, [r3, #0]
 80015a6:	2204      	movs	r2, #4
 80015a8:	4013      	ands	r3, r2
 80015aa:	d109      	bne.n	80015c0 <HAL_RCC_ClockConfig+0xe0>
      {
        return HAL_ERROR;
 80015ac:	2301      	movs	r3, #1
 80015ae:	e0ca      	b.n	8001746 <HAL_RCC_ClockConfig+0x266>
    }
    /* MSI is selected as System Clock Source */
    else
    {
      /* Check the MSI ready flag */
      if(__HAL_RCC_GET_FLAG(RCC_FLAG_MSIRDY) == 0U)
 80015b0:	4b69      	ldr	r3, [pc, #420]	; (8001758 <HAL_RCC_ClockConfig+0x278>)
 80015b2:	681a      	ldr	r2, [r3, #0]
 80015b4:	2380      	movs	r3, #128	; 0x80
 80015b6:	009b      	lsls	r3, r3, #2
 80015b8:	4013      	ands	r3, r2
 80015ba:	d101      	bne.n	80015c0 <HAL_RCC_ClockConfig+0xe0>
      {
        return HAL_ERROR;
 80015bc:	2301      	movs	r3, #1
 80015be:	e0c2      	b.n	8001746 <HAL_RCC_ClockConfig+0x266>
      }
    }
    __HAL_RCC_SYSCLK_CONFIG(RCC_ClkInitStruct->SYSCLKSource);
 80015c0:	4b65      	ldr	r3, [pc, #404]	; (8001758 <HAL_RCC_ClockConfig+0x278>)
 80015c2:	68db      	ldr	r3, [r3, #12]
 80015c4:	2203      	movs	r2, #3
 80015c6:	4393      	bics	r3, r2
 80015c8:	0019      	movs	r1, r3
 80015ca:	687b      	ldr	r3, [r7, #4]
 80015cc:	685a      	ldr	r2, [r3, #4]
 80015ce:	4b62      	ldr	r3, [pc, #392]	; (8001758 <HAL_RCC_ClockConfig+0x278>)
 80015d0:	430a      	orrs	r2, r1
 80015d2:	60da      	str	r2, [r3, #12]

    /* Get Start Tick */
    tickstart = HAL_GetTick();
 80015d4:	f7ff f950 	bl	8000878 <HAL_GetTick>
 80015d8:	0003      	movs	r3, r0
 80015da:	60fb      	str	r3, [r7, #12]

    if(RCC_ClkInitStruct->SYSCLKSource == RCC_SYSCLKSOURCE_HSE)
 80015dc:	687b      	ldr	r3, [r7, #4]
 80015de:	685b      	ldr	r3, [r3, #4]
 80015e0:	2b02      	cmp	r3, #2
 80015e2:	d111      	bne.n	8001608 <HAL_RCC_ClockConfig+0x128>
    {
      while (__HAL_RCC_GET_SYSCLK_SOURCE() != RCC_SYSCLKSOURCE_STATUS_HSE)
 80015e4:	e009      	b.n	80015fa <HAL_RCC_ClockConfig+0x11a>
      {
        if((HAL_GetTick() - tickstart ) > CLOCKSWITCH_TIMEOUT_VALUE)
 80015e6:	f7ff f947 	bl	8000878 <HAL_GetTick>
 80015ea:	0002      	movs	r2, r0
 80015ec:	68fb      	ldr	r3, [r7, #12]
 80015ee:	1ad3      	subs	r3, r2, r3
 80015f0:	4a58      	ldr	r2, [pc, #352]	; (8001754 <HAL_RCC_ClockConfig+0x274>)
 80015f2:	4293      	cmp	r3, r2
 80015f4:	d901      	bls.n	80015fa <HAL_RCC_ClockConfig+0x11a>
        {
          return HAL_TIMEOUT;
 80015f6:	2303      	movs	r3, #3
 80015f8:	e0a5      	b.n	8001746 <HAL_RCC_ClockConfig+0x266>
      while (__HAL_RCC_GET_SYSCLK_SOURCE() != RCC_SYSCLKSOURCE_STATUS_HSE)
 80015fa:	4b57      	ldr	r3, [pc, #348]	; (8001758 <HAL_RCC_ClockConfig+0x278>)
 80015fc:	68db      	ldr	r3, [r3, #12]
 80015fe:	220c      	movs	r2, #12
 8001600:	4013      	ands	r3, r2
 8001602:	2b08      	cmp	r3, #8
 8001604:	d1ef      	bne.n	80015e6 <HAL_RCC_ClockConfig+0x106>
 8001606:	e03a      	b.n	800167e <HAL_RCC_ClockConfig+0x19e>
        }
      }
    }
    else if(RCC_ClkInitStruct->SYSCLKSource == RCC_SYSCLKSOURCE_PLLCLK)
 8001608:	687b      	ldr	r3, [r7, #4]
 800160a:	685b      	ldr	r3, [r3, #4]
 800160c:	2b03      	cmp	r3, #3
 800160e:	d111      	bne.n	8001634 <HAL_RCC_ClockConfig+0x154>
    {
      while (__HAL_RCC_GET_SYSCLK_SOURCE() != RCC_SYSCLKSOURCE_STATUS_PLLCLK)
 8001610:	e009      	b.n	8001626 <HAL_RCC_ClockConfig+0x146>
      {
        if((HAL_GetTick() - tickstart ) > CLOCKSWITCH_TIMEOUT_VALUE)
 8001612:	f7ff f931 	bl	8000878 <HAL_GetTick>
 8001616:	0002      	movs	r2, r0
 8001618:	68fb      	ldr	r3, [r7, #12]
 800161a:	1ad3      	subs	r3, r2, r3
 800161c:	4a4d      	ldr	r2, [pc, #308]	; (8001754 <HAL_RCC_ClockConfig+0x274>)
 800161e:	4293      	cmp	r3, r2
 8001620:	d901      	bls.n	8001626 <HAL_RCC_ClockConfig+0x146>
        {
          return HAL_TIMEOUT;
 8001622:	2303      	movs	r3, #3
 8001624:	e08f      	b.n	8001746 <HAL_RCC_ClockConfig+0x266>
      while (__HAL_RCC_GET_SYSCLK_SOURCE() != RCC_SYSCLKSOURCE_STATUS_PLLCLK)
 8001626:	4b4c      	ldr	r3, [pc, #304]	; (8001758 <HAL_RCC_ClockConfig+0x278>)
 8001628:	68db      	ldr	r3, [r3, #12]
 800162a:	220c      	movs	r2, #12
 800162c:	4013      	ands	r3, r2
 800162e:	2b0c      	cmp	r3, #12
 8001630:	d1ef      	bne.n	8001612 <HAL_RCC_ClockConfig+0x132>
 8001632:	e024      	b.n	800167e <HAL_RCC_ClockConfig+0x19e>
        }
      }
    }
    else if(RCC_ClkInitStruct->SYSCLKSource == RCC_SYSCLKSOURCE_HSI)
 8001634:	687b      	ldr	r3, [r7, #4]
 8001636:	685b      	ldr	r3, [r3, #4]
 8001638:	2b01      	cmp	r3, #1
 800163a:	d11b      	bne.n	8001674 <HAL_RCC_ClockConfig+0x194>
    {
      while (__HAL_RCC_GET_SYSCLK_SOURCE() != RCC_SYSCLKSOURCE_STATUS_HSI)
 800163c:	e009      	b.n	8001652 <HAL_RCC_ClockConfig+0x172>
      {
        if((HAL_GetTick() - tickstart ) > CLOCKSWITCH_TIMEOUT_VALUE)
 800163e:	f7ff f91b 	bl	8000878 <HAL_GetTick>
 8001642:	0002      	movs	r2, r0
 8001644:	68fb      	ldr	r3, [r7, #12]
 8001646:	1ad3      	subs	r3, r2, r3
 8001648:	4a42      	ldr	r2, [pc, #264]	; (8001754 <HAL_RCC_ClockConfig+0x274>)
 800164a:	4293      	cmp	r3, r2
 800164c:	d901      	bls.n	8001652 <HAL_RCC_ClockConfig+0x172>
        {
          return HAL_TIMEOUT;
 800164e:	2303      	movs	r3, #3
 8001650:	e079      	b.n	8001746 <HAL_RCC_ClockConfig+0x266>
      while (__HAL_RCC_GET_SYSCLK_SOURCE() != RCC_SYSCLKSOURCE_STATUS_HSI)
 8001652:	4b41      	ldr	r3, [pc, #260]	; (8001758 <HAL_RCC_ClockConfig+0x278>)
 8001654:	68db      	ldr	r3, [r3, #12]
 8001656:	220c      	movs	r2, #12
 8001658:	4013      	ands	r3, r2
 800165a:	2b04      	cmp	r3, #4
 800165c:	d1ef      	bne.n	800163e <HAL_RCC_ClockConfig+0x15e>
 800165e:	e00e      	b.n	800167e <HAL_RCC_ClockConfig+0x19e>
    }
    else
    {
      while(__HAL_RCC_GET_SYSCLK_SOURCE() != RCC_SYSCLKSOURCE_STATUS_MSI)
      {
        if((HAL_GetTick() - tickstart ) > CLOCKSWITCH_TIMEOUT_VALUE)
 8001660:	f7ff f90a 	bl	8000878 <HAL_GetTick>
 8001664:	0002      	movs	r2, r0
 8001666:	68fb      	ldr	r3, [r7, #12]
 8001668:	1ad3      	subs	r3, r2, r3
 800166a:	4a3a      	ldr	r2, [pc, #232]	; (8001754 <HAL_RCC_ClockConfig+0x274>)
 800166c:	4293      	cmp	r3, r2
 800166e:	d901      	bls.n	8001674 <HAL_RCC_ClockConfig+0x194>
        {
          return HAL_TIMEOUT;
 8001670:	2303      	movs	r3, #3
 8001672:	e068      	b.n	8001746 <HAL_RCC_ClockConfig+0x266>
      while(__HAL_RCC_GET_SYSCLK_SOURCE() != RCC_SYSCLKSOURCE_STATUS_MSI)
 8001674:	4b38      	ldr	r3, [pc, #224]	; (8001758 <HAL_RCC_ClockConfig+0x278>)
 8001676:	68db      	ldr	r3, [r3, #12]
 8001678:	220c      	movs	r2, #12
 800167a:	4013      	ands	r3, r2
 800167c:	d1f0      	bne.n	8001660 <HAL_RCC_ClockConfig+0x180>
        }
      }
    }
  }
  /* Decreasing the number of wait states because of lower CPU frequency */
  if(FLatency < __HAL_FLASH_GET_LATENCY())
 800167e:	4b34      	ldr	r3, [pc, #208]	; (8001750 <HAL_RCC_ClockConfig+0x270>)
 8001680:	681b      	ldr	r3, [r3, #0]
 8001682:	2201      	movs	r2, #1
 8001684:	4013      	ands	r3, r2
 8001686:	683a      	ldr	r2, [r7, #0]
 8001688:	429a      	cmp	r2, r3
 800168a:	d21e      	bcs.n	80016ca <HAL_RCC_ClockConfig+0x1ea>
  {
    /* Program the new number of wait states to the LATENCY bits in the FLASH_ACR register */
    __HAL_FLASH_SET_LATENCY(FLatency);
 800168c:	4b30      	ldr	r3, [pc, #192]	; (8001750 <HAL_RCC_ClockConfig+0x270>)
 800168e:	681b      	ldr	r3, [r3, #0]
 8001690:	2201      	movs	r2, #1
 8001692:	4393      	bics	r3, r2
 8001694:	0019      	movs	r1, r3
 8001696:	4b2e      	ldr	r3, [pc, #184]	; (8001750 <HAL_RCC_ClockConfig+0x270>)
 8001698:	683a      	ldr	r2, [r7, #0]
 800169a:	430a      	orrs	r2, r1
 800169c:	601a      	str	r2, [r3, #0]

    /* Check that the new number of wait states is taken into account to access the Flash
    memory by polling the FLASH_ACR register */
    tickstart = HAL_GetTick();
 800169e:	f7ff f8eb 	bl	8000878 <HAL_GetTick>
 80016a2:	0003      	movs	r3, r0
 80016a4:	60fb      	str	r3, [r7, #12]

    while (__HAL_FLASH_GET_LATENCY() != FLatency)
 80016a6:	e009      	b.n	80016bc <HAL_RCC_ClockConfig+0x1dc>
    {
      if ((HAL_GetTick() - tickstart) > CLOCKSWITCH_TIMEOUT_VALUE)
 80016a8:	f7ff f8e6 	bl	8000878 <HAL_GetTick>
 80016ac:	0002      	movs	r2, r0
 80016ae:	68fb      	ldr	r3, [r7, #12]
 80016b0:	1ad3      	subs	r3, r2, r3
 80016b2:	4a28      	ldr	r2, [pc, #160]	; (8001754 <HAL_RCC_ClockConfig+0x274>)
 80016b4:	4293      	cmp	r3, r2
 80016b6:	d901      	bls.n	80016bc <HAL_RCC_ClockConfig+0x1dc>
      {
        return HAL_TIMEOUT;
 80016b8:	2303      	movs	r3, #3
 80016ba:	e044      	b.n	8001746 <HAL_RCC_ClockConfig+0x266>
    while (__HAL_FLASH_GET_LATENCY() != FLatency)
 80016bc:	4b24      	ldr	r3, [pc, #144]	; (8001750 <HAL_RCC_ClockConfig+0x270>)
 80016be:	681b      	ldr	r3, [r3, #0]
 80016c0:	2201      	movs	r2, #1
 80016c2:	4013      	ands	r3, r2
 80016c4:	683a      	ldr	r2, [r7, #0]
 80016c6:	429a      	cmp	r2, r3
 80016c8:	d1ee      	bne.n	80016a8 <HAL_RCC_ClockConfig+0x1c8>
      }
    }
  }

  /*-------------------------- PCLK1 Configuration ---------------------------*/
  if(((RCC_ClkInitStruct->ClockType) & RCC_CLOCKTYPE_PCLK1) == RCC_CLOCKTYPE_PCLK1)
 80016ca:	687b      	ldr	r3, [r7, #4]
 80016cc:	681b      	ldr	r3, [r3, #0]
 80016ce:	2204      	movs	r2, #4
 80016d0:	4013      	ands	r3, r2
 80016d2:	d009      	beq.n	80016e8 <HAL_RCC_ClockConfig+0x208>
  {
    assert_param(IS_RCC_PCLK(RCC_ClkInitStruct->APB1CLKDivider));
    MODIFY_REG(RCC->CFGR, RCC_CFGR_PPRE1, RCC_ClkInitStruct->APB1CLKDivider);
 80016d4:	4b20      	ldr	r3, [pc, #128]	; (8001758 <HAL_RCC_ClockConfig+0x278>)
 80016d6:	68db      	ldr	r3, [r3, #12]
 80016d8:	4a20      	ldr	r2, [pc, #128]	; (800175c <HAL_RCC_ClockConfig+0x27c>)
 80016da:	4013      	ands	r3, r2
 80016dc:	0019      	movs	r1, r3
 80016de:	687b      	ldr	r3, [r7, #4]
 80016e0:	68da      	ldr	r2, [r3, #12]
 80016e2:	4b1d      	ldr	r3, [pc, #116]	; (8001758 <HAL_RCC_ClockConfig+0x278>)
 80016e4:	430a      	orrs	r2, r1
 80016e6:	60da      	str	r2, [r3, #12]
  }

  /*-------------------------- PCLK2 Configuration ---------------------------*/
  if(((RCC_ClkInitStruct->ClockType) & RCC_CLOCKTYPE_PCLK2) == RCC_CLOCKTYPE_PCLK2)
 80016e8:	687b      	ldr	r3, [r7, #4]
 80016ea:	681b      	ldr	r3, [r3, #0]
 80016ec:	2208      	movs	r2, #8
 80016ee:	4013      	ands	r3, r2
 80016f0:	d00a      	beq.n	8001708 <HAL_RCC_ClockConfig+0x228>
  {
    assert_param(IS_RCC_PCLK(RCC_ClkInitStruct->APB2CLKDivider));
    MODIFY_REG(RCC->CFGR, RCC_CFGR_PPRE2, ((RCC_ClkInitStruct->APB2CLKDivider) << 3));
 80016f2:	4b19      	ldr	r3, [pc, #100]	; (8001758 <HAL_RCC_ClockConfig+0x278>)
 80016f4:	68db      	ldr	r3, [r3, #12]
 80016f6:	4a1a      	ldr	r2, [pc, #104]	; (8001760 <HAL_RCC_ClockConfig+0x280>)
 80016f8:	4013      	ands	r3, r2
 80016fa:	0019      	movs	r1, r3
 80016fc:	687b      	ldr	r3, [r7, #4]
 80016fe:	691b      	ldr	r3, [r3, #16]
 8001700:	00da      	lsls	r2, r3, #3
 8001702:	4b15      	ldr	r3, [pc, #84]	; (8001758 <HAL_RCC_ClockConfig+0x278>)
 8001704:	430a      	orrs	r2, r1
 8001706:	60da      	str	r2, [r3, #12]
  }

  /* Update the SystemCoreClock global variable */
  SystemCoreClock = HAL_RCC_GetSysClockFreq() >> AHBPrescTable[(RCC->CFGR & RCC_CFGR_HPRE)>> RCC_CFGR_HPRE_Pos];
 8001708:	f000 f832 	bl	8001770 <HAL_RCC_GetSysClockFreq>
 800170c:	0001      	movs	r1, r0
 800170e:	4b12      	ldr	r3, [pc, #72]	; (8001758 <HAL_RCC_ClockConfig+0x278>)
 8001710:	68db      	ldr	r3, [r3, #12]
 8001712:	091b      	lsrs	r3, r3, #4
 8001714:	220f      	movs	r2, #15
 8001716:	4013      	ands	r3, r2
 8001718:	4a12      	ldr	r2, [pc, #72]	; (8001764 <HAL_RCC_ClockConfig+0x284>)
 800171a:	5cd3      	ldrb	r3, [r2, r3]
 800171c:	000a      	movs	r2, r1
 800171e:	40da      	lsrs	r2, r3
 8001720:	4b11      	ldr	r3, [pc, #68]	; (8001768 <HAL_RCC_ClockConfig+0x288>)
 8001722:	601a      	str	r2, [r3, #0]

  /* Configure the source of time base considering new system clocks settings*/
  status = HAL_InitTick(uwTickPrio);
 8001724:	4b11      	ldr	r3, [pc, #68]	; (800176c <HAL_RCC_ClockConfig+0x28c>)
 8001726:	681b      	ldr	r3, [r3, #0]
 8001728:	250b      	movs	r5, #11
 800172a:	197c      	adds	r4, r7, r5
 800172c:	0018      	movs	r0, r3
 800172e:	f7ff f85d 	bl	80007ec <HAL_InitTick>
 8001732:	0003      	movs	r3, r0
 8001734:	7023      	strb	r3, [r4, #0]
  if(status != HAL_OK)
 8001736:	197b      	adds	r3, r7, r5
 8001738:	781b      	ldrb	r3, [r3, #0]
 800173a:	2b00      	cmp	r3, #0
 800173c:	d002      	beq.n	8001744 <HAL_RCC_ClockConfig+0x264>
  {
    return status;
 800173e:	197b      	adds	r3, r7, r5
 8001740:	781b      	ldrb	r3, [r3, #0]
 8001742:	e000      	b.n	8001746 <HAL_RCC_ClockConfig+0x266>
  }

  return HAL_OK;
 8001744:	2300      	movs	r3, #0
}
 8001746:	0018      	movs	r0, r3
 8001748:	46bd      	mov	sp, r7
 800174a:	b004      	add	sp, #16
 800174c:	bdb0      	pop	{r4, r5, r7, pc}
 800174e:	46c0      	nop			; (mov r8, r8)
 8001750:	40022000 	.word	0x40022000
 8001754:	00001388 	.word	0x00001388
 8001758:	40021000 	.word	0x40021000
 800175c:	fffff8ff 	.word	0xfffff8ff
 8001760:	ffffc7ff 	.word	0xffffc7ff
 8001764:	080027dc 	.word	0x080027dc
 8001768:	20000000 	.word	0x20000000
 800176c:	20000004 	.word	0x20000004

08001770 <HAL_RCC_GetSysClockFreq>:
  *         right SYSCLK value. Otherwise, any configuration based on this function will be incorrect.
  *
  * @retval SYSCLK frequency
  */
uint32_t HAL_RCC_GetSysClockFreq(void)
{
 8001770:	b5b0      	push	{r4, r5, r7, lr}
 8001772:	b08e      	sub	sp, #56	; 0x38
 8001774:	af00      	add	r7, sp, #0
  uint32_t tmpreg, pllm, plld, pllvco, msiclkrange;    /* no init needed */
  uint32_t sysclockfreq;

  tmpreg = RCC->CFGR;
 8001776:	4b4c      	ldr	r3, [pc, #304]	; (80018a8 <HAL_RCC_GetSysClockFreq+0x138>)
 8001778:	68db      	ldr	r3, [r3, #12]
 800177a:	62fb      	str	r3, [r7, #44]	; 0x2c

  /* Get SYSCLK source -------------------------------------------------------*/
  switch (tmpreg & RCC_CFGR_SWS)
 800177c:	6afa      	ldr	r2, [r7, #44]	; 0x2c
 800177e:	230c      	movs	r3, #12
 8001780:	4013      	ands	r3, r2
 8001782:	2b0c      	cmp	r3, #12
 8001784:	d014      	beq.n	80017b0 <HAL_RCC_GetSysClockFreq+0x40>
 8001786:	d900      	bls.n	800178a <HAL_RCC_GetSysClockFreq+0x1a>
 8001788:	e07b      	b.n	8001882 <HAL_RCC_GetSysClockFreq+0x112>
 800178a:	2b04      	cmp	r3, #4
 800178c:	d002      	beq.n	8001794 <HAL_RCC_GetSysClockFreq+0x24>
 800178e:	2b08      	cmp	r3, #8
 8001790:	d00b      	beq.n	80017aa <HAL_RCC_GetSysClockFreq+0x3a>
 8001792:	e076      	b.n	8001882 <HAL_RCC_GetSysClockFreq+0x112>
  {
    case RCC_SYSCLKSOURCE_STATUS_HSI:  /* HSI used as system clock source */
    {
      if ((RCC->CR & RCC_CR_HSIDIVF) != 0U)
 8001794:	4b44      	ldr	r3, [pc, #272]	; (80018a8 <HAL_RCC_GetSysClockFreq+0x138>)
 8001796:	681b      	ldr	r3, [r3, #0]
 8001798:	2210      	movs	r2, #16
 800179a:	4013      	ands	r3, r2
 800179c:	d002      	beq.n	80017a4 <HAL_RCC_GetSysClockFreq+0x34>
      {
        sysclockfreq =  (HSI_VALUE >> 2);
 800179e:	4b43      	ldr	r3, [pc, #268]	; (80018ac <HAL_RCC_GetSysClockFreq+0x13c>)
 80017a0:	633b      	str	r3, [r7, #48]	; 0x30
      }
      else
      {
        sysclockfreq =  HSI_VALUE;
      }
      break;
 80017a2:	e07c      	b.n	800189e <HAL_RCC_GetSysClockFreq+0x12e>
        sysclockfreq =  HSI_VALUE;
 80017a4:	4b42      	ldr	r3, [pc, #264]	; (80018b0 <HAL_RCC_GetSysClockFreq+0x140>)
 80017a6:	633b      	str	r3, [r7, #48]	; 0x30
      break;
 80017a8:	e079      	b.n	800189e <HAL_RCC_GetSysClockFreq+0x12e>
    }
    case RCC_SYSCLKSOURCE_STATUS_HSE:  /* HSE used as system clock */
    {
      sysclockfreq = HSE_VALUE;
 80017aa:	4b42      	ldr	r3, [pc, #264]	; (80018b4 <HAL_RCC_GetSysClockFreq+0x144>)
 80017ac:	633b      	str	r3, [r7, #48]	; 0x30
      break;
 80017ae:	e076      	b.n	800189e <HAL_RCC_GetSysClockFreq+0x12e>
    }
    case RCC_SYSCLKSOURCE_STATUS_PLLCLK:  /* PLL used as system clock */
    {
      pllm = PLLMulTable[(uint32_t)(tmpreg & RCC_CFGR_PLLMUL) >> RCC_CFGR_PLLMUL_Pos];
 80017b0:	6afb      	ldr	r3, [r7, #44]	; 0x2c
 80017b2:	0c9a      	lsrs	r2, r3, #18
 80017b4:	230f      	movs	r3, #15
 80017b6:	401a      	ands	r2, r3
 80017b8:	4b3f      	ldr	r3, [pc, #252]	; (80018b8 <HAL_RCC_GetSysClockFreq+0x148>)
 80017ba:	5c9b      	ldrb	r3, [r3, r2]
 80017bc:	62bb      	str	r3, [r7, #40]	; 0x28
      plld = ((uint32_t)(tmpreg & RCC_CFGR_PLLDIV) >> RCC_CFGR_PLLDIV_Pos) + 1U;
 80017be:	6afb      	ldr	r3, [r7, #44]	; 0x2c
 80017c0:	0d9a      	lsrs	r2, r3, #22
 80017c2:	2303      	movs	r3, #3
 80017c4:	4013      	ands	r3, r2
 80017c6:	3301      	adds	r3, #1
 80017c8:	627b      	str	r3, [r7, #36]	; 0x24
      if (__HAL_RCC_GET_PLL_OSCSOURCE() != RCC_PLLSOURCE_HSI)
 80017ca:	4b37      	ldr	r3, [pc, #220]	; (80018a8 <HAL_RCC_GetSysClockFreq+0x138>)
 80017cc:	68da      	ldr	r2, [r3, #12]
 80017ce:	2380      	movs	r3, #128	; 0x80
 80017d0:	025b      	lsls	r3, r3, #9
 80017d2:	4013      	ands	r3, r2
 80017d4:	d01a      	beq.n	800180c <HAL_RCC_GetSysClockFreq+0x9c>
      {
        /* HSE used as PLL clock source */
        pllvco = (uint32_t)(((uint64_t)HSE_VALUE * (uint64_t)pllm) / (uint64_t)plld);
 80017d6:	6abb      	ldr	r3, [r7, #40]	; 0x28
 80017d8:	61bb      	str	r3, [r7, #24]
 80017da:	2300      	movs	r3, #0
 80017dc:	61fb      	str	r3, [r7, #28]
 80017de:	4a35      	ldr	r2, [pc, #212]	; (80018b4 <HAL_RCC_GetSysClockFreq+0x144>)
 80017e0:	2300      	movs	r3, #0
 80017e2:	69b8      	ldr	r0, [r7, #24]
 80017e4:	69f9      	ldr	r1, [r7, #28]
 80017e6:	f7fe fd3b 	bl	8000260 <__aeabi_lmul>
 80017ea:	0002      	movs	r2, r0
 80017ec:	000b      	movs	r3, r1
 80017ee:	0010      	movs	r0, r2
 80017f0:	0019      	movs	r1, r3
 80017f2:	6a7b      	ldr	r3, [r7, #36]	; 0x24
 80017f4:	613b      	str	r3, [r7, #16]
 80017f6:	2300      	movs	r3, #0
 80017f8:	617b      	str	r3, [r7, #20]
 80017fa:	693a      	ldr	r2, [r7, #16]
 80017fc:	697b      	ldr	r3, [r7, #20]
 80017fe:	f7fe fd0f 	bl	8000220 <__aeabi_uldivmod>
 8001802:	0002      	movs	r2, r0
 8001804:	000b      	movs	r3, r1
 8001806:	0013      	movs	r3, r2
 8001808:	637b      	str	r3, [r7, #52]	; 0x34
 800180a:	e037      	b.n	800187c <HAL_RCC_GetSysClockFreq+0x10c>
      }
      else
      {
        if ((RCC->CR & RCC_CR_HSIDIVF) != 0U)
 800180c:	4b26      	ldr	r3, [pc, #152]	; (80018a8 <HAL_RCC_GetSysClockFreq+0x138>)
 800180e:	681b      	ldr	r3, [r3, #0]
 8001810:	2210      	movs	r2, #16
 8001812:	4013      	ands	r3, r2
 8001814:	d01a      	beq.n	800184c <HAL_RCC_GetSysClockFreq+0xdc>
        {
          pllvco = (uint32_t)((((uint64_t)(HSI_VALUE >> 2)) * (uint64_t)pllm) / (uint64_t)plld);
 8001816:	6abb      	ldr	r3, [r7, #40]	; 0x28
 8001818:	60bb      	str	r3, [r7, #8]
 800181a:	2300      	movs	r3, #0
 800181c:	60fb      	str	r3, [r7, #12]
 800181e:	4a23      	ldr	r2, [pc, #140]	; (80018ac <HAL_RCC_GetSysClockFreq+0x13c>)
 8001820:	2300      	movs	r3, #0
 8001822:	68b8      	ldr	r0, [r7, #8]
 8001824:	68f9      	ldr	r1, [r7, #12]
 8001826:	f7fe fd1b 	bl	8000260 <__aeabi_lmul>
 800182a:	0002      	movs	r2, r0
 800182c:	000b      	movs	r3, r1
 800182e:	0010      	movs	r0, r2
 8001830:	0019      	movs	r1, r3
 8001832:	6a7b      	ldr	r3, [r7, #36]	; 0x24
 8001834:	603b      	str	r3, [r7, #0]
 8001836:	2300      	movs	r3, #0
 8001838:	607b      	str	r3, [r7, #4]
 800183a:	683a      	ldr	r2, [r7, #0]
 800183c:	687b      	ldr	r3, [r7, #4]
 800183e:	f7fe fcef 	bl	8000220 <__aeabi_uldivmod>
 8001842:	0002      	movs	r2, r0
 8001844:	000b      	movs	r3, r1
 8001846:	0013      	movs	r3, r2
 8001848:	637b      	str	r3, [r7, #52]	; 0x34
 800184a:	e017      	b.n	800187c <HAL_RCC_GetSysClockFreq+0x10c>
        }
        else
        {
         pllvco = (uint32_t)(((uint64_t)HSI_VALUE * (uint64_t)pllm) / (uint64_t)plld);
 800184c:	6abb      	ldr	r3, [r7, #40]	; 0x28
 800184e:	0018      	movs	r0, r3
 8001850:	2300      	movs	r3, #0
 8001852:	0019      	movs	r1, r3
 8001854:	4a16      	ldr	r2, [pc, #88]	; (80018b0 <HAL_RCC_GetSysClockFreq+0x140>)
 8001856:	2300      	movs	r3, #0
 8001858:	f7fe fd02 	bl	8000260 <__aeabi_lmul>
 800185c:	0002      	movs	r2, r0
 800185e:	000b      	movs	r3, r1
 8001860:	0010      	movs	r0, r2
 8001862:	0019      	movs	r1, r3
 8001864:	6a7b      	ldr	r3, [r7, #36]	; 0x24
 8001866:	001c      	movs	r4, r3
 8001868:	2300      	movs	r3, #0
 800186a:	001d      	movs	r5, r3
 800186c:	0022      	movs	r2, r4
 800186e:	002b      	movs	r3, r5
 8001870:	f7fe fcd6 	bl	8000220 <__aeabi_uldivmod>
 8001874:	0002      	movs	r2, r0
 8001876:	000b      	movs	r3, r1
 8001878:	0013      	movs	r3, r2
 800187a:	637b      	str	r3, [r7, #52]	; 0x34
        }
      }
      sysclockfreq = pllvco;
 800187c:	6b7b      	ldr	r3, [r7, #52]	; 0x34
 800187e:	633b      	str	r3, [r7, #48]	; 0x30
      break;
 8001880:	e00d      	b.n	800189e <HAL_RCC_GetSysClockFreq+0x12e>
    }
    case RCC_SYSCLKSOURCE_STATUS_MSI:  /* MSI used as system clock source */
    default: /* MSI used as system clock */
    {
      msiclkrange = (RCC->ICSCR & RCC_ICSCR_MSIRANGE ) >> RCC_ICSCR_MSIRANGE_Pos;
 8001882:	4b09      	ldr	r3, [pc, #36]	; (80018a8 <HAL_RCC_GetSysClockFreq+0x138>)
 8001884:	685b      	ldr	r3, [r3, #4]
 8001886:	0b5b      	lsrs	r3, r3, #13
 8001888:	2207      	movs	r2, #7
 800188a:	4013      	ands	r3, r2
 800188c:	623b      	str	r3, [r7, #32]
      sysclockfreq = (32768U * (1UL << (msiclkrange + 1U)));
 800188e:	6a3b      	ldr	r3, [r7, #32]
 8001890:	3301      	adds	r3, #1
 8001892:	2280      	movs	r2, #128	; 0x80
 8001894:	0212      	lsls	r2, r2, #8
 8001896:	409a      	lsls	r2, r3
 8001898:	0013      	movs	r3, r2
 800189a:	633b      	str	r3, [r7, #48]	; 0x30
      break;
 800189c:	46c0      	nop			; (mov r8, r8)
    }
  }
  return sysclockfreq;
 800189e:	6b3b      	ldr	r3, [r7, #48]	; 0x30
}
 80018a0:	0018      	movs	r0, r3
 80018a2:	46bd      	mov	sp, r7
 80018a4:	b00e      	add	sp, #56	; 0x38
 80018a6:	bdb0      	pop	{r4, r5, r7, pc}
 80018a8:	40021000 	.word	0x40021000
 80018ac:	003d0900 	.word	0x003d0900
 80018b0:	00f42400 	.word	0x00f42400
 80018b4:	007a1200 	.word	0x007a1200
 80018b8:	080027f4 	.word	0x080027f4

080018bc <HAL_RCC_GetHCLKFreq>:
  * @note   The SystemCoreClock CMSIS variable is used to store System Clock Frequency
  *         and updated within this function
  * @retval HCLK frequency
  */
uint32_t HAL_RCC_GetHCLKFreq(void)
{
 80018bc:	b580      	push	{r7, lr}
 80018be:	af00      	add	r7, sp, #0
  return SystemCoreClock;
 80018c0:	4b02      	ldr	r3, [pc, #8]	; (80018cc <HAL_RCC_GetHCLKFreq+0x10>)
 80018c2:	681b      	ldr	r3, [r3, #0]
}
 80018c4:	0018      	movs	r0, r3
 80018c6:	46bd      	mov	sp, r7
 80018c8:	bd80      	pop	{r7, pc}
 80018ca:	46c0      	nop			; (mov r8, r8)
 80018cc:	20000000 	.word	0x20000000

080018d0 <HAL_RCC_GetPCLK1Freq>:
  * @note   Each time PCLK1 changes, this function must be called to update the
  *         right PCLK1 value. Otherwise, any configuration based on this function will be incorrect.
  * @retval PCLK1 frequency
  */
uint32_t HAL_RCC_GetPCLK1Freq(void)
{
 80018d0:	b580      	push	{r7, lr}
 80018d2:	af00      	add	r7, sp, #0
  /* Get HCLK source and Compute PCLK1 frequency ---------------------------*/
  return (HAL_RCC_GetHCLKFreq() >> APBPrescTable[(RCC->CFGR & RCC_CFGR_PPRE1) >> RCC_CFGR_PPRE1_Pos]);
 80018d4:	f7ff fff2 	bl	80018bc <HAL_RCC_GetHCLKFreq>
 80018d8:	0001      	movs	r1, r0
 80018da:	4b06      	ldr	r3, [pc, #24]	; (80018f4 <HAL_RCC_GetPCLK1Freq+0x24>)
 80018dc:	68db      	ldr	r3, [r3, #12]
 80018de:	0a1b      	lsrs	r3, r3, #8
 80018e0:	2207      	movs	r2, #7
 80018e2:	4013      	ands	r3, r2
 80018e4:	4a04      	ldr	r2, [pc, #16]	; (80018f8 <HAL_RCC_GetPCLK1Freq+0x28>)
 80018e6:	5cd3      	ldrb	r3, [r2, r3]
 80018e8:	40d9      	lsrs	r1, r3
 80018ea:	000b      	movs	r3, r1
}
 80018ec:	0018      	movs	r0, r3
 80018ee:	46bd      	mov	sp, r7
 80018f0:	bd80      	pop	{r7, pc}
 80018f2:	46c0      	nop			; (mov r8, r8)
 80018f4:	40021000 	.word	0x40021000
 80018f8:	080027ec 	.word	0x080027ec

080018fc <HAL_RCC_GetPCLK2Freq>:
  * @note   Each time PCLK2 changes, this function must be called to update the
  *         right PCLK2 value. Otherwise, any configuration based on this function will be incorrect.
  * @retval PCLK2 frequency
  */
uint32_t HAL_RCC_GetPCLK2Freq(void)
{
 80018fc:	b580      	push	{r7, lr}
 80018fe:	af00      	add	r7, sp, #0
  /* Get HCLK source and Compute PCLK2 frequency ---------------------------*/
  return (HAL_RCC_GetHCLKFreq()>> APBPrescTable[(RCC->CFGR & RCC_CFGR_PPRE2) >> RCC_CFGR_PPRE2_Pos]);
 8001900:	f7ff ffdc 	bl	80018bc <HAL_RCC_GetHCLKFreq>
 8001904:	0001      	movs	r1, r0
 8001906:	4b06      	ldr	r3, [pc, #24]	; (8001920 <HAL_RCC_GetPCLK2Freq+0x24>)
 8001908:	68db      	ldr	r3, [r3, #12]
 800190a:	0adb      	lsrs	r3, r3, #11
 800190c:	2207      	movs	r2, #7
 800190e:	4013      	ands	r3, r2
 8001910:	4a04      	ldr	r2, [pc, #16]	; (8001924 <HAL_RCC_GetPCLK2Freq+0x28>)
 8001912:	5cd3      	ldrb	r3, [r2, r3]
 8001914:	40d9      	lsrs	r1, r3
 8001916:	000b      	movs	r3, r1
}
 8001918:	0018      	movs	r0, r3
 800191a:	46bd      	mov	sp, r7
 800191c:	bd80      	pop	{r7, pc}
 800191e:	46c0      	nop			; (mov r8, r8)
 8001920:	40021000 	.word	0x40021000
 8001924:	080027ec 	.word	0x080027ec

08001928 <HAL_RCCEx_PeriphCLKConfig>:
  * @retval HAL status
  * @note   If HAL_ERROR returned, first switch-OFF HSE clock oscillator with @ref HAL_RCC_OscConfig()
  *         to possibly update HSE divider.
  */
HAL_StatusTypeDef HAL_RCCEx_PeriphCLKConfig(RCC_PeriphCLKInitTypeDef  *PeriphClkInit)
{
 8001928:	b580      	push	{r7, lr}
 800192a:	b086      	sub	sp, #24
 800192c:	af00      	add	r7, sp, #0
 800192e:	6078      	str	r0, [r7, #4]
  uint32_t tickstart;
  uint32_t temp_reg;
  FlagStatus       pwrclkchanged = RESET;
 8001930:	2017      	movs	r0, #23
 8001932:	183b      	adds	r3, r7, r0
 8001934:	2200      	movs	r2, #0
 8001936:	701a      	strb	r2, [r3, #0]

  /* Check the parameters */
  assert_param(IS_RCC_PERIPHCLOCK(PeriphClkInit->PeriphClockSelection));

  /*------------------------------- RTC/LCD Configuration ------------------------*/
  if ((((PeriphClkInit->PeriphClockSelection) & RCC_PERIPHCLK_RTC) == RCC_PERIPHCLK_RTC)
 8001938:	687b      	ldr	r3, [r7, #4]
 800193a:	681b      	ldr	r3, [r3, #0]
 800193c:	2220      	movs	r2, #32
 800193e:	4013      	ands	r3, r2
 8001940:	d100      	bne.n	8001944 <HAL_RCCEx_PeriphCLKConfig+0x1c>
 8001942:	e0c7      	b.n	8001ad4 <HAL_RCCEx_PeriphCLKConfig+0x1ac>
#endif /* LCD */

    /* As soon as function is called to change RTC clock source, activation of the
       power domain is done. */
    /* Requires to enable write access to Backup Domain of necessary */
    if(__HAL_RCC_PWR_IS_CLK_DISABLED())
 8001944:	4b9b      	ldr	r3, [pc, #620]	; (8001bb4 <HAL_RCCEx_PeriphCLKConfig+0x28c>)
 8001946:	6b9a      	ldr	r2, [r3, #56]	; 0x38
 8001948:	2380      	movs	r3, #128	; 0x80
 800194a:	055b      	lsls	r3, r3, #21
 800194c:	4013      	ands	r3, r2
 800194e:	d109      	bne.n	8001964 <HAL_RCCEx_PeriphCLKConfig+0x3c>
    {
      __HAL_RCC_PWR_CLK_ENABLE();
 8001950:	4b98      	ldr	r3, [pc, #608]	; (8001bb4 <HAL_RCCEx_PeriphCLKConfig+0x28c>)
 8001952:	6b9a      	ldr	r2, [r3, #56]	; 0x38
 8001954:	4b97      	ldr	r3, [pc, #604]	; (8001bb4 <HAL_RCCEx_PeriphCLKConfig+0x28c>)
 8001956:	2180      	movs	r1, #128	; 0x80
 8001958:	0549      	lsls	r1, r1, #21
 800195a:	430a      	orrs	r2, r1
 800195c:	639a      	str	r2, [r3, #56]	; 0x38
      pwrclkchanged = SET;
 800195e:	183b      	adds	r3, r7, r0
 8001960:	2201      	movs	r2, #1
 8001962:	701a      	strb	r2, [r3, #0]
    }

    if(HAL_IS_BIT_CLR(PWR->CR, PWR_CR_DBP))
 8001964:	4b94      	ldr	r3, [pc, #592]	; (8001bb8 <HAL_RCCEx_PeriphCLKConfig+0x290>)
 8001966:	681a      	ldr	r2, [r3, #0]
 8001968:	2380      	movs	r3, #128	; 0x80
 800196a:	005b      	lsls	r3, r3, #1
 800196c:	4013      	ands	r3, r2
 800196e:	d11a      	bne.n	80019a6 <HAL_RCCEx_PeriphCLKConfig+0x7e>
    {
      /* Enable write access to Backup domain */
      SET_BIT(PWR->CR, PWR_CR_DBP);
 8001970:	4b91      	ldr	r3, [pc, #580]	; (8001bb8 <HAL_RCCEx_PeriphCLKConfig+0x290>)
 8001972:	681a      	ldr	r2, [r3, #0]
 8001974:	4b90      	ldr	r3, [pc, #576]	; (8001bb8 <HAL_RCCEx_PeriphCLKConfig+0x290>)
 8001976:	2180      	movs	r1, #128	; 0x80
 8001978:	0049      	lsls	r1, r1, #1
 800197a:	430a      	orrs	r2, r1
 800197c:	601a      	str	r2, [r3, #0]

      /* Wait for Backup domain Write protection disable */
      tickstart = HAL_GetTick();
 800197e:	f7fe ff7b 	bl	8000878 <HAL_GetTick>
 8001982:	0003      	movs	r3, r0
 8001984:	613b      	str	r3, [r7, #16]

      while(HAL_IS_BIT_CLR(PWR->CR, PWR_CR_DBP))
 8001986:	e008      	b.n	800199a <HAL_RCCEx_PeriphCLKConfig+0x72>
      {
        if((HAL_GetTick() - tickstart) > RCC_DBP_TIMEOUT_VALUE)
 8001988:	f7fe ff76 	bl	8000878 <HAL_GetTick>
 800198c:	0002      	movs	r2, r0
 800198e:	693b      	ldr	r3, [r7, #16]
 8001990:	1ad3      	subs	r3, r2, r3
 8001992:	2b64      	cmp	r3, #100	; 0x64
 8001994:	d901      	bls.n	800199a <HAL_RCCEx_PeriphCLKConfig+0x72>
        {
          return HAL_TIMEOUT;
 8001996:	2303      	movs	r3, #3
 8001998:	e107      	b.n	8001baa <HAL_RCCEx_PeriphCLKConfig+0x282>
      while(HAL_IS_BIT_CLR(PWR->CR, PWR_CR_DBP))
 800199a:	4b87      	ldr	r3, [pc, #540]	; (8001bb8 <HAL_RCCEx_PeriphCLKConfig+0x290>)
 800199c:	681a      	ldr	r2, [r3, #0]
 800199e:	2380      	movs	r3, #128	; 0x80
 80019a0:	005b      	lsls	r3, r3, #1
 80019a2:	4013      	ands	r3, r2
 80019a4:	d0f0      	beq.n	8001988 <HAL_RCCEx_PeriphCLKConfig+0x60>
        }
      }
    }

    /* Check if user wants to change HSE RTC prescaler whereas HSE is enabled */
    temp_reg = (RCC->CR & RCC_CR_RTCPRE);
 80019a6:	4b83      	ldr	r3, [pc, #524]	; (8001bb4 <HAL_RCCEx_PeriphCLKConfig+0x28c>)
 80019a8:	681a      	ldr	r2, [r3, #0]
 80019aa:	23c0      	movs	r3, #192	; 0xc0
 80019ac:	039b      	lsls	r3, r3, #14
 80019ae:	4013      	ands	r3, r2
 80019b0:	60fb      	str	r3, [r7, #12]
    if ((temp_reg != (PeriphClkInit->RTCClockSelection & RCC_CR_RTCPRE))
 80019b2:	687b      	ldr	r3, [r7, #4]
 80019b4:	685a      	ldr	r2, [r3, #4]
 80019b6:	23c0      	movs	r3, #192	; 0xc0
 80019b8:	039b      	lsls	r3, r3, #14
 80019ba:	4013      	ands	r3, r2
 80019bc:	68fa      	ldr	r2, [r7, #12]
 80019be:	429a      	cmp	r2, r3
 80019c0:	d013      	beq.n	80019ea <HAL_RCCEx_PeriphCLKConfig+0xc2>
#if defined (LCD)
     || (temp_reg != (PeriphClkInit->LCDClockSelection & RCC_CR_RTCPRE))
#endif /* LCD */
       )
    { /* Check HSE State */
      if ((PeriphClkInit->RTCClockSelection & RCC_CSR_RTCSEL) == RCC_CSR_RTCSEL_HSE)
 80019c2:	687b      	ldr	r3, [r7, #4]
 80019c4:	685a      	ldr	r2, [r3, #4]
 80019c6:	23c0      	movs	r3, #192	; 0xc0
 80019c8:	029b      	lsls	r3, r3, #10
 80019ca:	401a      	ands	r2, r3
 80019cc:	23c0      	movs	r3, #192	; 0xc0
 80019ce:	029b      	lsls	r3, r3, #10
 80019d0:	429a      	cmp	r2, r3
 80019d2:	d10a      	bne.n	80019ea <HAL_RCCEx_PeriphCLKConfig+0xc2>
      {
        if (HAL_IS_BIT_SET(RCC->CR, RCC_CR_HSERDY))
 80019d4:	4b77      	ldr	r3, [pc, #476]	; (8001bb4 <HAL_RCCEx_PeriphCLKConfig+0x28c>)
 80019d6:	681a      	ldr	r2, [r3, #0]
 80019d8:	2380      	movs	r3, #128	; 0x80
 80019da:	029b      	lsls	r3, r3, #10
 80019dc:	401a      	ands	r2, r3
 80019de:	2380      	movs	r3, #128	; 0x80
 80019e0:	029b      	lsls	r3, r3, #10
 80019e2:	429a      	cmp	r2, r3
 80019e4:	d101      	bne.n	80019ea <HAL_RCCEx_PeriphCLKConfig+0xc2>
        {
          /* To update HSE divider, first switch-OFF HSE clock oscillator*/
          return HAL_ERROR;
 80019e6:	2301      	movs	r3, #1
 80019e8:	e0df      	b.n	8001baa <HAL_RCCEx_PeriphCLKConfig+0x282>
        }
      }
    }

    /* Reset the Backup domain only if the RTC Clock source selection is modified from reset value */
    temp_reg = (RCC->CSR & RCC_CSR_RTCSEL);
 80019ea:	4b72      	ldr	r3, [pc, #456]	; (8001bb4 <HAL_RCCEx_PeriphCLKConfig+0x28c>)
 80019ec:	6d1a      	ldr	r2, [r3, #80]	; 0x50
 80019ee:	23c0      	movs	r3, #192	; 0xc0
 80019f0:	029b      	lsls	r3, r3, #10
 80019f2:	4013      	ands	r3, r2
 80019f4:	60fb      	str	r3, [r7, #12]

    if((temp_reg != 0x00000000U) && (((temp_reg != (PeriphClkInit->RTCClockSelection & RCC_CSR_RTCSEL)) \
 80019f6:	68fb      	ldr	r3, [r7, #12]
 80019f8:	2b00      	cmp	r3, #0
 80019fa:	d03b      	beq.n	8001a74 <HAL_RCCEx_PeriphCLKConfig+0x14c>
 80019fc:	687b      	ldr	r3, [r7, #4]
 80019fe:	685a      	ldr	r2, [r3, #4]
 8001a00:	23c0      	movs	r3, #192	; 0xc0
 8001a02:	029b      	lsls	r3, r3, #10
 8001a04:	4013      	ands	r3, r2
 8001a06:	68fa      	ldr	r2, [r7, #12]
 8001a08:	429a      	cmp	r2, r3
 8001a0a:	d033      	beq.n	8001a74 <HAL_RCCEx_PeriphCLKConfig+0x14c>
      && (((PeriphClkInit->PeriphClockSelection) & RCC_PERIPHCLK_RTC) == RCC_PERIPHCLK_RTC))
 8001a0c:	687b      	ldr	r3, [r7, #4]
 8001a0e:	681b      	ldr	r3, [r3, #0]
 8001a10:	2220      	movs	r2, #32
 8001a12:	4013      	ands	r3, r2
 8001a14:	d02e      	beq.n	8001a74 <HAL_RCCEx_PeriphCLKConfig+0x14c>
       && (((PeriphClkInit->PeriphClockSelection) & RCC_PERIPHCLK_LCD) == RCC_PERIPHCLK_LCD))
#endif /* LCD */
     ))
    {
      /* Store the content of CSR register before the reset of Backup Domain */
      temp_reg = (RCC->CSR & ~(RCC_CSR_RTCSEL));
 8001a16:	4b67      	ldr	r3, [pc, #412]	; (8001bb4 <HAL_RCCEx_PeriphCLKConfig+0x28c>)
 8001a18:	6d1b      	ldr	r3, [r3, #80]	; 0x50
 8001a1a:	4a68      	ldr	r2, [pc, #416]	; (8001bbc <HAL_RCCEx_PeriphCLKConfig+0x294>)
 8001a1c:	4013      	ands	r3, r2
 8001a1e:	60fb      	str	r3, [r7, #12]

      /* RTC Clock selection can be changed only if the Backup Domain is reset */
      __HAL_RCC_BACKUPRESET_FORCE();
 8001a20:	4b64      	ldr	r3, [pc, #400]	; (8001bb4 <HAL_RCCEx_PeriphCLKConfig+0x28c>)
 8001a22:	6d1a      	ldr	r2, [r3, #80]	; 0x50
 8001a24:	4b63      	ldr	r3, [pc, #396]	; (8001bb4 <HAL_RCCEx_PeriphCLKConfig+0x28c>)
 8001a26:	2180      	movs	r1, #128	; 0x80
 8001a28:	0309      	lsls	r1, r1, #12
 8001a2a:	430a      	orrs	r2, r1
 8001a2c:	651a      	str	r2, [r3, #80]	; 0x50
      __HAL_RCC_BACKUPRESET_RELEASE();
 8001a2e:	4b61      	ldr	r3, [pc, #388]	; (8001bb4 <HAL_RCCEx_PeriphCLKConfig+0x28c>)
 8001a30:	6d1a      	ldr	r2, [r3, #80]	; 0x50
 8001a32:	4b60      	ldr	r3, [pc, #384]	; (8001bb4 <HAL_RCCEx_PeriphCLKConfig+0x28c>)
 8001a34:	4962      	ldr	r1, [pc, #392]	; (8001bc0 <HAL_RCCEx_PeriphCLKConfig+0x298>)
 8001a36:	400a      	ands	r2, r1
 8001a38:	651a      	str	r2, [r3, #80]	; 0x50

      /* Restore the Content of CSR register */
      RCC->CSR = temp_reg;
 8001a3a:	4b5e      	ldr	r3, [pc, #376]	; (8001bb4 <HAL_RCCEx_PeriphCLKConfig+0x28c>)
 8001a3c:	68fa      	ldr	r2, [r7, #12]
 8001a3e:	651a      	str	r2, [r3, #80]	; 0x50

       /* Wait for LSERDY if LSE was enabled */
      if (HAL_IS_BIT_SET(temp_reg, RCC_CSR_LSEON))
 8001a40:	68fa      	ldr	r2, [r7, #12]
 8001a42:	2380      	movs	r3, #128	; 0x80
 8001a44:	005b      	lsls	r3, r3, #1
 8001a46:	4013      	ands	r3, r2
 8001a48:	d014      	beq.n	8001a74 <HAL_RCCEx_PeriphCLKConfig+0x14c>
      {
        /* Get Start Tick */
        tickstart = HAL_GetTick();
 8001a4a:	f7fe ff15 	bl	8000878 <HAL_GetTick>
 8001a4e:	0003      	movs	r3, r0
 8001a50:	613b      	str	r3, [r7, #16]

        /* Wait till LSE is ready */
        while(__HAL_RCC_GET_FLAG(RCC_FLAG_LSERDY) == 0U)
 8001a52:	e009      	b.n	8001a68 <HAL_RCCEx_PeriphCLKConfig+0x140>
        {
          if((HAL_GetTick() - tickstart ) > RCC_LSE_TIMEOUT_VALUE)
 8001a54:	f7fe ff10 	bl	8000878 <HAL_GetTick>
 8001a58:	0002      	movs	r2, r0
 8001a5a:	693b      	ldr	r3, [r7, #16]
 8001a5c:	1ad3      	subs	r3, r2, r3
 8001a5e:	4a59      	ldr	r2, [pc, #356]	; (8001bc4 <HAL_RCCEx_PeriphCLKConfig+0x29c>)
 8001a60:	4293      	cmp	r3, r2
 8001a62:	d901      	bls.n	8001a68 <HAL_RCCEx_PeriphCLKConfig+0x140>
          {
            return HAL_TIMEOUT;
 8001a64:	2303      	movs	r3, #3
 8001a66:	e0a0      	b.n	8001baa <HAL_RCCEx_PeriphCLKConfig+0x282>
        while(__HAL_RCC_GET_FLAG(RCC_FLAG_LSERDY) == 0U)
 8001a68:	4b52      	ldr	r3, [pc, #328]	; (8001bb4 <HAL_RCCEx_PeriphCLKConfig+0x28c>)
 8001a6a:	6d1a      	ldr	r2, [r3, #80]	; 0x50
 8001a6c:	2380      	movs	r3, #128	; 0x80
 8001a6e:	009b      	lsls	r3, r3, #2
 8001a70:	4013      	ands	r3, r2
 8001a72:	d0ef      	beq.n	8001a54 <HAL_RCCEx_PeriphCLKConfig+0x12c>
    {
      __HAL_RCC_LCD_CONFIG(PeriphClkInit->LCDClockSelection);
    } 
#endif /* LCD */

    if(((PeriphClkInit->PeriphClockSelection) & RCC_PERIPHCLK_RTC) == RCC_PERIPHCLK_RTC)
 8001a74:	687b      	ldr	r3, [r7, #4]
 8001a76:	681b      	ldr	r3, [r3, #0]
 8001a78:	2220      	movs	r2, #32
 8001a7a:	4013      	ands	r3, r2
 8001a7c:	d01f      	beq.n	8001abe <HAL_RCCEx_PeriphCLKConfig+0x196>
    {
      __HAL_RCC_RTC_CONFIG(PeriphClkInit->RTCClockSelection);
 8001a7e:	687b      	ldr	r3, [r7, #4]
 8001a80:	685a      	ldr	r2, [r3, #4]
 8001a82:	23c0      	movs	r3, #192	; 0xc0
 8001a84:	029b      	lsls	r3, r3, #10
 8001a86:	401a      	ands	r2, r3
 8001a88:	23c0      	movs	r3, #192	; 0xc0
 8001a8a:	029b      	lsls	r3, r3, #10
 8001a8c:	429a      	cmp	r2, r3
 8001a8e:	d10c      	bne.n	8001aaa <HAL_RCCEx_PeriphCLKConfig+0x182>
 8001a90:	4b48      	ldr	r3, [pc, #288]	; (8001bb4 <HAL_RCCEx_PeriphCLKConfig+0x28c>)
 8001a92:	681b      	ldr	r3, [r3, #0]
 8001a94:	4a4c      	ldr	r2, [pc, #304]	; (8001bc8 <HAL_RCCEx_PeriphCLKConfig+0x2a0>)
 8001a96:	4013      	ands	r3, r2
 8001a98:	0019      	movs	r1, r3
 8001a9a:	687b      	ldr	r3, [r7, #4]
 8001a9c:	685a      	ldr	r2, [r3, #4]
 8001a9e:	23c0      	movs	r3, #192	; 0xc0
 8001aa0:	039b      	lsls	r3, r3, #14
 8001aa2:	401a      	ands	r2, r3
 8001aa4:	4b43      	ldr	r3, [pc, #268]	; (8001bb4 <HAL_RCCEx_PeriphCLKConfig+0x28c>)
 8001aa6:	430a      	orrs	r2, r1
 8001aa8:	601a      	str	r2, [r3, #0]
 8001aaa:	4b42      	ldr	r3, [pc, #264]	; (8001bb4 <HAL_RCCEx_PeriphCLKConfig+0x28c>)
 8001aac:	6d19      	ldr	r1, [r3, #80]	; 0x50
 8001aae:	687b      	ldr	r3, [r7, #4]
 8001ab0:	685a      	ldr	r2, [r3, #4]
 8001ab2:	23c0      	movs	r3, #192	; 0xc0
 8001ab4:	029b      	lsls	r3, r3, #10
 8001ab6:	401a      	ands	r2, r3
 8001ab8:	4b3e      	ldr	r3, [pc, #248]	; (8001bb4 <HAL_RCCEx_PeriphCLKConfig+0x28c>)
 8001aba:	430a      	orrs	r2, r1
 8001abc:	651a      	str	r2, [r3, #80]	; 0x50
    }

    /* Require to disable power clock if necessary */
    if(pwrclkchanged == SET)
 8001abe:	2317      	movs	r3, #23
 8001ac0:	18fb      	adds	r3, r7, r3
 8001ac2:	781b      	ldrb	r3, [r3, #0]
 8001ac4:	2b01      	cmp	r3, #1
 8001ac6:	d105      	bne.n	8001ad4 <HAL_RCCEx_PeriphCLKConfig+0x1ac>
    {
      __HAL_RCC_PWR_CLK_DISABLE();
 8001ac8:	4b3a      	ldr	r3, [pc, #232]	; (8001bb4 <HAL_RCCEx_PeriphCLKConfig+0x28c>)
 8001aca:	6b9a      	ldr	r2, [r3, #56]	; 0x38
 8001acc:	4b39      	ldr	r3, [pc, #228]	; (8001bb4 <HAL_RCCEx_PeriphCLKConfig+0x28c>)
 8001ace:	493f      	ldr	r1, [pc, #252]	; (8001bcc <HAL_RCCEx_PeriphCLKConfig+0x2a4>)
 8001ad0:	400a      	ands	r2, r1
 8001ad2:	639a      	str	r2, [r3, #56]	; 0x38
    }
  }

#if defined (RCC_CCIPR_USART1SEL)
  /*------------------------------- USART1 Configuration ------------------------*/
  if(((PeriphClkInit->PeriphClockSelection) & RCC_PERIPHCLK_USART1) == RCC_PERIPHCLK_USART1)
 8001ad4:	687b      	ldr	r3, [r7, #4]
 8001ad6:	681b      	ldr	r3, [r3, #0]
 8001ad8:	2201      	movs	r2, #1
 8001ada:	4013      	ands	r3, r2
 8001adc:	d009      	beq.n	8001af2 <HAL_RCCEx_PeriphCLKConfig+0x1ca>
  {
    /* Check the parameters */
    assert_param(IS_RCC_USART1CLKSOURCE(PeriphClkInit->Usart1ClockSelection));

    /* Configure the USART1 clock source */
    __HAL_RCC_USART1_CONFIG(PeriphClkInit->Usart1ClockSelection);
 8001ade:	4b35      	ldr	r3, [pc, #212]	; (8001bb4 <HAL_RCCEx_PeriphCLKConfig+0x28c>)
 8001ae0:	6cdb      	ldr	r3, [r3, #76]	; 0x4c
 8001ae2:	2203      	movs	r2, #3
 8001ae4:	4393      	bics	r3, r2
 8001ae6:	0019      	movs	r1, r3
 8001ae8:	687b      	ldr	r3, [r7, #4]
 8001aea:	689a      	ldr	r2, [r3, #8]
 8001aec:	4b31      	ldr	r3, [pc, #196]	; (8001bb4 <HAL_RCCEx_PeriphCLKConfig+0x28c>)
 8001aee:	430a      	orrs	r2, r1
 8001af0:	64da      	str	r2, [r3, #76]	; 0x4c
  }
#endif /* RCC_CCIPR_USART1SEL */

  /*----------------------------- USART2 Configuration --------------------------*/
  if(((PeriphClkInit->PeriphClockSelection) & RCC_PERIPHCLK_USART2) == RCC_PERIPHCLK_USART2)
 8001af2:	687b      	ldr	r3, [r7, #4]
 8001af4:	681b      	ldr	r3, [r3, #0]
 8001af6:	2202      	movs	r2, #2
 8001af8:	4013      	ands	r3, r2
 8001afa:	d009      	beq.n	8001b10 <HAL_RCCEx_PeriphCLKConfig+0x1e8>
  {
    /* Check the parameters */
    assert_param(IS_RCC_USART2CLKSOURCE(PeriphClkInit->Usart2ClockSelection));

    /* Configure the USART2 clock source */
    __HAL_RCC_USART2_CONFIG(PeriphClkInit->Usart2ClockSelection);
 8001afc:	4b2d      	ldr	r3, [pc, #180]	; (8001bb4 <HAL_RCCEx_PeriphCLKConfig+0x28c>)
 8001afe:	6cdb      	ldr	r3, [r3, #76]	; 0x4c
 8001b00:	220c      	movs	r2, #12
 8001b02:	4393      	bics	r3, r2
 8001b04:	0019      	movs	r1, r3
 8001b06:	687b      	ldr	r3, [r7, #4]
 8001b08:	68da      	ldr	r2, [r3, #12]
 8001b0a:	4b2a      	ldr	r3, [pc, #168]	; (8001bb4 <HAL_RCCEx_PeriphCLKConfig+0x28c>)
 8001b0c:	430a      	orrs	r2, r1
 8001b0e:	64da      	str	r2, [r3, #76]	; 0x4c
  }

  /*------------------------------ LPUART1 Configuration ------------------------*/
  if(((PeriphClkInit->PeriphClockSelection) & RCC_PERIPHCLK_LPUART1) == RCC_PERIPHCLK_LPUART1)
 8001b10:	687b      	ldr	r3, [r7, #4]
 8001b12:	681b      	ldr	r3, [r3, #0]
 8001b14:	2204      	movs	r2, #4
 8001b16:	4013      	ands	r3, r2
 8001b18:	d009      	beq.n	8001b2e <HAL_RCCEx_PeriphCLKConfig+0x206>
  {
    /* Check the parameters */
    assert_param(IS_RCC_LPUART1CLKSOURCE(PeriphClkInit->Lpuart1ClockSelection));

    /* Configure the LPUAR1 clock source */
    __HAL_RCC_LPUART1_CONFIG(PeriphClkInit->Lpuart1ClockSelection);
 8001b1a:	4b26      	ldr	r3, [pc, #152]	; (8001bb4 <HAL_RCCEx_PeriphCLKConfig+0x28c>)
 8001b1c:	6cdb      	ldr	r3, [r3, #76]	; 0x4c
 8001b1e:	4a2c      	ldr	r2, [pc, #176]	; (8001bd0 <HAL_RCCEx_PeriphCLKConfig+0x2a8>)
 8001b20:	4013      	ands	r3, r2
 8001b22:	0019      	movs	r1, r3
 8001b24:	687b      	ldr	r3, [r7, #4]
 8001b26:	691a      	ldr	r2, [r3, #16]
 8001b28:	4b22      	ldr	r3, [pc, #136]	; (8001bb4 <HAL_RCCEx_PeriphCLKConfig+0x28c>)
 8001b2a:	430a      	orrs	r2, r1
 8001b2c:	64da      	str	r2, [r3, #76]	; 0x4c
  }

  /*------------------------------ I2C1 Configuration ------------------------*/
  if(((PeriphClkInit->PeriphClockSelection) & RCC_PERIPHCLK_I2C1) == RCC_PERIPHCLK_I2C1)
 8001b2e:	687b      	ldr	r3, [r7, #4]
 8001b30:	681b      	ldr	r3, [r3, #0]
 8001b32:	2208      	movs	r2, #8
 8001b34:	4013      	ands	r3, r2
 8001b36:	d009      	beq.n	8001b4c <HAL_RCCEx_PeriphCLKConfig+0x224>
  {
    /* Check the parameters */
    assert_param(IS_RCC_I2C1CLKSOURCE(PeriphClkInit->I2c1ClockSelection));

    /* Configure the I2C1 clock source */
    __HAL_RCC_I2C1_CONFIG(PeriphClkInit->I2c1ClockSelection);
 8001b38:	4b1e      	ldr	r3, [pc, #120]	; (8001bb4 <HAL_RCCEx_PeriphCLKConfig+0x28c>)
 8001b3a:	6cdb      	ldr	r3, [r3, #76]	; 0x4c
 8001b3c:	4a25      	ldr	r2, [pc, #148]	; (8001bd4 <HAL_RCCEx_PeriphCLKConfig+0x2ac>)
 8001b3e:	4013      	ands	r3, r2
 8001b40:	0019      	movs	r1, r3
 8001b42:	687b      	ldr	r3, [r7, #4]
 8001b44:	695a      	ldr	r2, [r3, #20]
 8001b46:	4b1b      	ldr	r3, [pc, #108]	; (8001bb4 <HAL_RCCEx_PeriphCLKConfig+0x28c>)
 8001b48:	430a      	orrs	r2, r1
 8001b4a:	64da      	str	r2, [r3, #76]	; 0x4c
  }

#if defined (RCC_CCIPR_I2C3SEL)
    /*------------------------------ I2C3 Configuration ------------------------*/
  if(((PeriphClkInit->PeriphClockSelection) & RCC_PERIPHCLK_I2C3) == RCC_PERIPHCLK_I2C3)
 8001b4c:	687b      	ldr	r3, [r7, #4]
 8001b4e:	681a      	ldr	r2, [r3, #0]
 8001b50:	2380      	movs	r3, #128	; 0x80
 8001b52:	005b      	lsls	r3, r3, #1
 8001b54:	4013      	ands	r3, r2
 8001b56:	d009      	beq.n	8001b6c <HAL_RCCEx_PeriphCLKConfig+0x244>
  {
    /* Check the parameters */
    assert_param(IS_RCC_I2C3CLKSOURCE(PeriphClkInit->I2c3ClockSelection));

    /* Configure the I2C3 clock source */
    __HAL_RCC_I2C3_CONFIG(PeriphClkInit->I2c3ClockSelection);
 8001b58:	4b16      	ldr	r3, [pc, #88]	; (8001bb4 <HAL_RCCEx_PeriphCLKConfig+0x28c>)
 8001b5a:	6cdb      	ldr	r3, [r3, #76]	; 0x4c
 8001b5c:	4a17      	ldr	r2, [pc, #92]	; (8001bbc <HAL_RCCEx_PeriphCLKConfig+0x294>)
 8001b5e:	4013      	ands	r3, r2
 8001b60:	0019      	movs	r1, r3
 8001b62:	687b      	ldr	r3, [r7, #4]
 8001b64:	699a      	ldr	r2, [r3, #24]
 8001b66:	4b13      	ldr	r3, [pc, #76]	; (8001bb4 <HAL_RCCEx_PeriphCLKConfig+0x28c>)
 8001b68:	430a      	orrs	r2, r1
 8001b6a:	64da      	str	r2, [r3, #76]	; 0x4c
  }
#endif /* RCC_CCIPR_I2C3SEL */

#if defined(USB)
 /*---------------------------- USB and RNG configuration --------------------*/
  if(((PeriphClkInit->PeriphClockSelection) & RCC_PERIPHCLK_USB) == (RCC_PERIPHCLK_USB))
 8001b6c:	687b      	ldr	r3, [r7, #4]
 8001b6e:	681b      	ldr	r3, [r3, #0]
 8001b70:	2240      	movs	r2, #64	; 0x40
 8001b72:	4013      	ands	r3, r2
 8001b74:	d009      	beq.n	8001b8a <HAL_RCCEx_PeriphCLKConfig+0x262>
  {
    assert_param(IS_RCC_USBCLKSOURCE(PeriphClkInit->UsbClockSelection));
    __HAL_RCC_USB_CONFIG(PeriphClkInit->UsbClockSelection);
 8001b76:	4b0f      	ldr	r3, [pc, #60]	; (8001bb4 <HAL_RCCEx_PeriphCLKConfig+0x28c>)
 8001b78:	6cdb      	ldr	r3, [r3, #76]	; 0x4c
 8001b7a:	4a17      	ldr	r2, [pc, #92]	; (8001bd8 <HAL_RCCEx_PeriphCLKConfig+0x2b0>)
 8001b7c:	4013      	ands	r3, r2
 8001b7e:	0019      	movs	r1, r3
 8001b80:	687b      	ldr	r3, [r7, #4]
 8001b82:	6a1a      	ldr	r2, [r3, #32]
 8001b84:	4b0b      	ldr	r3, [pc, #44]	; (8001bb4 <HAL_RCCEx_PeriphCLKConfig+0x28c>)
 8001b86:	430a      	orrs	r2, r1
 8001b88:	64da      	str	r2, [r3, #76]	; 0x4c
  }
#endif /* USB */

  /*---------------------------- LPTIM1 configuration ------------------------*/
  if(((PeriphClkInit->PeriphClockSelection) & RCC_PERIPHCLK_LPTIM1) == (RCC_PERIPHCLK_LPTIM1))
 8001b8a:	687b      	ldr	r3, [r7, #4]
 8001b8c:	681b      	ldr	r3, [r3, #0]
 8001b8e:	2280      	movs	r2, #128	; 0x80
 8001b90:	4013      	ands	r3, r2
 8001b92:	d009      	beq.n	8001ba8 <HAL_RCCEx_PeriphCLKConfig+0x280>
  {
    assert_param(IS_RCC_LPTIMCLK(PeriphClkInit->LptimClockSelection));
    __HAL_RCC_LPTIM1_CONFIG(PeriphClkInit->LptimClockSelection);
 8001b94:	4b07      	ldr	r3, [pc, #28]	; (8001bb4 <HAL_RCCEx_PeriphCLKConfig+0x28c>)
 8001b96:	6cdb      	ldr	r3, [r3, #76]	; 0x4c
 8001b98:	4a10      	ldr	r2, [pc, #64]	; (8001bdc <HAL_RCCEx_PeriphCLKConfig+0x2b4>)
 8001b9a:	4013      	ands	r3, r2
 8001b9c:	0019      	movs	r1, r3
 8001b9e:	687b      	ldr	r3, [r7, #4]
 8001ba0:	69da      	ldr	r2, [r3, #28]
 8001ba2:	4b04      	ldr	r3, [pc, #16]	; (8001bb4 <HAL_RCCEx_PeriphCLKConfig+0x28c>)
 8001ba4:	430a      	orrs	r2, r1
 8001ba6:	64da      	str	r2, [r3, #76]	; 0x4c
  }

  return HAL_OK;
 8001ba8:	2300      	movs	r3, #0
}
 8001baa:	0018      	movs	r0, r3
 8001bac:	46bd      	mov	sp, r7
 8001bae:	b006      	add	sp, #24
 8001bb0:	bd80      	pop	{r7, pc}
 8001bb2:	46c0      	nop			; (mov r8, r8)
 8001bb4:	40021000 	.word	0x40021000
 8001bb8:	40007000 	.word	0x40007000
 8001bbc:	fffcffff 	.word	0xfffcffff
 8001bc0:	fff7ffff 	.word	0xfff7ffff
 8001bc4:	00001388 	.word	0x00001388
 8001bc8:	ffcfffff 	.word	0xffcfffff
 8001bcc:	efffffff 	.word	0xefffffff
 8001bd0:	fffff3ff 	.word	0xfffff3ff
 8001bd4:	ffffcfff 	.word	0xffffcfff
 8001bd8:	fbffffff 	.word	0xfbffffff
 8001bdc:	fff3ffff 	.word	0xfff3ffff

08001be0 <HAL_UART_Init>:
  *        parameters in the UART_InitTypeDef and initialize the associated handle.
  * @param huart UART handle.
  * @retval HAL status
  */
HAL_StatusTypeDef HAL_UART_Init(UART_HandleTypeDef *huart)
{
 8001be0:	b580      	push	{r7, lr}
 8001be2:	b082      	sub	sp, #8
 8001be4:	af00      	add	r7, sp, #0
 8001be6:	6078      	str	r0, [r7, #4]
  /* Check the UART handle allocation */
  if (huart == NULL)
 8001be8:	687b      	ldr	r3, [r7, #4]
 8001bea:	2b00      	cmp	r3, #0
 8001bec:	d101      	bne.n	8001bf2 <HAL_UART_Init+0x12>
  {
    return HAL_ERROR;
 8001bee:	2301      	movs	r3, #1
 8001bf0:	e044      	b.n	8001c7c <HAL_UART_Init+0x9c>
  {
    /* Check the parameters */
    assert_param((IS_UART_INSTANCE(huart->Instance)) || (IS_LPUART_INSTANCE(huart->Instance)));
  }

  if (huart->gState == HAL_UART_STATE_RESET)
 8001bf2:	687b      	ldr	r3, [r7, #4]
 8001bf4:	6fdb      	ldr	r3, [r3, #124]	; 0x7c
 8001bf6:	2b00      	cmp	r3, #0
 8001bf8:	d107      	bne.n	8001c0a <HAL_UART_Init+0x2a>
  {
    /* Allocate lock resource and initialize it */
    huart->Lock = HAL_UNLOCKED;
 8001bfa:	687b      	ldr	r3, [r7, #4]
 8001bfc:	2278      	movs	r2, #120	; 0x78
 8001bfe:	2100      	movs	r1, #0
 8001c00:	5499      	strb	r1, [r3, r2]

    /* Init the low level hardware */
    huart->MspInitCallback(huart);
#else
    /* Init the low level hardware : GPIO, CLOCK */
    HAL_UART_MspInit(huart);
 8001c02:	687b      	ldr	r3, [r7, #4]
 8001c04:	0018      	movs	r0, r3
 8001c06:	f7fe fd45 	bl	8000694 <HAL_UART_MspInit>
#endif /* (USE_HAL_UART_REGISTER_CALLBACKS) */
  }

  huart->gState = HAL_UART_STATE_BUSY;
 8001c0a:	687b      	ldr	r3, [r7, #4]
 8001c0c:	2224      	movs	r2, #36	; 0x24
 8001c0e:	67da      	str	r2, [r3, #124]	; 0x7c

  __HAL_UART_DISABLE(huart);
 8001c10:	687b      	ldr	r3, [r7, #4]
 8001c12:	681b      	ldr	r3, [r3, #0]
 8001c14:	681a      	ldr	r2, [r3, #0]
 8001c16:	687b      	ldr	r3, [r7, #4]
 8001c18:	681b      	ldr	r3, [r3, #0]
 8001c1a:	2101      	movs	r1, #1
 8001c1c:	438a      	bics	r2, r1
 8001c1e:	601a      	str	r2, [r3, #0]

  /* Set the UART Communication parameters */
  if (UART_SetConfig(huart) == HAL_ERROR)
 8001c20:	687b      	ldr	r3, [r7, #4]
 8001c22:	0018      	movs	r0, r3
 8001c24:	f000 f8d0 	bl	8001dc8 <UART_SetConfig>
 8001c28:	0003      	movs	r3, r0
 8001c2a:	2b01      	cmp	r3, #1
 8001c2c:	d101      	bne.n	8001c32 <HAL_UART_Init+0x52>
  {
    return HAL_ERROR;
 8001c2e:	2301      	movs	r3, #1
 8001c30:	e024      	b.n	8001c7c <HAL_UART_Init+0x9c>
  }

  if (huart->AdvancedInit.AdvFeatureInit != UART_ADVFEATURE_NO_INIT)
 8001c32:	687b      	ldr	r3, [r7, #4]
 8001c34:	6a5b      	ldr	r3, [r3, #36]	; 0x24
 8001c36:	2b00      	cmp	r3, #0
 8001c38:	d003      	beq.n	8001c42 <HAL_UART_Init+0x62>
  {
    UART_AdvFeatureConfig(huart);
 8001c3a:	687b      	ldr	r3, [r7, #4]
 8001c3c:	0018      	movs	r0, r3
 8001c3e:	f000 fb61 	bl	8002304 <UART_AdvFeatureConfig>
  }

  /* In asynchronous mode, the following bits must be kept cleared:
  - LINEN and CLKEN bits in the USART_CR2 register,
  - SCEN, HDSEL and IREN  bits in the USART_CR3 register.*/
  CLEAR_BIT(huart->Instance->CR2, (USART_CR2_LINEN | USART_CR2_CLKEN));
 8001c42:	687b      	ldr	r3, [r7, #4]
 8001c44:	681b      	ldr	r3, [r3, #0]
 8001c46:	685a      	ldr	r2, [r3, #4]
 8001c48:	687b      	ldr	r3, [r7, #4]
 8001c4a:	681b      	ldr	r3, [r3, #0]
 8001c4c:	490d      	ldr	r1, [pc, #52]	; (8001c84 <HAL_UART_Init+0xa4>)
 8001c4e:	400a      	ands	r2, r1
 8001c50:	605a      	str	r2, [r3, #4]
  CLEAR_BIT(huart->Instance->CR3, (USART_CR3_SCEN | USART_CR3_HDSEL | USART_CR3_IREN));
 8001c52:	687b      	ldr	r3, [r7, #4]
 8001c54:	681b      	ldr	r3, [r3, #0]
 8001c56:	689a      	ldr	r2, [r3, #8]
 8001c58:	687b      	ldr	r3, [r7, #4]
 8001c5a:	681b      	ldr	r3, [r3, #0]
 8001c5c:	212a      	movs	r1, #42	; 0x2a
 8001c5e:	438a      	bics	r2, r1
 8001c60:	609a      	str	r2, [r3, #8]

  __HAL_UART_ENABLE(huart);
 8001c62:	687b      	ldr	r3, [r7, #4]
 8001c64:	681b      	ldr	r3, [r3, #0]
 8001c66:	681a      	ldr	r2, [r3, #0]
 8001c68:	687b      	ldr	r3, [r7, #4]
 8001c6a:	681b      	ldr	r3, [r3, #0]
 8001c6c:	2101      	movs	r1, #1
 8001c6e:	430a      	orrs	r2, r1
 8001c70:	601a      	str	r2, [r3, #0]

  /* TEACK and/or REACK to check before moving huart->gState and huart->RxState to Ready */
  return (UART_CheckIdleState(huart));
 8001c72:	687b      	ldr	r3, [r7, #4]
 8001c74:	0018      	movs	r0, r3
 8001c76:	f000 fbf9 	bl	800246c <UART_CheckIdleState>
 8001c7a:	0003      	movs	r3, r0
}
 8001c7c:	0018      	movs	r0, r3
 8001c7e:	46bd      	mov	sp, r7
 8001c80:	b002      	add	sp, #8
 8001c82:	bd80      	pop	{r7, pc}
 8001c84:	ffffb7ff 	.word	0xffffb7ff

08001c88 <HAL_UART_Transmit>:
  * @param Size    Amount of data elements (u8 or u16) to be sent.
  * @param Timeout Timeout duration.
  * @retval HAL status
  */
HAL_StatusTypeDef HAL_UART_Transmit(UART_HandleTypeDef *huart, const uint8_t *pData, uint16_t Size, uint32_t Timeout)
{
 8001c88:	b580      	push	{r7, lr}
 8001c8a:	b08a      	sub	sp, #40	; 0x28
 8001c8c:	af02      	add	r7, sp, #8
 8001c8e:	60f8      	str	r0, [r7, #12]
 8001c90:	60b9      	str	r1, [r7, #8]
 8001c92:	603b      	str	r3, [r7, #0]
 8001c94:	1dbb      	adds	r3, r7, #6
 8001c96:	801a      	strh	r2, [r3, #0]
  const uint8_t  *pdata8bits;
  const uint16_t *pdata16bits;
  uint32_t tickstart;

  /* Check that a Tx process is not already ongoing */
  if (huart->gState == HAL_UART_STATE_READY)
 8001c98:	68fb      	ldr	r3, [r7, #12]
 8001c9a:	6fdb      	ldr	r3, [r3, #124]	; 0x7c
 8001c9c:	2b20      	cmp	r3, #32
 8001c9e:	d000      	beq.n	8001ca2 <HAL_UART_Transmit+0x1a>
